:100000000C9414080C9445080C9445080C9445086D
:100010000C9445080C9445080C9445080C9445082C
:100020000C9445080C9445080C9445080C9445081C
:100030000C9445080C94AC710C9445080C9445083C
:100040000C9445080C9445080C9445080C944508FC
:100050000C9445080C9445080C9445080C945A8F50
:100060000C9445080C9443930C9479930C94450894
:100070000C9445080C9445080C9445080C944508CC
:100080000C9445080C9445080C944508FEC70000E4
:100090000C94EE930C942494F8C700000C94898778
:1000A000F4C70000F2C70000F0C70000EEC7000070
:1000B000ECC70000EAC70000E8C70000E6C7000080
:1000C000E4C70000E2C70000E0C700000C94999468
:1000D0000C94CF94DAC700000C9444950C947A9554
:1000E000D4C70000AA508A50B350B350B350B35095
:1000F000B350B350B350B350B350B350E14EF34E7E
:10010000FA4E004F074F0D4F124F1B4F224F394FE2
:100110003C4FB3504E4F514F544F574F714F734F49
:100120007A4F814F944F9B4FA24FB350B350B3506F
:10013000B350B350B350B350B350B350B350DD4F7E
:10014000B350B350B350B350B350B350E150A79035
:10015000AA9099909D90A390E190AE90B290B890A3
:10016000BC90C090C690CA90CE90E190D490D890A8
:10017000DC90084AD73B3BCE016E84BCBFFDC12F4B
:100180003D6C74319ABD56833DDA3D00C77F11BE88
:10019000D9E4BB4C3E916BAAAABE000000803F0789
:1001A000634236B79BD8A71A39685618AEBAAB5512
:1001B0008C1D3CB7CC5763BD6DEDFD753EF61772D7
:1001C00031BF000000803F08000000BE92244912A9
:1001D0003EABAAAA2ABECDCCCC4C3E00000080BECD
:1001E000ABAAAAAA3E00000000BF000000803F00AA
:1001F00000000000084178D3BB4387D1133D190E9E
:100200003CC3BD4282AD2B3E68EC8276BED98FE105
:10021000A93E4C80EFFFBE01C4FF7F3F00000000FD
:1002200000004D6F74696F6E004D6F74696F6E00E2
:10023000696E7075742044535463616C69627261B5
:1002400074653A004E6F2053656E736F7221004ED5
:100250006F20445320546865726D6F6D65746572CC
:100260002100445320546865726D2E005556204974
:100270006E742E00555620496E74656E73697479DC
:1002800000234E6F2073656E736F722100536F757C
:100290006E64204C6576656C004D6561737572699E
:1002A0006E672E2E00234E6F2073656E736F722162
:1002B00000536F756E64204C6576656C00234E6F3D
:1002C0002073656E736F7220666F7220504D21002F
:1002D0004E6F2073656E736F722100206E672F4C16
:1002E00000504D313A322E353A3130004D65617350
:1002F0007572696E672E2E004F3220436F6E630059
:10030000434F3220436F6E630053656E736F7220EC
:100310006572726F722100234E6F2073656E736F6A
:10032000722100434F3220436F6E63004D6561734D
:100330007572696E6700234E6F2070482073656E7A
:10034000736F72210070482076616C756500234ED2
:100350006F2054422073656E736F723F004E6F20A2
:1003600073656E736F72210049522054656D70651C
:10037000726174757265004D6561737572696E673F
:100380002E2E004E6F2073656E736F723F004952C0
:100390002054656D7065726174757265004D65619C
:1003A000737572696E672E2E004C696768742049F8
:1003B0006E74656E7369747900416E676C65732F36
:1003C000003E6128782C792C7A292F673A006765DE
:1003D0007453656C665465737442697428293A20B5
:1003E000006973496E74657272757074456E6162EE
:1003F0006C65642831293A2000676574496E74651C
:1004000072727570744D617070696E672831293A27
:100410002000676574496E74657272757074536FED
:10042000757263652831293A2000676574496E74D6
:10043000657272757074536F7572636528293A20FE
:10044000006765745261746528293A20332E31346F
:100450003135393F00616363656C2E69734C6F778A
:10046000506F77657228293A2000616363656C2EAE
:10047000697341736C65657028293A200061636374
:10048000656C2E6973546170536F757263654F6E3E
:100490005A28293A2000616363656C2E69735461A0
:1004A00070536F757263654F6E5928293A20006149
:1004B0006363656C2E6973546170536F7572636505
:1004C0004F6E5828293A2000616363656C2E69736A
:1004D0004163746976697479536F757263654F6EA1
:1004E0005A28293A2000616363656C2E6973416361
:1004F000746976697479536F757263654F6E5928A4
:10050000293A200069734163746976697479536F7D
:10051000757263654F6E5828293A200069735461DB
:1005200070446574656374696F6E4F6E5A28293B19
:100530002066616C73653F20006973546170446587
:1005400074656374696F6E4F6E5A28293B2074720C
:1005500075653F2000697354617044657465637408
:10056000696F6E4F6E5928293B2066616C73653F39
:1005700020006973546170446574656374696F6EBB
:100580004F6E5928293B20747275653F20006973AE
:10059000546170446574656374696F6E4F6E58285A
:1005A000293B2066616C73653F200069735461705C
:1005B000446574656374696F6E4F6E5828293B20DB
:1005C000747275653F20006765745375707072654D
:1005D000737342697428293B2066616C73653F2000
:1005E000006765745375707072657373426974281F
:1005F000293B20747275653F2000697341637469FB
:1006000076697479416328293A20006973496E61DB
:10061000637469766974795A456E61626C656428A1
:10062000293A20006973496E616374697669747947
:1006300059456E61626C656428293A2000697349E6
:100640006E616374697669747958456E61626C6530
:100650006428293A20006973416374697669747962
:100660005A456E61626C656428293A2000697341BD
:100670006374697669747959456E61626C65642842
:10068000293A200069734163746976697479584521
:100690006E61626C656428293A2000676574467251
:1006A000656546616C6C4475726174696F6E28296A
:1006B0003A20006765744672656546616C6C5468E3
:1006C000726573686F6C6428293A200067657454FA
:1006D000696D65496E616374697669747928293A30
:1006E0002000676574496E61637469766974795432
:1006F00068726573686F6C642829200067657441AF
:10070000637469766974795468726573686F6C6430
:1007100028292000676574446F75626C65546170A8
:1007200057696E646F7728292000676574446F7578
:10073000626C655461704C6174656E637928293A06
:1007400020006765745461704475726174696F6EDE
:1007500028293A2000676574417869734F6666738B
:1007600065742826782C2026792C20267A293A2090
:10077000006765745461705468726573686F6C6467
:1007800028293A200058595A2047733A20005859CE
:100790005A20434F554E54533A20007365742067D6
:1007A00061696E735B5D3A006761696E735F6F725A
:1007B00069675B5D3A00466C616D65204952004F88
:1007C0006666206169722D636F6E6421004974272B
:1007D0007320746F6F20636F6F6C210054656D70B0
:1007E0002069732066696E65210049732061697212
:1007F0002D636F6E64206F6E3F0049742773207104
:100800007569746520686F742100497427732076B8
:1008100065727920686F74210054656D7020487589
:100820006D696469747900234E6F2073656E736F10
:100830007220666F722074656D7020262068756D59
:10084000696469747921004E6F2053656E736F720D
:10085000210020666F722074656D702026206875F7
:100860006D696469747921002353656E736F72201A
:100870004572726F72200053656E736F72204572FD
:10088000726F7221002357726F6E672073656E73EB
:100890006F7220666F722074656D702026206875F7
:1008A0006D6964697479210057726F6E67205365B2
:1008B0006E736F72210054656D702048756D6964A8
:1008C000697479004F6666206169722D636F6E648A
:1008D00021004974277320746F6F20636F6F6C2140
:1008E0000054656D702069732066696E652100494A
:1008F00073206169722D636F6E64206F6E3F0049D3
:1009000074277320717569746520686F74210049BC
:10091000742773207665727920686F742120002314
:10092000616E6F7468657220495220696E707574CB
:100930003D00496E76616C6964206B657921002306
:100940007265706C6965733D0054696D65206C61FA
:100950007073653A00233A53686F772F486964656E
:10096000204C4344002A3A546869732048656C70EF
:100970000044433A436C656172204C434400444256
:100980003A5265736574204C6F676765720044372F
:100990003A4D6F74696F6E0044363A445320546583
:1009A0006D700044353A555620496E74656E736912
:1009B00074790044343A4F3220636F6E632E0044E2
:1009C000333A434F3220636F6E632E0044323A5005
:1009D0004D28313A322E353A3130290044323A50DE
:1009E0004D28313A322E353A3130292A0044313AF5
:1009F0005475726269646974790044303A566F6C58
:100A00007461676500393A6F722033442061636313
:100A1000656C2E00393A496E636C2E20616E672E2C
:100A200000383A70482076616C756500373A495253
:100A30002054656D7000373A49522054656D702A14
:100A400000363A4D61676E65746963206669656C4E
:100A50006400353A476173204C6576656C00343A22
:100A6000495220466C616D6500333A4C6967687481
:100A700020496E742E00323A616E642048656967C1
:100A8000687400323A54656D7020507265737375E6
:100A9000726500313A54656D702048756D696469FE
:100AA000747900303A536F756E64204C6576656CCE
:100AB00000303A536F756E64204C6576656C2A0081
:100AC0002020202020202020202020202020200046
:100AD0002020202020202020202020202020200036
:100AE0002020202020202020202020202020202006
:100AF0000020202020202020202020202020202016
:100B00002000202020202020202020202020202005
:100B100020200020202020202020202020202020F5
:100B200020202000482D6669656C643A2028004C1E
:100B30006F6767657220446972656374696F6E00E0
:100B4000482D6669656C6400536561726368204472
:100B50006972656374696F6E00232D2D2D2D2D2D07
:100B60002D2D2D2D2D2D2D2D2D2D2D2D2D2D2D2DB5
:100B70002D2D2D2D2D2D2D2D2D2D2D2D2D2D0023DC
:100B80005265736F6C7574696F6E3A202020002374
:100B90004D696E2056616C75653A20202020002337
:100BA0004D61782056616C75653A20202020002325
:100BB000556E697175652049443A20202020002334
:100BC000447269766572205665723A2020200023AF
:100BD00053656E736F723A2020202020202000235E
:100BE0002D2D2D2D204D61676E6574696320536531
:100BF0006E736F72202D2D2D2D2D2D2D2D2D2D2D24
:100C00002D2D2D2D2D2D2D2D2D006E6F20484D437A
:100C100035383833206D61676E657469632073659C
:100C20006E736F72202E2E2E20436865636B2077C3
:100C30006972696E672100236B65793D0020766FCC
:100C40006C746167653D00235475726269646974F0
:100C500079205570706572204C696D69743A200076
:100C600020766F6C746167653D002354757262690C
:100C700064697479204C6F776572204C696D697472
:100C80003A200023547572626964697479204C6F4C
:100C9000776572204C696D69742056696E663A20DA
:100CA0000023434F32204D415820766F6C7420282A
:100CB0000023434F32207A65726F20766F6C742068
:100CC0002800234F322063616C6962726174696F1E
:100CD0006E3A200023547572626964697479204CFD
:100CE0006F776572204C696D69742056313A200027
:100CF00043616C6962726174696F6E2050726573D2
:100D0000737572653D00536561206C6576656C2076
:100D1000502863616C63293D00234572726F723AFB
:100D2000707265737375726520424D503038352C82
:100D300020636865636B20776972696E672100497B
:100D4000522054656D702073656E736F7220666FEC
:100D5000756E6400504D322E352073656E736F7260
:100D6000206C696B656C7920666F756E64004564F4
:100D700055484B205345534C6F6767657200536568
:100D80006E736F7220736C6F7420616E642074795F
:100D900070653A0057656C636F6D6520746F204510
:100DA0006455484B00005EBCE2613FDD83C29C7E1F
:100DB00020A3FD1F41009D23BE46DB65F88C11AFCB
:100DC00032CA57E97400000A0B02090C0D0E08071D
:100DD000030401000000000000000000000000000B
:100DE0000000000000000000000000000000000003
:100DF00000121110000000000000000000000000C0
:100E0000000000000000000000000001021020208F
:100E1000080810204010204080020102010804024E
:100E200001010204081020408080402010080402C4
:100E3000018004020180402010080402010804021D
:100E40000101020408102040800102040810204023
:100E50008005050505070508080808020202020AC0
:100E60000A0808040404040101010101010101034D
:100E700003030303030303040707070C0C0C0C0C08
:100E80000C0C0C0202020206060606060606060BFB
:100E90000B0B0B0B0B0B0B00002000230026002973
:100EA000002C002F003200000100000301060109A0
:100EB0000100002200250028002B002E0031003404
:100EC0000002010000050108010B010000210024BF
:100ED0000027002A002D003000330001010000042B
:100EE0000107010A014E414E494E495459494E46A7
:100EF000CDCCCC3D0AD7233C17B7D13877CC2B3299
:100F00009595E6241FB14F0A000020410000C84219
:100F100000401C4620BCBE4CCA1B0E5AAEC59D7478
:100F200000407A10F35A00A0724E18090010A5D4A0
:100F3000E80000E87648170000E40B54020000CAFD
:100F40009A3B000000E1F505000080969800000043
:100F500040420F000000A0860100000010270000A2
:100F60000000E803000000006400000000000A0028
:100F7000000000000100000000002C76D888DC672B
:100F80004F0823DFC1DFAE59E1B1B796E5E3E45383
:100F9000C63AE651997696E8E6C28426EB898C9BA0
:100FA00062ED407C6FFCEFBC9C9F40F2BAA56FA540
:100FB000F490055A2AF75C936B6CF9676DC11BFCC2
:100FC000E0E40D47FEF520E6B500D0ED902E0300DD
:100FD000943577050080841E080000204E0A00002A
:100FE00000C80C333333330F986E12831141EF8DE9
:100FF0002114893BE65516CFFEE6DB18D1844B3829
:101000001BF77C1D901DA4BBE424203284725E2259
:101010008100C9F124ECA1E53D275D3AA086AB93A0
:1010200056940195AC95FE3A11241FBECFEFD1E244
:10103000DEBFCDBF00E00CBF1BE0A0E0B2E0EAE104
:10104000F5E501E00BBF02C007900D92A834B1078F
:10105000D9F722E1A8E4BBE001C01D92A830B20795
:10106000E1F710E1C6E2D0E100E006C022970109F5
:10107000FE010BBF0E94F6A2CA31D10780E008072B
:10108000A9F70E94249E0C947CAA0C940000CF9295
:10109000DF92EF92FF920F931F93E82FF92F05C075
:1010A000015011092109310961F1908196239417AA
:1010B000B9F305C0015011092109310911F19081DD
:1010C00096239413F7CFC12CD12CE12CF12C0AC01C
:1010D0008FEFC81AD80AE80AF80A0C151D052E0564
:1010E0003F0579F080818623841791F36C2D7D2D47
:1010F0008E2D9F2D1F910F91FF90EF90DF90CF903D
:10110000089560E070E080E090E01F910F91FF9003
:10111000EF90DF90CF9008952FE53AE0FC01318306
:101120002083089508952FE53AE0FC013183208360
:101130000C94329E2F923F924F925F926F927F92C9
:101140008F929F92AF92BF92CF92DF92EF92FF92D7
:101150000F931F93CF93DF93CDB7DEB72E970FB6C4
:10116000F894DEBF0FBECDBF8C017E876D87DC019A
:101170004D915C91119712962D913C9113974217C6
:1011800053072CF4942F852FA901292F382FD8012C
:10119000149660E070E0CB01E2E0F0E0ED84FE84C4
:1011A000EE15FF0544F5CD90DD90C216D3065CF434
:1011B0004901AA2497FCA094BA2C680D791D8A1DB8
:1011C0009B1D960116C04C155D055CF44A01AA24CE
:1011D00097FCA094BA2C680D791D8A1D9B1DA60151
:1011E00008C0EE24D7FCE094FE2C6C0D7D1D8E1DF6
:1011F0009F1D3196D3CF0E94CB9F6B017C016D85E3
:101200007E8562507109882777FD8095982F0E940E
:10121000CB9F9B01AC01C701B6010E94FF9E6B01F1
:101220007C012D853E85243131050CF4BFC0480179
:10123000412C512C3201A12CB12CD4016D917D9106
:101240004D01882777FD8095982F0E94CB9FA7019D
:1012500096010E94349E9B01AC010E945FA19B01FC
:10126000AC01C301B2010E94359E2B013C01BFEFCE
:10127000AB1ABB0AED85FE85AE16BF06F1F6BF01BF
:1012800061507109882777FD8095982F0E94CB9F28
:101290009B01AC01C301B2010E94FF9E0E9412A2F9
:1012A0004B015C0120E030E040E85FE30E94A0A039
:1012B00018160CF07BC018870F83212C312C1B8251
:1012C0001C821D821E821A821982AF81B8858D917F
:1012D0009D91B887AF839C01442737FD4095542FDB
:1012E00029873A874B875C87CA01B9010E94CB9F47
:1012F000A70196010E94349E2B013C0120E030E0C2
:10130000A9010E94A0A0181624F0C301B2019058B0
:1013100002C0C301B201A50194010E94FB9E87FF98
:1013200013C08B819C81AD81BE8129853A854B8517
:101330005C85820F931FA41FB51F8B839C83AD8395
:10134000BE833FEF231A330A49815A814F5F5F4FB3
:101350005A8349838D859E854817590709F0B5CF73
:1013600020E030E040EC5FE3C501B4010E945FA1E2
:101370004B015C0195E0291631040CF49CCF6B8184
:101380007C818D819E810E94CB9F6B017C01B1018C
:10139000882777FD8095982F0E94CB9F9B01AC01F9
:1013A000C701B6010E94FF9E6B017C01C701B60117
:1013B0002E960FB6F894DEBF0FBECDBFDF91CF9152
:1013C0001F910F91FF90EF90DF90CF90BF90AF9063
:1013D0009F908F907F906F905F904F903F902F9055
:1013E0000895CF93DF93EC01FB01248135810E94A6
:1013F0006F9DCE01DF91CF91089526E00C94B092BD
:10140000DC01ED91FC910190F081E02D1994EF92B7
:10141000FF920F931F93CF93DF931F92CDB7DEB749
:101420007C01FC0100811181C80169830E947BA6B7
:101430006981681719F0C8010E9483A6C7010F903F
:10144000DF91CF911F910F91FF90EF900895EF9250
:10145000FF920F931F93CF93DF931F921F92CDB7ED
:10146000DEB70BE81BE08B589B407C01C701800F67
:10147000911FF80161918F019A838983CE010196B2
:10148000C6DFFCE001311F0789F78BE89BE00F9076
:101490000F90DF91CF911F910F91FF90EF900895E2
:1014A0000F931F93CF93DF931F921F92CDB7DEB799
:1014B00002EF1DE0F80160818EED93E09A8389834D
:1014C000CE010196A4DFF80161818FED93E09A834C
:1014D0008983CE0101969BDFC8010F900F90DF91A9
:1014E000CF911F910F9108950F931F93CF93DF9387
:1014F00000D000D0CDB7DEB78C018091AF0C88232F
:10150000A1F061EB76E0CE0101960E94189AB80135
:10151000CE0101960E943F9CBC018EE89FE00E9494
:101520007996CE0101960E94AD9926960FB6F89451
:10153000DEBF0FBECDBFDF91CF911F910F910895F8
:10154000AF92BF92CF92DF92EF92FF921F93CF9311
:10155000DF93CDB7DEB762970FB6F894DEBF0FBE4C
:10156000CDBF6C017B015A018091FB04882309F4F3
:101570008CC08091FA04882309F487C077FF09C0E2
:10158000E094F09440E06E2D82EE9DE00E94C86FE2
:1015900058C040E060E082EE9DE00E94C86F0E946B
:1015A000A48F28EE33E040E050E00E94C4A2CA01BC
:1015B000B9012091F6043091F7044091F80450915C
:1015C000F9040E94C4A2AB01BC012AE0CE0101963D
:1015D0000E940E9BBE016F5F7F4FCE0107960E9457
:1015E000979A62E578E0CE0107960E94509CBC0174
:1015F000CE010D960E94979ACE0107960E94AD9952
:10160000CE0101960E94AD99BE01635F7F4F82EECD
:101610009DE00E945096198940E0612F82EE9DE086
:101620000E94C86FE114F10411F4E12E06C040E0FD
:101630006E2D82EE9DE00E94C86FCE010D960E9435
:10164000AD99B60182EE9DE00E94509663E17BE089
:1016500082EE9DE00E942D96F60164816E0D40E0C1
:1016600082EE9DE00E94C86F0E94A48F6093DE0D01
:101670007093DF0D8093E00D9093E10DB501882705
:1016800077FD8095982F0E94D38F62960FB6F894BD
:10169000DEBF0FBECDBFDF91CF911F91FF90EF90C6
:1016A000DF90CF90BF90AF9008954F925F926F926E
:1016B0007F92AF92BF92CF92DF92EF92FF920F9301
:1016C0001F93CF93DF93CDB7DEB762970FB6F89431
:1016D000DEBF0FBECDBF6C017B015A018091FB04C0
:1016E000882309F4A4C08091FA04882309F49FC0D8
:1016F0000E94A48F0091DE0D1091DF0D2091E00D6E
:101700003091E10D4090EA045090EB046090EC04BD
:101710007090ED04040D151D261D371D06171707C3
:101720002807390708F083C0F7FE0AC08701009533
:10173000109540E0602F82EE9DE00E94C86F53C07C
:1017400040E060E082EE9DE00E94C86F0E94A48F9E
:1017500028EE33E040E050E00E94C4A2CA01B90183
:101760002091F6043091F7044091F8045091F90467
:101770000E94C4A2AB01BC012AE0CE0101960E94E6
:101780000E9BBE016F5F7F4FCE0107960E94979A16
:1017900062E578E0CE0107960E94509CBC01CE0124
:1017A0000D960E94979ACE0107960E94AD99CE01A0
:1017B00001960E94AD99BE01635F7F4F82EE9DE06E
:1017C0000E94509609891A89E114F10441F00E0D26
:1017D0001F1D40E0602F82EE9DE00E94C86FCE0189
:1017E0000D960E94AD99B60182EE9DE00E94509642
:1017F00062E07BE082EE9DE00E942D96F60164811E
:10180000600F40E082EE9DE00E94C86F0E94A48FAE
:101810006093DE0D7093DF0D8093E00D9093E10DEA
:10182000B501882777FD8095982F0E94D38F629607
:101830000FB6F894DEBF0FBECDBFDF91CF911F91E1
:101840000F91FF90EF90DF90CF90BF90AF907F907F
:101850006F905F904F9008958F929F92AF92BF923A
:10186000CF92DF92EF92FF920F931F93CF93DF936C
:101870007C016B01EA018091FB04882309F474C0A8
:101880008091FA04882309F46FC077FF1CC0C094CC
:10189000D09441E06C2D82EE9DE00E94C86FB701AC
:1018A00082EE9DE00E94509661EF7AE082EE9DE02C
:1018B0000E942D96F70164816C0D41E082EE9DE05F
:1018C0000E94C86F3EC00E94A48F0091EA0410914C
:1018D000EB042091EC043091ED048090DA0D9090AF
:1018E000DB0DA090DC0DB090DD0D080D191D2A1D3B
:1018F0003B1D0617170728073907B0F541E06C2D87
:1019000082EE9DE00E94C86FB70182EE9DE00E94CA
:10191000509660EE7AE082EE9DE00E942D96F701EF
:1019200064816C0D41E082EE9DE00E94C86F0E94D0
:10193000A48F6093DA0D7093DB0D8093DC0D909390
:10194000DD0DBE01882777FD8095982FDF91CF911F
:101950001F910F91FF90EF90DF90CF90BF90AF90CD
:101960009F908F900C94D38FDF91CF911F910F9107
:10197000FF90EF90DF90CF90BF90AF909F908F90AF
:1019800008958091FB04882379F08091FA048823DC
:1019900059F06FED82EE9DE00E945F9668E875E079
:1019A00082EE9DE00C945E960895CF93DF93EC0158
:1019B0008091FB048823A1F08091FA04882381F0B0
:1019C0006FED82EE9DE00E945F968C819D81892B58
:1019D00039F0BE0182EE9DE0DF91CF910C945096DC
:1019E000DF91CF9108958091FB04882301F18091CC
:1019F000FA048823E1F082EE9DE00E94BC6F40E093
:101A000060E082EE9DE00E94C86F60ED7AE082EEB9
:101A10009DE00E942D9641E060E082EE9DE00E94F4
:101A2000C86F60EC7AE082EE9DE00C942D960895EC
:101A30004F925F926F927F928F929F92AF92BF92DE
:101A4000CF92DF92EF92FF920F931F93CF93DF938A
:101A5000CDB7DEB76E970FB6F894DEBF0FBECDBF21
:101A60008C010E94A48F28EEC22E23E0D22EE12CFE
:101A7000F12CA70196010E94A2A28090F6049090FA
:101A8000F704A090F804B090F904CA01B901A501C7
:101A900094010E94A2A249015A010E94A48FA701A9
:101AA00096010E94A2A2C090F604D090F704E090A4
:101AB000F804F090F904CA01B901A70196010E9447
:101AC000A2A220E13EE040E050E00E94C4A26901F1
:101AD0007A012CE330E040E050E00E94C4A22901EA
:101AE0003A01AB01BC012AE0CE0101960E940E9B97
:101AF0002AE0B301A201CE0107960E940E9B2AE0C4
:101B0000B701A601CE010D960E940E9B2AE0B501F9
:101B1000A401CE0149960E940E9BBE01675E7F4FD5
:101B2000CE0143960E94979A62E175E0CE014396FA
:101B30000E94509CBE01635F7F4F0E943F9C65E105
:101B400075E00E94509CBE01695F7F4F0E943F9CE0
:101B500068E175E00E94509CBE016F5F7F4F0E945C
:101B60003F9C66E876E00E94509CBC01C8010E9440
:101B7000979ACE0143960E94AD99CE0149960E9454
:101B8000AD99CE010D960E94AD99CE0107960E94A7
:101B9000AD99CE0101960E94AD99C8016E960FB61F
:101BA000F894DEBF0FBECDBFDF91CF911F910F9193
:101BB000FF90EF90DF90CF90BF90AF909F908F906D
:101BC0007F906F905F904F900895CF93DF93CDB744
:101BD000DEB72C970FB6F894DEBF0FBECDBF809155
:101BE000010C9091020C892B01F56BE175E0CE019F
:101BF00007960E94189A6EEC7DE0CE0107960E942F
:101C00003F9CBC01CE0101960E94979A48EC50E09F
:101C10006FEF7FEFCE01019693DCCE0101960E941B
:101C2000AD99CE0107960E94AD998091010C9091DB
:101C3000020C019701F56FE175E0CE0107960E9455
:101C4000189A6EEC7DE0CE0107960E943F9CBC0185
:101C5000CE0101960E94979A48EC50E06FEF7FEF1B
:101C6000CE0101966DDCCE0101960E94AD99CE01A8
:101C700007960E94AD9965E275E0CE0107960E9435
:101C8000189A68EC7DE0CE0107960E943F9CBC014B
:101C9000CE0101960E94979A40ED57E06FEF7FEFDB
:101CA000CE010196D9DDCE0101960E94AD99CE01FB
:101CB00007960E94AD998091F00D9091F10D0197DA
:101CC00019F461EB7AE002C063EA7AE0CE01019692
:101CD0000E94B69B48EC50E06FEF7FEFCE0101967B
:101CE000E4DCCE0101960E94AD9963E97AE0CE0171
:101CF00001960E94B69B40ED57E06FEF7FEFCE015B
:101D00000196AADDCE0101960E94AD9963E87AE0C2
:101D1000CE0101960E94B69B48EC50E06FEF7FEF3A
:101D2000CE010196C2DCCE0101960E94AD9966E714
:101D30007AE0CE0101960E94B69B40ED57E06FEF2E
:101D40007FEFCE01019688DDCE0101960E94AD990C
:101D500069E67AE0CE0101960E94B69B48EC50E01D
:101D60006FEF7FEFCE010196A0DCCE0101960E94BD
:101D7000AD996EE57AE0CE0101960E94B69B40EDEA
:101D800057E06FEF7FEFCE01019666DDCE01019641
:101D90000E94AD9962E57AE0CE0101960E94B69B61
:101DA00048EC50E06FEF7FEFCE0101967EDCCE0174
:101DB00001960E94AD9961E47AE0CE0101960E94FD
:101DC000B69B40ED57E06FEF7FEFCE01019644DD0B
:101DD000CE0101960E94AD998091F00D9091F10D88
:101DE000039719F466E37AE002C06CE27AE0CE0170
:101DF00001960E94B69B48EC50E06FEF7FEFCE015A
:101E0000019653DCCE0101960E94AD9961E27AE021
:101E1000CE0101960E94B69B40ED57E06FEF7FEF39
:101E2000CE01019619DDCE0101960E94AD9964E1C3
:101E30007AE0CE0101960E94B69B48EC50E06FEF2D
:101E40007FEFCE01019631DCCE0101960E94AD9963
:101E500065E07AE0CE0101960E94B69B40ED57E026
:101E60006FEF7FEFCE010196F7DCCE0101960E9465
:101E7000AD996AEF79E0CE0101960E94B69B48ECDD
:101E800050E06FEF7FEFCE0101960FDCCE0101969F
:101E90000E94AD996DEE79E0CE0101960E94B69B4D
:101EA00040ED57E06FEF7FEFCE010196D5DCCE011C
:101EB00001960E94AD998091F00D9091F10D0297DD
:101EC00019F46CED79E002C06CEC79E0CE0101967A
:101ED0000E94B69B48EC50E06FEF7FEFCE01019679
:101EE000E4DBCE0101960E94AD996FEB79E0CE0163
:101EF00001960E94B69B40ED57E06FEF7FEFCE0159
:101F00000196AADCCE0101960E94AD9963EB79E0BF
:101F1000CE0101960E94B69B48EC50E06FEF7FEF38
:101F2000CE010196C2DBCE0101960E94AD9963EA13
:101F300079E0CE0101960E94B69B40ED57E06FEF2D
:101F40007FEFCE01019688DCCE0101960E94AD990B
:101F500068E979E0CE0101960E94B69B48EC50E01A
:101F60006FEF7FEFCE010196A0DBCE0101960E94BC
:101F7000AD996EE879E0CE0101960E94B69B40EDE6
:101F800057E06FEF7FEFCE01019666DCCE01019640
:101F90000E94AD996EE779E0CE0101960E94B69B52
:101FA00048EC50E06FEF7FEFCE0101967EDBCE0173
:101FB00001960E94AD9961E779E0CE0101960E94F9
:101FC000B69B40ED57E06FEF7FEFCE01019644DC0A
:101FD000CE0101960E94AD9965E679E0CE010196A9
:101FE0000E94B69B48EC50E06FEF7FEFCE01019668
:101FF0005CDBCE0101960E94AD9965E579E0CE01EA
:1020000001960E94B69B40ED57E06FEF7FEFCE0147
:10201000019622DCCE0101960E94AD9969E479E037
:10202000CE0101960E94B69B48EC50E06FEF7FEF27
:10203000CE0101963ADBCE0101960E94AD99CE0108
:102040000196F6DC40ED57E06FEF7FEFCE01019691
:1020500003DCCE0101960E94AD992C960FB6F89440
:10206000DEBF0FBECDBFDF91CF9108954F925F923B
:102070006F927F928F929F92AF92BF92CF92DF9298
:10208000EF92FF92CF93DF93CDB7DEB72C970FB6C9
:10209000F894DEBF0FBECDBFA6DC82EE9CE00E94AE
:1020A000116A2B013C0182EE9CE00E94A2694B0167
:1020B0005C01609138027091390280913A029091EE
:1020C0003B020E94CB9FAB01BC0182EE9CE00E94D0
:1020D000AE6B6B017C01C301B2010E94CB9F20E07B
:1020E00030E048EC52E40E94FF9EAB01BC0122E0CC
:1020F000CE0101960E943A9BBE016F5F7F4F84EB39
:102100009CE00E949F9ACE0101960E94AD9961EEDB
:1021100078E084EB9CE00E94EF9B64EB7CE08AEB30
:102120009CE00E94829A6DED78E0CE0101960E94BB
:10213000189A64EB7CE0CE0101960E943F9CBC01A2
:1021400084EB9CE00E94829ACE0101960E94AD9998
:1021500062E476E080EC9CE00E94B59A21E0B50153
:10216000A401CE0101960E943A9BBE016F5F7F4F92
:1021700080EC9CE00E94E99BCE0101960E94AD9903
:102180006AE275E080EC9CE00E94EF9B21E0B701E1
:10219000A601CE0107960E943A9BBE01695F7F4F60
:1021A000CE0101960E94979A60E077E0CE010196F9
:1021B0000E94509CBC0180EC9CE00E94E99BCE01F7
:1021C00001960E94AD99CE0107960E94AD9964EBED
:1021D0007CE0CE0101960E94979A61E475E0CE0101
:1021E00001960E94509C60EC7CE00E943F9CBC01E8
:1021F00080EC9CE00E94829ACE0101960E94AD99EB
:102200006AEB7CE0CE0101960E94979A4AE050E08A
:1022100060E070E0CE01019693D9CE0101960E9454
:10222000AD9921E0B501A401CE0101960E943A9B2F
:10223000BE016F5F7F4F86EC9CE00E949F9ACE01AB
:1022400001960E94AD9966EC7CE0CE0101960E9459
:10225000979A4AE050E06FEF7FEFCE010196FCDAEB
:10226000CE0101960E94AD9965E070E080E090E0BB
:102270000E94D38F60E375E0CE0101960E94189A08
:10228000CE01019692DBCE0101960E94AD9921E02C
:10229000B701A601CE0107960E943A9BBE01695F75
:1022A0007F4FCE0101960E94979A60E077E0CE01C1
:1022B00001960E94509CBC0186EC9CE00E94829A90
:1022C000CE0101960E94AD99CE0107960E94AD996C
:1022D00066EC7CE0CE0101960E94979A4AE050E0BD
:1022E00068EF7FEFCE010196B7DACE0101960E942A
:1022F000AD9965E070E080E090E00E94D38F80911E
:10230000B10C882331F068E572E080E090E00E9433
:10231000D38F2C960FB6F894DEBF0FBECDBFDF91E2
:10232000CF91FF90EF90DF90CF90BF90AF909F90B4
:102330008F907F906F905F904F900895CF93DF9331
:10234000EC018C819D81892B61F0BE018EE89FE0BC
:102350000E947996BE0185E691E1DF91CF910C94C0
:102360007996DF91CF9108951F93CF93DF93CDB7E7
:10237000DEB7A8970FB6F894DEBF0FBECDBF182FFB
:1023800089EF9CE00E94718481110EC06AE07CE0BC
:10239000CE0101960E94B69BCE010196CFDFCE0101
:1023A00001960E94AD99A3C0BE016F5F7F4F89EF78
:1023B0009CE00E945383112309F493C06FED7BE0EE
:1023C0008EE89FE00E9469966FEC7BE08EE89FE0CC
:1023D0000E942D96BE016F5F7F4F8EE89FE00E94A6
:1023E00089966FEB7BE08EE89FE00E942D964D85ED
:1023F0005E856F8578892AE030E08EE89FE00E9454
:1024000065976FEA7BE08EE89FE00E942D964989F0
:102410005A896B897C892AE030E08EE89FE00E942F
:1024200065976FE97BE08EE89FE00E942D9620E0A3
:1024300030E040E251E4698D7A8D8B8D9C8D0E9455
:102440005FA1AB01BC0122E030E08EE89FE00E947A
:10245000819863E475E08EE89FE00E9489966FE8BA
:102460007BE08EE89FE00E942D9620E030E040E285
:1024700051E46D8D7E8D8F8D98A10E945FA1AB017F
:10248000BC0122E030E08EE89FE00E94819863E486
:1024900075E08EE89FE00E9489966FE77BE08EE80A
:1024A0009FE00E942D9620E030E040E251E469A1D7
:1024B0007AA18BA19CA10E945FA1AB01BC0122E08B
:1024C00030E08EE89FE00E94819863E475E08EE83A
:1024D0009FE00E94899669E57BE08EE89FE00E947C
:1024E000699664EF71E080E090E00E94D38FA89637
:1024F0000FB6F894DEBF0FBECDBFDF91CF911F9115
:1025000008954F925F926F927F928F929F92AF92B7
:10251000BF92CF92DF92EF92FF920F931F93CF93D0
:10252000DF93CDB7DEB7CA54D1090FB6F894DEBF3A
:102530000FBECDBF8C016AE37BE0CE01CD960E9439
:10254000189A6AE37BE0CE01C7960E94189ABE01F2
:102550006F5F7F4F89EF9CE00E9404854D885E8805
:102560006F88788CC98CDA8CEB8CFC8C8D8D9E8D71
:10257000AF8DB8A12B968CAF9DAFAEAFBFAF2B97F1
:10258000C8010197039708F0E2C1A7019601C301B2
:10259000B20190580E94A89E2BED3FE049EC5FE30A
:1025A0000E94359E209134023091350240913602CE
:1025B000509137020E94359E4B015C0120E030E0D3
:1025C000A9010E94FB9E87FD09C080929D0C9092FC
:1025D0009E0CA0929F0CB092A00C10C02BED3FE07F
:1025E00049EC50E4C501B4010E94359E60939D0CF6
:1025F00070939E0C80939F0C9093A00C80909D0CE8
:1026000090909E0CA0909F0CB090A00C2BED3FE002
:1026100049EC50E4C501B4010E94A0A0181684F44E
:102620002BED3FE049EC50E4C501B4010E94349E1B
:1026300060939D0C70939E0C80939F0C9093A00CC4
:1026400020E030E044E353E460919D0C70919E0CD7
:1026500080919F0C9091A00C0E945FA12BED3FE018
:1026600049E450E40E94FF9E6093990C70939A0C89
:1026700080939B0C90939C0C0E94989F4AE0CE0103
:102680008B960E94E39A67E475E0CE0185960E94DE
:10269000189ABE01655D7F4FCE0185960E943F9CD2
:1026A00061E575E00E94509CBC0186EC9CE00E94B4
:1026B000829ACE0185960E94AD99CE018B960E949A
:1026C000AD998090990C90909A0CA0909B0CB09032
:1026D0009C0C20E030E044EB52E4C501B4010E94C0
:1026E000FB9E181694F020E030E040E05FE3C50167
:1026F000B4010E94359E0E94989F4AE0CE018B96BD
:102700000E94E39A68E575E023C020E030E044E3EE
:1027100053E4C501B4010E94FB9E1816A4F1A50163
:10272000940160E070E884E393E40E94349E609337
:10273000990C70939A0C80939B0C90939C0C0E9424
:10274000989F4AE0CE018B960E94E39A6BE575E074
:10275000CE0185960E94189ABE01655D7F4FCE011D
:1027600085960E943F9CBC01CE01CD960E94829A24
:10277000CE0185960E94AD99CE018B960E94AD99AF
:1027800069EB76E063C020E030E047E853E4C50140
:10279000B4010E94FB9E181604F120E030E044E3EF
:1027A00053E4C501B4010E94349E20E030E040E0D3
:1027B0005FE30E94359E6093990C70939A0C80930E
:1027C0009B0C90939C0C0E94989F4AE0CE018B96A4
:1027D0000E94E39A6BE575E01FC0A501940160E0DB
:1027E00070E084EB93E40E94349E20E030E040E00F
:1027F0005FE30E94359E6093990C70939A0C8093CE
:102800009B0C90939C0C0E94989F4AE0CE018B9663
:102810000E94E39A68E575E0CE0185960E94189AB9
:10282000BE01655D7F4FCE0185960E943F9CBC0135
:10283000CE01CD960E94829ACE0185960E94AD99D6
:10284000CE018B960E94AD996EE575E0CE01C796DC
:102850000E94B59ABE01635C7F4FCE0185960E94AF
:10286000979A4AE050E060E070E0CE0185960E94C1
:10287000A00ACE0185960E94AD990E94A48F209156
:10288000EA043091EB044091EC045091ED04809007
:10289000DE0D9090DF0DA090E00DB090E10D280DC1
:1028A000391D4A1D5B1D261737074807590708F4CD
:1028B00041C20E94A48F0E94C99F4B015C0160919C
:1028C000EA047091EB048091EC049091ED040E9475
:1028D000CB9F20E030E040E85EE30E945FA12796B6
:1028E0006CAF7DAF8EAF9FAF27976091DE0D70917B
:1028F000DF0D8091E00D9091E10D0E94CB9F9B0137
:10290000AC0127966CAD7DAD8EAD9FAD27970E9433
:10291000359E9B01AC01C501B4010E94FB9E87FD61
:1029200009C261E475E0CE0185960E94189ABE0145
:10293000695C7F4FCE0185960E943F9CBC01CE0111
:10294000CD960E94E99BCE0185960E94AD99C80163
:102950000297029708F0C8C120E030E040E251E45D
:10296000C301B2010E945FA14B015C0120E030E095
:1029700040E251E4C701B6010E945FA16B017C01F6
:1029800020E030E040E251E42B966CAD7DAD8EADA1
:102990009FAD2B970E945FA12B013C010E94A48F49
:1029A0002091110C3091120C4091130C5091140C89
:1029B000621B730B840B950B0E94C99F20E030E0D3
:1029C0004AE754E40E94FF9EAB01BC0123E0CE0124
:1029D0008B960E943A9B69E675E0CE0185960E942F
:1029E000189ABE01655D7F4FCE0185960E943F9C7F
:1029F00062E578E00E94509CBC0184EB9CE00E9460
:102A0000829ACE0185960E94AD99CE018B960E9446
:102A1000AD9964EB7CE0CE0185960E94979A66ECB6
:102A20007CE0CE0185960E943F9CBE01635C7F4F97
:102A30000E943F9CBC01CE01CD960E94829ACE019D
:102A400085960E94AD9964E27BE080EC9CE00E9458
:102A5000969B21E0B501A401CE0185960E943A9B88
:102A6000BE016B5D7F4F80EC9CE00E94E99BCE0134
:102A700085960E94AD9921E0B301A201CE01859611
:102A80000E943A9B21E0B701A601CE01C1960E94A7
:102A90003A9B61E475E0CE018B960E94189ABE01C4
:102AA0006F5C7F4FCE018B960E943F9C61E475E086
:102AB0000E94509CBE016B5D7F4F0E943F9C60E670
:102AC00075E00E94509CBC0180EC9CE00E94E99B58
:102AD000CE018B960E94AD99CE01C1960E94AD9910
:102AE000CE0185960E94AD99A5019401C501B4015E
:102AF0000E945FA14B015C01A7019601C701B601CD
:102B00000E945FA19B01AC01C501B4010E94359EEA
:102B10006B017C01A3019201C301B2010E945FA17C
:102B20009B01AC01C701B6010E94359E0E9412A212
:102B30006093950C7093960C8093970C9093980CDF
:102B400064E675E080EC9CE00E94EF9B4091950C60
:102B50005091960C6091970C7091980C21E0CE01E9
:102B60008B960E943A9BBE01655D7F4FCE01859694
:102B70000E94979A64E475E0CE0185960E94509C6D
:102B8000BC0186EC9CE00E94829ACE0185960E9450
:102B9000AD99CE018B960E94AD9966EC7CE080ECFD
:102BA0009CE00E94E99BC090950CD090960CE09020
:102BB000970CF090980C20E030E04AE754E4C7010D
:102BC000B6010E94A0A087FD29C020E030E04AE7BE
:102BD00054E4C701B6010E94FF9EAB01BC0123E093
:102BE000CE018B960E94689BBE01655D7F4FCE0132
:102BF00085960E94979A65E475E0CE0185960E94BD
:102C0000509CBC0186EC9CE00E94829ACE01859685
:102C10000E94AD99CE018B960E94AD9920E030E6DE
:102C20004AE656E46091950C7091960C8091970C51
:102C30009091980C0E94FB9EBE01635C7F4F87FFC2
:102C40004FC0CE0185960E94979A68E675E0CE0146
:102C500085960E94509C60EC7CE00E943F9CBC01E9
:102C600080EC9CE00E94829ACE0185960E94AD99EC
:102C70000330110599F460EC7CE0CE0185960E944A
:102C8000979ACE0185965ADBCE0185960E94AD9922
:102C90006AE37BE080EC9CE00E94B59A6BE675E00D
:102CA000CE018B960E94189A66EC7CE0CE018B9642
:102CB0000E943F9CBC01CE0185960E94979A4AE0F3
:102CC00050E06FEF7FEFCE0185960E942C0CCE0175
:102CD00085960E94AD99CE018B960E94AD9904C055
:102CE00080EC9CE00E94829A6AE070E080E090E0D4
:102CF0000E94D38FCE01C7960E94AD99CE01CD968A
:102D00000E94AD99C65BDF4F0FB6F894DEBF0FBED1
:102D1000CDBFDF91CF911F910F91FF90EF90DF908A
:102D2000CF90BF90AF909F908F907F906F905F906B
:102D30004F9008956AE37BE0CE0185960E94189A31
:102D4000CE0185960E94D50CCE0185960E94AD9944
:102D5000BE01695C7F4F82EE9DE00E945096E1CDFE
:102D60008F929F92AF92BF92CF92DF92EF92FF929B
:102D70000F931F93CF93DF9300D000D0CDB7DEB772
:102D80008C01C0900A02D0900B02E0900C02F090EF
:102D90000D0220E030E040E450E4C701B6010E949B
:102DA000A0A018166CF420E030E04AEF54E4C7010C
:102DB000B6010E945FA10E94989F6B017C0106C032
:102DC00030E3C32E35E7D32EE12CF12C0E94F30C17
:102DD00040E060E082EE9DE00E94C86F68E47BE026
:102DE00082EE9DE00E942D9641E060E082EE9DE043
:102DF0000E94C86F60E47BE082EE9DE00E942D9609
:102E000064E670E080E090E00E94D38F0E94A48F7F
:102E10006093110C7093120C8093130C9093140C0C
:102E20000E94A48F8090110C9090120CA090130C13
:102E3000B090140CDC01CB0188199909AA09BB09CF
:102E40008C159D05AE05BF055CF4C8015ADB0E94D8
:102E5000A48F64E170E080E090E00E94D38FE0CF27
:102E60000130110509F041C060EC7CE08AEB9CE088
:102E70000E94829A0E94F30C6AEB7CE0CE010196DC
:102E80000E94979A4AE050E060E070E0CE0101961F
:102E90000E94A00ACE0101960E94AD996FE27BE0EC
:102EA000CE0101960E94B69B4AE050E06FEF7FEFA3
:102EB000CE0101960E942C0CCE0101960E94AD9984
:102EC00064E775E0CE0101960E94189A60EC7CE000
:102ED000CE0101960E943F9CBC0180EC9CE00E94C8
:102EE000829ACE0101960E94AD9926960FB6F8946B
:102EF000DEBF0FBECDBFDF91CF911F910F91FF902D
:102F0000EF90DF90CF90BF90AF909F908F900895FB
:102F1000CF92DF92EF92FF92CF93DF9300D000D059
:102F2000CDB7DEB70E94F30C6EE170E080E090E078
:102F30000E94D38F82EE9CE00E94A2696B017C010B
:102F400064E670E080E090E00E94D38F62E476E077
:102F500080EC9CE00E94B59A21E0B701A601CE0169
:102F600001960E943A9BBE016F5F7F4F80EC9CE010
:102F70000E94E99BCE0101960E94AD9960EC7CE035
:102F8000CE0101960E94979A4AE050E060E070E01E
:102F9000CE0101960E94A00ACE0101960E94AD9931
:102FA0000E94C10C67E875E080EC9CE00E94EF9BFA
:102FB000C092A50CD092A60CE092A70CF092A80C9F
:102FC00020E030E040EF51E4C701B6010E94A0A02C
:102FD00087FD03C06FE079E054C020E030E040EDB1
:102FE00051E4C701B6010E94A0A087FD1FC06FEF8A
:102FF00078E0CE0101960E94B69B4AE050E06FEF68
:103000007FEFCE0101960E942C0CCE0101960E940A
:10301000AD9980910005882331F06CED75E080E07A
:1030200090E00E94D38F6FEE78E02BC020E030E07C
:1030300040EB51E4C701B6010E94A0A087FD03C088
:1030400061EE78E01EC062ED78E0CE0101960E944C
:10305000B69B4AE050E06FEF7FEFCE0101960E94F1
:103060002C0CCE0101960E94AD9980910005882319
:1030700031F06CED75E080E090E00E94D38F64EC5D
:1030800078E0CE0101960E94B69B4AE050E06FEFD7
:103090007FEFCE0101960E942C0CCE0101960E947A
:1030A000AD996CE271E080E090E00E94D38F809156
:1030B0000005882331F068EE73E080E090E00E9424
:1030C000D38F26960FB6F894DEBF0FBECDBFDF912B
:1030D000CF91FF90EF90DF90CF900895CF92DF9245
:1030E000EF92FF920F931F93CF93DF938C018B305E
:1030F000910529F48BE29DE00E94CB7C08C08631CB
:10310000910509F054C08BE29DE00E94537D8F3FF2
:103110002FEF920709F44BC0009731F0029609F4A3
:1031200049C0CCEFDFEF48C0C0902B0DD0902C0DE4
:10313000E0902D0DF0902E0D20E030E048EC52E4B0
:10314000C701B6010E94A0A018161CF0C0E0D0E094
:1031500002C0CBEFDFEF20E030E0A901C701B601EC
:103160000E94FB9E87FF02C0CAEFDFEFC0902F0DC9
:10317000D090300DE090310DF090320D20E030E035
:1031800048EC52ECC701B6010E94FB9E87FF02C0CB
:10319000C9EFDFEF20E030E040EF52E4C701B601B5
:1031A0000E94A0A0181644F4C8EFDFEF05C0CFEFCF
:1031B000DFEF02C0CEEFDFEF0C30110509F05FC08A
:1031C0008EE19DE00E94F87D853F09F456C034F4FD
:1031D000843F09F04FC0CDEFDFEF51C0863F19F0BB
:1031E000882321F047C0CFEFDFEF49C0C0901E0D0C
:1031F000D0901F0DE090200DF090210D20E030E0E8
:1032000048EC52E4C701B6010E94A0A018161CF0B9
:10321000C0E0D0E002C0CBEFDFEF20E030E040EADA
:1032200050E4C701B6010E94FB9E87FF02C0CAEFAF
:10323000DFEFC090220DD090230DE090240DF09090
:10324000250D20E030E040EF51ECC701B6010E94AF
:10325000FB9E87FF02C0C9EFDFEF20E030E040EFC8
:1032600052E4C701B6010E94A0A0181644F4C8EFAA
:10327000DFEF05C0CCEFDFEF02C0CEEFDFEFCE0116
:10328000DF91CF911F910F91FF90EF90DF90CF9042
:103290000895AF92BF92CF92DF92EF92FF920F9379
:1032A0001F93CF93DF93CDB7DEB72C970FB6F8946B
:1032B000DEBF0FBECDBF66EB78E0CE0101960E9467
:1032C000B69B4AE050E06FEF7FEFCE0101960E947F
:1032D0002C0CCE0101960E94AD996091C6047091AC
:1032E000C7048091FE049091FF04F8DE44E1C42EEF
:1032F000D12CE12CF12CA12CB12C8FEFA81AB80AFB
:10330000C701B6010E94D38F6091C6047091C704B3
:103310008091FE049091FF04E1DE8C0183E0A81609
:10332000B10434F484E1C80ED11CE11CF11CE5CFDA
:103330008EE1A816B1041CF4012BA1F704C00115FD
:10334000110509F011C18091FE049091FF048B30AA
:103350009105C9F480912F0D9091300DA091310D00
:10336000B091320D8093A50C9093A60CA093A70C5E
:10337000B093A80C80912B0D90912C0DA0912D0D48
:10338000B0912E0D1DC08631910521F30C9701F5EA
:103390008091220D9091230DA091240DB091250DC7
:1033A0008093A50C9093A60CA093A70CB093A80CA7
:1033B00080911E0D90911F0DA091200DB091210DB7
:1033C0008093A10C9093A20CA093A30CB093A40C97
:1033D0004091A50C5091A60C6091A70C7091A80C7F
:1033E00021E0CE0107960E943A9B62E476E0CE018E
:1033F00001960E94189ABE01695F7F4FCE01019627
:103400000E943F9CBC0180EC9CE00E94829ACE010D
:1034100001960E94AD99CE0107960E94AD99409108
:10342000A10C5091A20C6091A30C7091A40C21E00E
:10343000CE0107960E943A9B6AE875E0CE0101969C
:103440000E94189ABE01695F7F4FCE0101960E94CB
:103450003F9CBC0180EC9CE00E94E99BCE01019660
:103460000E94AD99CE0107960E94AD9961E376E086
:1034700080EC9CE00E94EF9B6AE37BE0CE0101962A
:103480000E94189A44E150E060E070E0CE0101969D
:103490000E94A00ACE0101960E94AD99C090A50C91
:1034A000D090A60CE090A70CF090A80C20E030E0A3
:1034B000A901C701B6010E94A0A020E030E040E0D1
:1034C0005FE387FD05C0C701B6010E94359E04C0B9
:1034D000C701B6010E94349E0E94989F2AE0AB016A
:1034E000BC01CE0101960E940E9BBE016F5F7F4F13
:1034F0008AEB9CE00E949F9ACE0101960E94AD99B2
:1035000040E067E082EE9DE00E94C86F6AEB7CE0DD
:1035100082EE9DE00E9450966FED82EE9DE00E944B
:103520005F9660E375E082EE9DE00E945E9660919A
:10353000A10C7091A20C8091A30C9091A40C0E94FC
:10354000989F4AE050E082EE9DE00E94489761E338
:1035500076E082EE9DE00E945E9664E670E080E098
:1035600090E00E94D38F65C00F3F8FEF1807ACF03B
:1035700068EA78E0CE0101960E94B69B4AE050E0EE
:1035800060E070E0CE0101960E94A00ACE01019693
:103590000E94AD9965E878E048C00E3F8FEF1807AC
:1035A00081F167E778E0CE0101960E94B69B4AE080
:1035B00050E060E070E0CE0101960E94A00ACE01CA
:1035C00001960E94AD9968E678E080EC9CE00E944C
:1035D000969B4AE0B801CE0101960E94E39ABE0193
:1035E0006F5F7F4F80EC9CE00E94E99BCE010196CB
:1035F0000E94AD9962E578E080EC9CE00E94119C0D
:1036000018C067E478E0CE0101960E94B69B4AE0BC
:1036100050E060E070E0CE0101960E94A00ACE0169
:1036200001960E94AD9967E278E080EC9CE00E94F0
:10363000969B2C960FB6F894DEBF0FBECDBFDF91E0
:10364000CF911F910F91FF90EF90DF90CF90BF909F
:10365000AF900895CF92DF92EF92FF920F931F9356
:10366000CF93DF93CDB7DEB72C970FB6F894DEBFBC
:103670000FBECDBF69E178E0CE0101960E94B69BF6
:103680004CE251E06FEF7FEFCE0101960E942C0CCF
:10369000CE0101960E94AD996091C6047091C70455
:1036A0008091FE049091FF0419DD54E1C52ED12CC8
:1036B000E12CF12C00E010E00F5F1F4FC701B601B5
:1036C0000E94D38F6091C6047091C7048091FE045C
:1036D0009091FF0403DD0330110534F484E1C80E3A
:1036E000D11CE11CF11CE8CF0A3011051CF4892B18
:1036F000A9F703C0892B09F094C18091FE04909131
:10370000FF048B309105C9F480912F0D9091300DFD
:10371000A091310DB091320D8093A50C9093A60C21
:10372000A093A70CB093A80C80912B0D90912C0D19
:10373000A0912D0DB0912E0D1DC08631910521F364
:103740000C9701F58091220D9091230DA091240DED
:10375000B091250D8093A50C9093A60CA093A70C77
:10376000B093A80C80911E0D90911F0DA091200D7B
:10377000B091210D8093A10C9093A20CA093A30C67
:10378000B093A40C4091A50C5091A60C6091A70C8D
:103790007091A80C21E0CE0107960E943A9B62E44A
:1037A00076E0CE0101960E94189ABE01695F7F4FB4
:1037B000CE0101960E943F9CBC0180EC9CE00E94DF
:1037C000829ACE0101960E94AD99CE0107960E9481
:1037D000AD994091A10C5091A20C6091A30C7091F5
:1037E000A40C21E0CE0107960E943A9B6AE875E09E
:1037F000CE0101960E94189ABE01695F7F4FCE01EB
:1038000001960E943F9CBC0180EC9CE00E94E99BD9
:10381000CE0101960E94AD99CE0107960E94AD9906
:1038200061E376E080EC9CE00E94EF9B6AE37BE042
:10383000CE0101960E94189A44E150E060E070E0E9
:10384000CE0101960E94A00ACE0101960E94AD9978
:10385000C090A50CD090A60CE090A70CF090A80CFE
:1038600020E030E0A901C701B6010E94A0A020E03D
:1038700030E040E05FE387FD05C0C701B6010E946C
:10388000359E04C0C701B6010E94349E0E94989FD5
:103890002AE0AB01BC01CE0101960E940E9BBE0145
:1038A0006F5F7F4F8AEB9CE00E949F9ACE0101964A
:1038B0000E94AD9940E067E082EE9DE00E94C86FF3
:1038C0006AEB7CE082EE9DE00E9450966FED82EE06
:1038D0009DE00E945F9660E375E082EE9DE00E94AD
:1038E0005E966091A10C7091A20C8091A30C9091B6
:1038F000A40C0E94989F4AE050E082EE9DE00E9456
:10390000489761E376E082EE9DE00E945E9664E671
:1039100070E080E090E00E94D38F8CEC9CE00E94ED
:103920000E9EC090A50CD090A60CE090A70CF09035
:10393000A80C20E030E040EF51E4C701B6010E943E
:10394000A0A087FD03C06AE078E054C020E030E02A
:1039500040ED51E4C701B6010E94A0A087FD1FC041
:103960006AEF77E0CE0101960E94B69B4AE050E0F4
:103970006FEF7FEFCE0101960E942C0CCE010196D5
:103980000E94AD9980910005882331F06CED75E0BF
:1039900080E090E00E94D38F6AEE77E02BC020E0B9
:1039A00030E040EB51E4C701B6010E94A0A087FDC2
:1039B00003C06CED77E01EC06DEC77E0CE010196A0
:1039C0000E94B69B4AE050E06FEF7FEFCE01019678
:1039D0000E942C0CCE0101960E94AD9980910005A9
:1039E000882331F06CED75E080E090E00E94D38F89
:1039F0006FEB77E0CE0101960E94B69B4AE050E063
:103A00006FEF7FEFCE0101960E942C0CCE01019644
:103A10000E94AD9962E370E080E090E00E94D38F55
:103A200001C076DA2C960FB6F894DEBF0FBECDBF7C
:103A3000DF91CF911F910F91FF90EF90DF90CF908A
:103A40000895CF92DF92EF92FF921F93CF93DF936F
:103A5000CDB7DEB7AA970FB6F894DEBF0FBECDBFC5
:103A6000182F882351F08091AF0C882331F06AE33E
:103A70007BE08EE89FE00E94899689E39DE00E94AA
:103A80005489BE016F5F7F4F89E39DE00E94F488F7
:103A9000CE010D967C01112391F18091AF0C88230A
:103AA00071F168EA77E0C7010E94B69BC7010E94E6
:103AB000740AC7010E94AD99FE0131966F01F601AB
:103AC00041915191619171916F0126E030E08EE852
:103AD0009FE00E94819861E475E08EE89FE00E947B
:103AE0005E96CE14DF0459F76AE37BE0C7010E94BB
:103AF000189AC7010E94740AC7010E94AD9923E970
:103B000038E144E85FE369817A818B819C810E947E
:103B10005FA16D877E878F87988B22E430E645E82A
:103B20005FE36D817E818F8198850E945FA1698BA3
:103B30007A8B8B8B9C8B25E83BEE41E95FE36985B3
:103B40007A858B859C850E945FA16D8B7E8B8F8B88
:103B5000988FB70189E39DE00E94D488112309F46E
:103B60009EC08091AF0C882309F499C0B70189E306
:103B70009DE00E94F4886E01F9E1CF0ED11C6BE943
:103B800077E0C6010E94B69BC6010E94740AC60176
:103B90000E94AD99F70141915191619171917F011D
:103BA00022E030E08EE89FE00E94819861E475E0B9
:103BB0008EE89FE00E945E96EC14FD0459F76AE3DC
:103BC0007BE0C7010E94189AC7010E94740AC701CE
:103BD0000E94AD996E01F5E2CF0ED11C9601AE01A7
:103BE000495D5F4FBE01675D7F4F89E39DE00E94A5
:103BF000378A6EE877E08EE89FE00E942D9669A5EF
:103C00007AA54AE050E08EE89FE00E94489761E480
:103C100075E08EE89FE00E945E966FA178A54AE06D
:103C200050E08EE89FE00E94489761E475E08EE8DE
:103C30009FE00E945E966DA17EA14AE050E08EE872
:103C40009FE00E9448976AE37BE08EE89FE00E9435
:103C50008996B70189E39DE00E94758A65E877E05F
:103C60008EE89FE00E942D96F7014191519161915C
:103C700071917F012AE030E08EE89FE00E948198F8
:103C800061E475E08EE89FE00E945E96EC14FD040E
:103C900059F76AE37BE08EE89FE00E94899661E035
:103CA00070E089E39DE00E9468891123A9F080916A
:103CB000AF0C882389F061E777E08EE89FE00E94EF
:103CC0002D9689E39DE00E94BF8A4AE050E0BC0146
:103CD0008EE89FE00E944F9724E030E043E050E000
:103CE00062E070E089E39DE00E947589112309F488
:103CF00041C08091AF0C8823E9F165E577E08EE85B
:103D00009FE00E942D969E012B5D3F4FAE01495DC5
:103D10005F4FBE01675D7F4F89E39DE00E94D18ABE
:103D200069A57AA54AE050E08EE89FE00E94489796
:103D300061E475E08EE89FE00E945E966FA178A531
:103D40004AE050E08EE89FE00E94489761E475E009
:103D50008EE89FE00E945E966DA17EA14AE050E051
:103D60008EE89FE00E9448976AE37BE08EE89FE040
:103D70000E94899665E070E089E39DE00E94928947
:103D80001123A9F08091AF0C882389F062E477E0D9
:103D90008EE89FE00E942D9689E39DE00E94148B9F
:103DA0004AE050E0BC018EE89FE00E944F9766E039
:103DB00070E089E39DE00E949F891123A9F0809122
:103DC000AF0C882389F06AE277E08EE89FE00E94DA
:103DD0002D9689E39DE00E94268B4AE050E0BC01CD
:103DE0008EE89FE00E944F9767E070E089E39DE0D6
:103DF0000E94A2891123A9F08091AF0C882389F039
:103E000064E177E08EE89FE00E942D9689E39DE0D3
:103E10000E94388B4AE050E0BC018EE89FE00E948F
:103E20004F9768E070E089E39DE00E94AF8911231D
:103E3000A9F08091AF0C882389F06CEF76E08EE8D2
:103E40009FE00E942D9689E39DE00E944A8B4AE004
:103E500050E0BC018EE89FE00E944F9769E070E05F
:103E600089E39DE00E94BC891123A9F08091AF0CE9
:103E7000882389F062EE76E08EE89FE00E942D961E
:103E800089E39DE00E945C8B4AE050E0BC018EE833
:103E90009FE00E944F976AE070E089E39DE00E94F6
:103EA000C9891123A9F08091AF0C882389F06CECAB
:103EB00076E08EE89FE00E942D9689E39DE00E94C7
:103EC0006E8B4AE050E0BC018EE89FE00E944F9765
:103ED0006BE070E089E39DE00E94D6891123A9F090
:103EE0008091AF0C882389F063EB76E08EE89FE049
:103EF0000E942D9689E39DE00E94808B4AE050E06D
:103F0000BC018EE89FE00E944F976CE070E089E36F
:103F10009DE00E94E389112309F494C08091AF0CC5
:103F2000882309F48FC06BE976E08EE89FE00E9459
:103F30002D9689E39DE00E94928B4AE050E0BC01FF
:103F40008EE89FE00E944F9764E876E08EE89FE05D
:103F50000E942D9689E39DE00E94B78C682F70E047
:103F60004AE050E08EE89FE00E944F976DE676E0D1
:103F70008EE89FE00E942D9689E39DE00E94BB8C15
:103F8000682F70E04AE050E08EE89FE00E944F9773
:103F900066E576E08EE89FE00E942D9689E39DE03D
:103FA0000E94BF8C682F70E04AE050E08EE89FE0EE
:103FB0000E944F976DE376E08EE89FE00E942D9679
:103FC00089E39DE00E94C38C682F70E04AE050E0D6
:103FD0008EE89FE00E944F9764E276E08EE89FE0D3
:103FE0000E942D9689E39DE00E94C78C682F70E0A7
:103FF0004AE050E08EE89FE00E944F976BE076E049
:104000008EE89FE00E942D9689E39DE00E94CB8C74
:10401000682F70E04AE050E08EE89FE00E944F97E2
:104020006AEF75E08EE89FE00E942D9689E39DE09F
:104030000E94CF8C682F70E04AE050E08EE89FE04D
:104040000E944F9761E089E39DE00E946C8C61E0E3
:1040500089E39DE00E94718C61E089E39DE00E940C
:10406000768C1123B1F08091AF0C882391F061EE32
:1040700075E08EE89FE00E942D9689E39DE00E9406
:10408000D38C682F70E04AE050E08EE89FE00E94F9
:104090004F9760E089E39DE00E94768C1123B1F098
:1040A0008091AF0C882391F067EC75E08EE89FE07B
:1040B0000E942D9689E39DE00E94D38C682F70E0CA
:1040C0004AE050E08EE89FE00E944F9761E089E36C
:1040D0009DE00E947B8C1123B1F08091AF0C88236E
:1040E00091F06BEA75E08EE89FE00E942D9689E3DF
:1040F0009DE00E94D78C682F70E04AE050E08EE887
:104100009FE00E944F9760E089E39DE00E947B8CD6
:104110001123B1F08091AF0C882391F06EE875E027
:104120008EE89FE00E942D9689E39DE00E94D78C47
:10413000682F70E04AE050E08EE89FE00E944F97C1
:1041400061E089E39DE00E94808C1123B1F08091B1
:10415000AF0C882391F062E775E08EE89FE00E9443
:104160002D9689E39DE00E94DB8C682F70E04AE089
:1041700050E08EE89FE00E944F9760E089E39DE069
:104180000E94808C1123B1F08091AF0C882391F0B4
:1041900065E575E08EE89FE00E942D9689E39DE03D
:1041A0000E94DB8C682F70E04AE050E08EE89FE0D0
:1041B0000E944F9761E089E39DE00E94858C112366
:1041C000B1F08091AF0C882391F069E375E08EE83F
:1041D0009FE00E942D9689E39DE00E94DF8C682F6E
:1041E00070E04AE050E08EE89FE00E944F9760E068
:1041F00089E39DE00E94858C1123B1F08091AF0C82
:10420000882391F06CE175E08EE89FE00E942D9686
:1042100089E39DE00E94DF8C682F70E04AE050E067
:104220008EE89FE00E944F9761E089E39DE00E9445
:104230004E8C61E089E39DE00E94538C61E089E34C
:104240009DE00E94588C60E089E39DE00E945D8CB7
:1042500060E089E39DE00E94628C60E089E39DE07C
:104260000E94678C112309F495C08091AF0C8823BC
:1042700009F490C064E075E08EE89FE00E942D96FE
:1042800089E39DE00E94E38C682F70E04AE050E0F3
:104290008EE89FE00E944F9766EE74E08EE89FE004
:1042A0000E942D9689E39DE00E94E78C682F70E0C4
:1042B0004AE050E08EE89FE00E944F9768EC74E07F
:1042C0008EE89FE00E942D9689E39DE00E94EB8C92
:1042D000682F70E04AE050E08EE89FE00E944F9720
:1042E0006FEA74E08EE89FE00E942D9689E39DE0DE
:1042F0000E94EF8C682F70E04AE050E08EE89FE06B
:104300000E944F9766E974E08EE89FE00E942D9628
:1043100089E39DE00E94F38C682F70E04AE050E052
:104320008EE89FE00E944F976DE774E08EE89FE073
:104330000E942D9689E39DE00E94F78C682F70E023
:104340004AE050E08EE89FE00E944F976AE674E0F2
:104350008EE89FE00E942D9689E39DE00E94FB8CF1
:10436000682F70E04AE050E08EE89FE00E944F978F
:1043700065E574E08EE89FE00E942D9689E39DE05C
:104380000E94FF8C682F70E04AE050E08EE89FE0CA
:104390000E944F9760E089E39DE00E948A8C40ED87
:1043A0005FE069E470E489E39DE00E94CD8B112316
:1043B00009F44EC08091AF0C882309F449C061E430
:1043C00074E08EE89FE00E942D9689E39DE00E94B4
:1043D000A48BAB01BC0122E030E08EE89FE00E949C
:1043E00082986AE274E08EE89FE00E942D9689E34D
:1043F0009DE00E94088C4AE050E0682F8EE89FE024
:104400000E94819762E174E08EE89FE00E942D9601
:1044100061E089E39DE00E94038D682F70E04AE02F
:1044200050E08EE89FE00E944F9769EF73E08EE8BE
:104430009FE00E942D9661E089E39DE00E94078D38
:10444000682F70E04AE050E08EE89FE00E944F97AE
:1044500041E061E089E39DE00E948F8C1123B9F077
:104460008091AF0C882399F061EE73E08EE89FE0B5
:104470000E942D9661E089E39DE00E940B8D682FDC
:1044800070E04AE050E08EE89FE00E944F9741E0E4
:1044900061E089E39DE00E94948C60E089E39DE007
:1044A0000E94498C1123D1F08091AF0C8823B1F088
:1044B0006EEC73E08EE89FE00E942D9689E39DE00C
:1044C0000E94B38C682F70E04AE050E08EE89FE0D5
:1044D0000E944F9789E39DE00E940F8DAA960FB628
:1044E000F894DEBF0FBECDBFDF91CF911F91FF903B
:1044F000EF90DF90CF9008952F923F924F925F926E
:104500006F927F928F929F92AF92BF92CF92DF92E3
:10451000EF92FF920F931F93CF93DF93CDB7DEB748
:10452000C554D1090FB6F894DEBF0FBECDBF2B0125
:104530003C012DA33EA34FA358A70E94A48F22960F
:104540006CAF7DAF8EAF9FAF229720E9421621E07E
:1045500052066104710434F070E9472E55245394D7
:10456000612C712C8DA19EA1AFA1B8A5803197427D
:10457000A105B1052CF030E127E290E080E004C015
:104580003DA12EA19FA188A54091B10C411104C06D
:104590003DA32EA39FA388A722966CAD7DAD8EADC3
:1045A0009FAD229728EE33E040E050E00E94C4A285
:1045B00026962CAF3DAF4EAF5FAF2697F1E0FDAB37
:1045C00019A61AA61BA61CA68E01035F1F4F222741
:1045D0003327A901241935094609570929AB3AABF4
:1045E0004BAB5CAB29A53AA54BA55CA58DA19EA1C3
:1045F000AFA1B8A5281739074A075B070CF035C3E8
:1046000069A57AA58BA59CA50E94CB9F20E030E0F0
:104610004AE754E40E94FF9EAB01BC0123E0C801BD
:104620000E943A9BB8018AEB9CE00E949F9AC801C5
:104630000E94AD998DA19EA1AFA1B8A50A97A10531
:10464000B10594F42AE026964CAD5DAD6EAD7FAD1C
:104650002697C8010E940E9BB8018AEB9CE00E943D
:104660009F9AC8010E94AD99BE016F5F7F4F89E399
:104670009DE00E94758A61EC73E080EC9CE00E94F2
:10468000969BDE0111961D01C12CD12C7601F10102
:1046900081909190A190B1901F01A5019401C50155
:1046A000B4010E945FA19B01AC01C701B6010E9449
:1046B000359E6B017C0123E0B501A401CE01439638
:1046C0000E94689BBE016D5E7F4FC8010E94979A51
:1046D00061E475E0C8010E94509CBC0180EC9CE044
:1046E0000E94E99BC8010E94AD99CE0143960E94A9
:1046F000AD992016310659F6C701B6010E9412A2E3
:104700006B017C01FDE24F16F1E05F06610471046C
:1047100044F00E94F30C40E060E082EE9DE00E94D5
:10472000C86F23E0B701A601C8010E943A9B68E662
:1047300075E0CE0143960E94189A6AEB7CE0CE01A8
:1047400043960E943F9C60E975E00E94509CB8012E
:104750000E943F9C65E975E00E94509CBC0180EC82
:104760009CE00E94E99BCE0143960E94AD99C8014E
:104770000E94AD992DEC3CEC4CE45FE3C701B6011F
:104780000E94A0A029813A814B815C812DA73EA780
:104790004FA758AB18160CF0ACC12AE939E949E922
:1047A0005FE3C701B6010E94FB9E87FFA2C13DA93E
:1047B000332309F49EC189849A84AB84BC8420E0AD
:1047C00030E0A901C501B4010E94FB9ECD80DE80CE
:1047D000EF80F884882309F12DA53EA54FA558A99F
:1047E000CA01B9010E945FA16EAB7FAB88AF99AFE0
:1047F000A7019601C701B6010E945FA19B01AC0110
:104800006EA97FA988AD99AD0E94359E0E9412A223
:10481000A50194010E94A89E04C06BED7FE089EC85
:104820009FE320EE3EE245E652E40E945FA16EABBC
:104830007FAB88AF99AF20E030E0A901C701B60196
:104840000E94FB9E882309F12DA53EA54FA558A9DE
:10485000CA01B9010E945FA16AAF7BAF8CAF9DAF67
:10486000A5019401C501B4010E945FA19B01AC01A7
:104870006AAD7BAD8CAD9DAD0E94359E0E9412A2AB
:10488000A70196010E94A89E04C06BED7FE089EC11
:104890009FE320EE3EE245E652E40E945FA16AAF4C
:1048A0007BAF8CAF9DAF20E030E0A9016DA57EA568
:1048B0008FA598A90E94FB9E8823F9F0A501940179
:1048C000C501B4010E945FA14B015C01A7019601E3
:1048D000C701B6010E945FA19B01AC01C501B401F3
:1048E0000E94359E0E9412A22DA53EA54FA558A953
:1048F0000E94A89E6B017C0108C06BEDC62E6FE084
:10490000D62E69ECE62E6FE3F62E69E675E0C80157
:104910000E94189A6AEB7CE0C8010E943F9C68E9FB
:1049200075E00E94509CBC0180EC9CE00E94829A41
:10493000C8010E94AD9969E675E0C8010E94189A05
:104940006AEB7CE0C8010E943F9C62EB75E00E942C
:10495000509CBC018AEB9CE00E94829AC8010E9494
:10496000AD9921E04EA95FA968AD79ADC8010E945B
:104970003A9B21E04AAD5BAD6CAD7DADCE01439677
:104980000E943A9B20EE3EE245E652E4C701B601A2
:104990000E945FA1AB01BC0121E0CE014F960E94B5
:1049A0003A9BBE01615E7F4FCE0149960E94979A65
:1049B00061E475E0CE0149960E94509CBE016D5E97
:1049C0007F4F0E943F9C61E475E00E94509CB801BB
:1049D0000E943F9CBC0184EB9CE00E94829ACE0125
:1049E00049960E94AD99CE014F960E94AD99CE0195
:1049F00043960E94AD99C8010E94AD994DE24416BC
:104A000041E054066104710474F469A57AA58BA58C
:104A10009CA525E030E040E050E00E94C4A2672B56
:104A2000682B692BC1F56AEB7CE0C8010E94979A5C
:104A300045E050E06FEF7FEFC8010E94550BC801C1
:104A40000E94AD996BEB75E0C8010E94189A45E091
:104A500050E061EF7FEFC8010E94A00AC8010E94E8
:104A6000AD996AE37BE0C8010E94189AC8010E94D0
:104A7000D50CC8010E94AD9964EB7CE0C8010E948E
:104A8000979A45E050E060E070E0C8010E942C0C6D
:104A9000C8010E94AD9964EB7CE080EC9CE00E9430
:104AA000E99B5FE1451651046104710434F489A562
:104AB0009AA5ABA5BCA5B7FD11C060EC7CE0C80110
:104AC0000E94979AC8010E949E11C8010E94AD9948
:104AD0006AE37BE080EC9CE00E94B59AB201C301DE
:104AE00077FE04C069A97AA98BA99CA90E94D38FDB
:104AF000A9C023E04DA55EA56FA578A9C8010E94B5
:104B00003A9B69E675E0CE0143960E94189A6AEBDB
:104B10007CE0CE0143960E943F9C6DEB75E00E94C5
:104B2000509CB8010E943F9C66E975E00E94509C31
:104B3000BC018AEB9CE00E94829ACE0143960E94BF
:104B4000AD99C8010E94AD9949855A856B857C85D0
:104B500023E0C8010E94689B4D815E816F8178854A
:104B600023E0CE0149960E94689BBE01675E7F4F9D
:104B7000CE0143960E94979A62EC75E0CE0143966F
:104B80000E94509CB8010E943F9C66E975E00E941B
:104B9000509CBC0184EB9CE00E94829ACE0143961B
:104BA0000E94AD99CE0149960E94AD99C8010E941C
:104BB000AD999DE2491691E059066104710474F4BF
:104BC00069A57AA58BA59CA525E030E040E050E0E2
:104BD0000E94C4A2672B682B692BF1F46AEB7CE07E
:104BE000C8010E94979A4AE050E06FEF7FEFC8013A
:104BF0000E94550BC8010E94AD9964EB7CE0C8018E
:104C00000E94979A4AE050E060E070E0C8010E947C
:104C10002C0CC8010E94AD9960EC7CE0C8010E9498
:104C2000979AC8010E949E11C8010E94AD996AE33B
:104C30007BE080EC9CE00E94B59AC301B2010E9427
:104C4000D38F1DAA0E94A48F9B01AC0122968CAD2C
:104C50009DADAEADBFAD2297281B390B4A0B5B0B48
:104C600029A73AA74BA75CA7BDCC6AEB7CE0CE0195
:104C70000D960E94979A4AE050E06FEF7FEFCE01C9
:104C80000D960E94A00ACE010D960E94AD999DA995
:104C90009923B1F16BEB75E0CE010D960E94189A45
:104CA00045E050E061EF7FEFCE010D960E94A00A33
:104CB000CE010D960E94AD998091B10C882391F0A0
:104CC00069EB73E0CE010D960E94B69B45E050E083
:104CD00060E070E0CE010D960E94A00ACE010D9614
:104CE0000E94AD996AE37BE0CE010D960E94189A6E
:104CF000CE010D960E94D50CCE010D960E94AD9965
:104D000064EB7CE0CE010D960E94979A4AE050E059
:104D10006FEF7FEFCE010D960E942C0CCE010D9609
:104D20000E94AD99CB5BDF4F0FB6F894DEBF0FBE8C
:104D3000CDBFDF91CF911F910F91FF90EF90DF904A
:104D4000CF90BF90AF909F908F907F906F905F902B
:104D50004F903F902F9008958F929F92AF92BF9265
:104D6000CF92DF92EF92FF920F931F93CF93DF9337
:104D7000CDB7DEB72C970FB6F894DEBF0FBECDBF10
:104D800067E773E08AEB9CE00E94969B6AEB7CE00D
:104D9000CE0101960E94979A44E150E060E070E0F5
:104DA000CE0101960E94A00ACE0101960E94AD9903
:104DB00068E673E08AEB9CE00E94969B6AEB7CE0DD
:104DC000CE0101960E94979A44E150E06FEF7FEF89
:104DD000CE0101960E942C0CCE0101960E94AD9945
:104DE0008FEB9DE00E94D2704B015C018FEB9DE048
:104DF0000E94D4706B017C0104E010E020E030E000
:104E000048EC52E4C701B6010E94A0A018168CF429
:104E10000150110909F4D7C064E670E080E090E029
:104E20000E94D38F8FEB9DE00E94D4706B017C01B8
:104E3000E5CF21E0B501A401CE0107960E943A9B7F
:104E400067ED75E0CE0101960E94189ABE01695F78
:104E50007F4FCE0101960E943F9CBC0180EC9CE0FC
:104E60000E94829ACE0101960E94AD99CE010796CA
:104E70000E94AD9960EC7CE0CE0101960E94979A69
:104E800042E350E06FEF7FEFCE0101960E942C0CC1
:104E9000CE0101960E94AD9968E875E0CE010196B9
:104EA0000E94189ACE0101960E94D50CCE0101965F
:104EB0000E94AD9967E875E080EC9CE00E94EF9B52
:104EC00021E0B701A601CE0107960E943A9B62E459
:104ED00076E0CE0101960E94189ABE01695F7F4F6D
:104EE000CE0101960E943F9CBC0186EC9CE00E9492
:104EF000829ACE0101960E94AD99CE0107960E943A
:104F0000AD9961E475E0CE0101960E94189A66ECB5
:104F10007CE0CE0101960E943F9CBC018AEB9CE0A4
:104F20000E94829ACE0101960E94AD996AEB7CE0C4
:104F3000CE0101960E94979A4AE050E060E070E04E
:104F4000CE0101960E94550BCE0101960E94AD99AB
:104F500068E875E0CE0101960E94189ACE0101968C
:104F60000E94D50CCE0101960E94AD9967E875E0CC
:104F700086EC9CE00E94EF9B66EC7CE0CE01019603
:104F80000E94979A61E475E0CE0101960E94509CC0
:104F900060EC7CE00E943F9CBC0180EC9CE00E94A5
:104FA000829ACE0101960E94AD998091F00D909168
:104FB000F10D039709F044C084E090E09093F10D67
:104FC0008093F00D3DC06DE573E08AEB9CE00E949C
:104FD000969B6AEB7CE0CE0101960E94979A4AE08C
:104FE00050E060E070E0CE0101960E94A00ACE0180
:104FF00001960E94AD9965EC75E0CE0101960E9484
:10500000189A6AEB7CE0CE0101960E943F9CBC019D
:1050100080EC9CE00E94829ACE0101960E94AD999C
:105020008091F00D9091F10D049721F41092F10D03
:105030001092F00D81E090E09093E3048093E204FD
:1050400064E670E080E090E00E94D38F8091B10C24
:10505000882331F060E273E080E090E00E94D38F1B
:105060002C960FB6F894DEBF0FBECDBFDF91CF9167
:105070001F910F91FF90EF90DF90CF90BF90AF9076
:105080009F908F900895CF92DF92EF92FF920F93AF
:105090001F93CF93DF93CDB7DEB72C970FB6F8945D
:1050A000DEBF0FBECDBF8091B10C811102C00E9446
:1050B000F30C8091E2049091E304029741F0809117
:1050C000F00D9091F10D009721F0039711F044DE5F
:1050D0009DC188EC90E10E94129364E670E080E04C
:1050E00090E00E94D38F6DE973E08AEB9CE00E9410
:1050F000969B6AEB7CE0CE0101960E94979A44E170
:1051000050E060E070E0CE0101960E94A00ACE015E
:1051100001960E94AD996EE873E08AEB9CE00E94D4
:10512000969B6AEB7CE0CE0101960E94979A44E13F
:1051300050E06FEF7FEFCE0101960E942C0CCE0164
:1051400001960E94AD9960E070E08CEB9DE00E94BA
:105150007D7F6B017C0104E010E0A7019601C7018F
:10516000B6010E9453A2882309F442C001501109DC
:1051700009F02EC163E873E08AEB9CE00E94969BE5
:105180006AEB7CE0CE0101960E94979A4AE050E0DB
:1051900060E070E0CE0101960E94A00ACE01019667
:1051A0000E94AD9965EC75E0CE0101960E94189AB7
:1051B0006AEB7CE0CE0101960E943F9CBC0180EC32
:1051C0009CE00E94829ACE0101960E94AD99809146
:1051D000F00D9091F10D039721F41092F10D1092C2
:1051E000F00D82E090E09093E3048093E204DFC04E
:1051F00021E0B701A601CE0107960E943A9B67ED18
:1052000075E0CE0101960E94189ABE01695F7F4F3A
:10521000CE0101960E943F9CBC0180EC9CE00E9464
:10522000829ACE0101960E94AD99CE0107960E9406
:10523000AD9960EC7CE0CE0101960E94979A42E322
:1052400050E06FEF7FEFCE0101960E942C0CCE0153
:1052500001960E94AD9968E875E0CE0101960E9422
:10526000189ACE0101960E94D50CCE0101960E949B
:10527000AD9967E875E080EC9CE00E94EF9B60E0F0
:1052800070E08CEB9DE00E947B7F6B017C0104E071
:1052900010E0A7019601C701B6010E9453A288231E
:1052A00059F00150110909F0A2C06AE37BE086ECD5
:1052B0009CE00E94B59A5CC021E0B701A601CE0136
:1052C00007960E943A9B62E476E0CE0101960E9426
:1052D000189ABE01695F7F4FCE0101960E943F9CE4
:1052E000BC0186EC9CE00E94829ACE0101960E944D
:1052F000AD99CE0107960E94AD9961E475E0CE01AB
:1053000001960E94189A66EC7CE0CE0101960E94FC
:105310003F9CBC018AEB9CE00E94829ACE010196E0
:105320000E94AD996AEB7CE0CE0101960E94979AAB
:105330004AE050E06FEF7FEFCE0101960E94550BDF
:10534000CE0101960E94AD9968E875E0CE01019604
:105350000E94189ACE0101960E94D50CCE010196AA
:105360000E94AD9967E875E086EC9CE00E94EF9B97
:1053700066EC7CE0CE0101960E94979A61E475E0AC
:10538000CE0101960E94509C60EC7CE00E943F9C04
:10539000BC0180EC9CE00E94829ACE0101960E94A2
:1053A000AD9983E090E09093F10D8093F00D64E669
:1053B00070E080E090E00E94D38F8091B10C882350
:1053C00029F160E273E080E090E00E94D38F1EC07C
:1053D00068EC70E080E090E00E94D38F60E070E0C5
:1053E0008CEB9DE00E947D7F6B017C01B6CE68EC6A
:1053F00070E080E090E00E94D38F60E070E08CEB82
:105400009DE00E947B7F6B017C0143CF2C960FB601
:10541000F894DEBF0FBECDBFDF91CF911F910F91EA
:10542000FF90EF90DF90CF9008951F93CF93DF937D
:10543000182FC5E4DCE0812F0E946990899399932D
:105440006CE370E080E090E00E94D38F8CE0C5397F
:10545000D80789F768E270E085E49CE00E949A082A
:1054600020E030E040EA50E40E945FA120E030E01C
:1054700040E85AE30E945FA1DF91CF911F91089508
:105480004F925F926F927F928F929F92AF92BF9254
:10549000CF92DF92EF92FF920F931F93CF93DF9300
:1054A000CDB7DEB764970FB6F894DEBF0FBECDBFA1
:1054B0007C018B0160EE75E08AEB9CE00E94B59A5E
:1054C0000E94F30C6AEB7CE0CE0101960E94979A51
:1054D0004AE050E06FEF7FEFCE0101960E94A00AF4
:1054E000CE0101960E94AD99C7019FDF698B7A8B2F
:1054F0008B8B9C8B40901A0250901B0260901C0278
:1055000070901D02A3019201609116027091170222
:1055100080911802909119020E94349E4B015C0107
:1055200020E030E0A9010E94FB9E882309F451C0CD
:10553000C0902202D0902302E0902402F090250235
:1055400020E030E0A901C701B6010E94FB9E1816B9
:105550000CF03FC080911E0290911F02A09120028A
:10556000B09121028D879E87AF87B88B9C01AD01DA
:10557000C701B6010E94FB9E882359F1A70196013D
:105580006D857E858F8598890E94FF9E0E94ECA084
:105590006D877E878F87988BA301920169897A89AD
:1055A0008B899C890E94349EA50194010E94FF9ED4
:1055B0002D853E854F8558890E945FA10E946C9F72
:1055C0009B01AC01C701B6010E945FA16B017C0188
:1055D00003C0C12CD12C76016AEB7CE0CE01019690
:1055E0000E94979A4AE050E060E070E0CE01019698
:1055F0000E94A00ACE0101960E94AD9920E030E6FB
:105600004AEE56E4C701B6010E94A0A018163CF469
:105610006EE473E080EC9CE00E94969B44C0011510
:105620001105B9F421E0B701A601CE0107960E9449
:105630003A9B6AEE75E0CE0101960E94189ABE016F
:10564000695F7F4FCE0101960E943F9C6EEE75E030
:105650001BC00230110539F522E049895A896B894E
:105660007C89CE0107960E943A9B6AEE75E0CE01D6
:1056700001960E94189ABE01695F7F4FCE01019684
:105680000E943F9C62EF75E00E94509CBC0180EC40
:105690009CE00E94829ACE0101960E94AD99CE01B3
:1056A00007960E94AD9960EC7CE0CE0101960E94C5
:1056B000979A4AE050E06FEF7FEFCE0101960E948B
:1056C0002C0CCE0101960E94AD9964E670E080E05A
:1056D00090E00E94D38F8091B10C882331F060E27A
:1056E00073E080E090E00E94D38F64960FB6F89448
:1056F000DEBF0FBECDBFDF91CF911F910F91FF9005
:10570000EF90DF90CF90BF90AF909F908F907F9061
:105710006F905F904F9008954F925F926F927F923B
:105720008F929F92AF92BF92CF92DF92EF92FF92B1
:10573000CF93C82F8091600B81110DC00E94A48F60
:105740006093540B7093550B8093560B9093570BAB
:1057500081E08093600B8091580B81110DC00E94F5
:10576000A48F6093500B7093510B8093520B9093C6
:10577000530B81E08093580B1092440C1092430C11
:10578000E090430CF090440C88E2E816F1040CF031
:105790008AC08C2F0E946990F701EE0FFF1FEB5B10
:1057A000F34F9183808368E270E085E49CE00E947F
:1057B0009A0820E030E040EA50E40E945FA120E037
:1057C00030E040E85AE30E945FA16B017C016093E6
:1057D0004C0B70934D0B80934E0B90934F0B40905E
:1057E0002A0250902B0260902C0270902D02A3018F
:1057F0009201609126027091270280912802909177
:1058000029020E94349E9B01AC0160E070E080ECB4
:1058100090E40E94349E4B015C0120E030E0A9013D
:105820000E94FB9E20E030E040E650E4811105C07C
:10583000C701B6010E945FA11EC0C701B6010E9448
:105840005FA1A30192010E94359E20E030E040E874
:1058500050E40E94349EA50194010E94FF9E20E026
:1058600030E040EC50E40E945FA120E030E040E8EE
:1058700050E40E94359E6093480B7093490B8093CF
:105880004A0B90934B0B64E170E080E090E00E9443
:10589000D38F8091430C9091440C01969093440CCB
:1058A0008093430C6DCF6091480B7091490B8091B0
:1058B0004A0B90914B0BCF91FF90EF90DF90CF90E0
:1058C000BF90AF909F908F907F906F905F904F9020
:1058D0000895CF92DF92EF92FF92CF93DF93CDB7EF
:1058E000DEB72C970FB6F894DEBF0FBECDBF65E4D0
:1058F00073E08AEB9CE00E94969B6AEB7CE0CE0111
:1059000001960E94979A4AE050E060E070E0CE0174
:1059100001960E94A00ACE0101960E94AD99809145
:10592000810290918202F8DE6B017C0120E030E080
:10593000A9010E94A0A087FD22C022E0B701A60114
:10594000CE0107960E943A9B64EF75E0CE01019666
:105950000E94189ABE01695F7F4FCE0101960E9496
:105960003F9CBC0180EC9CE00E94829ACE01019693
:105970000E94AD99CE0107960E94AD9906C066E3DC
:1059800073E080EC9CE00E94969B60EC7CE0CE0192
:1059900001960E94979A4AE050E06FEF7FEFCE01A8
:1059A00001960E942C0CCE0101960E94AD992C9676
:1059B0000FB6F894DEBF0FBECDBFDF91CF91FF9041
:1059C000EF90DF90CF9008952F923F924F925F9289
:1059D0006F927F928F929F92AF92BF92CF92DF92FF
:1059E000EF92FF920F931F93CF93DF9300D01F92FC
:1059F000CDB7DEB76B017C015A8349835901FA01A7
:105A000020813181428153810E94FB9E181614F03F
:105A1000F50183C010E00150104C000F111F000F62
:105A2000111FE981FA81E00FF11F2081318142814C
:105A30005381C701B6010E94A0A087FF6BC011E08F
:105A4000612E712C4301880C991C880C991CE981EA
:105A5000FA81E80DF91D2080318042805380A20137
:105A60009101C701B6010E94A0A0181614F41F5F8F
:105A7000E7CFA2019101C701B6010E94FB9E8501FB
:105A8000080D191D811102C0F80147C0C3018150E2
:105A9000904C880F991F880F991FA981BA81A80F70
:105AA000B91F2D913D914D915C9129833A834B8390
:105AB0005C83F501E80FF91F80809180A280B3809C
:105AC000C701B6010E94349E6B017C01A5019401BF
:105AD000F80160817181828193810E94349E9B01D3
:105AE000AC01C701B6010E945FA16B017C01298155
:105AF0003A814B815C81C201B1010E94349E9B01BD
:105B0000AC01C701B6010E94FF9EA50194010E944D
:105B1000359E07C0F501E00FF11F60817181828120
:105B200093810F900F900F900F90DF91CF911F9165
:105B30000F91FF90EF90DF90CF90BF90AF909F902C
:105B40008F907F906F905F904F903F902F9008952F
:105B5000CF92DF92EF92FF921F93CF93DF93182F94
:105B6000CAE0D0E0C12CD12C7601812F0E9469902F
:105B7000BC01882777FD8095982F0E94CB9F9B01C1
:105B8000AC01C701B6010E94359E6B017C0162E346
:105B900070E080E090E00E94D38F219731F720E001
:105BA00030E040E251E4C701B6010E94FF9E20E0D0
:105BB00030E040EA50E40E945FA120E030E040E89D
:105BC0005AE30E945FA1DF91CF911F91FF90EF9068
:105BD000DF90CF900895FC0120E030E0772767FD4B
:105BE0007095AB0142505109DF01A81BB90BA417F6
:105BF000B50724F4A1912A0F311DF6CFA9014E5B00
:105C00005F4F860F971FFC013297208130E0322FC3
:105C1000222731968081280F311D81E042175307DA
:105C200009F080E00895FF920F931F93CF93DF93C5
:105C3000F82E0AE010E0C0E0D0E08F2D0E946990BD
:105C4000C80FD91F65E070E080E090E00E94D38F1C
:105C50000150110991F7CE016AE070E00E947BA229
:105C6000CB01DF91CF911F910F91FF9008950F937A
:105C70001F93CF93DF93CDB7DEB72E970FB6F8946F
:105C8000DEBF0FBECDBF8D879E870E94F30C8D8532
:105C90009E85C9DF8C0162E370E080E090E00E94A5
:105CA000D38FB801882777FD8095982F0E94CB9FCE
:105CB00020E030E040EA50E40E945FA120E030ECB8
:105CC0004FE754E40E94FF9EAB01BC0123E0CE01EC
:105CD00007960E943A9B63E077E0CE0101960E940E
:105CE000189ABE01695F7F4FCE0101960E943F9CCA
:105CF00063E076E00E94509CBC0180EC9CE00E9436
:105D0000829ACE0101960E94AD99CE0107960E941B
:105D1000AD9966E076E08AEB9CE00E94B59A6AEB6A
:105D20007CE0CE0101960E94979A4AE050E068E03C
:105D300070E0CE0101960E94A00ACE0101960E9459
:105D4000AD9960EC7CE0CE0101960E94979A4AE002
:105D500050E06FEF7FEFCE0101960E942C0CCE0138
:105D600001960E94AD996AEB7CE080EC9CE00E9479
:105D7000E99B8091B10C882331F060E273E080E010
:105D800090E00E94D38F2E960FB6F894DEBF0FBE20
:105D9000CDBFDF91CF911F910F910895CF93DF93E6
:105DA000CDB7DEB72C970FB6F894DEBF0FBECDBFD0
:105DB0003ADF9093AA0C8093A90C62E370E080E034
:105DC00090E00E94D38F6091A90C7091AA0C4AE0D8
:105DD000CE0101960E94E39ABE016F5F7F4F80EC77
:105DE0009CE00E949F9ACE0101960E94AD998091FD
:105DF0001C0D90911D0D892B09F45FC068E17DE0B9
:105E0000CE0107960E94979ABE01695F7F4FCE012F
:105E100001960E94979A44E150E060E070E0CE0164
:105E200001960E94A00ACE0101960E94AD996EE0F3
:105E300076E0CE0101960E94189A60EC7CE0CE01DB
:105E400001960E943F9CBC018AEB9CE00E94829AD2
:105E5000CE0101960E94AD996AEB7CE0CE010196DD
:105E60000E94979A44E150E06FEF7FEFCE010196D8
:105E70000E942C0CCE0101960E94AD99BE01695F73
:105E80007F4FCE0101960E94979A61E475E0CE01A2
:105E900001960E94509C6AEB7CE00E943F9CBC01F2
:105EA00080EC9CE00E94829ACE0101960E94AD99FE
:105EB000CE0107960E94AD9954C069E176E08AEB65
:105EC0009CE00E94B59A6AEB7CE0CE0101960E94AC
:105ED000979A44E150E060E070E0CE0101960E94A4
:105EE000A00ACE0101960E94AD996DE176E0CE0147
:105EF00001960E94189A60EC7CE0CE0101960E9407
:105F00003F9CBC018AEB9CE00E94829ACE010196E4
:105F10000E94AD996AEB7CE0CE0101960E94979AAF
:105F200044E150E06FEF7FEFCE0101960E942C0C10
:105F3000CE0101960E94AD996EE076E0CE01019609
:105F40000E94189A60EC7CE0CE0101960E943F9C72
:105F5000BC0180EC9CE00E94829ACE0101960E94D6
:105F6000AD998091B10C882331F060E273E080E05C
:105F700090E00E94D38F2C960FB6F894DEBF0FBE30
:105F8000CDBFDF91CF9108950F931F93CF93DF93F0
:105F9000CDB7DEB72C970FB6F894DEBF0FBECDBFDE
:105FA0008C0181E00E94669064E670E080E090E001
:105FB0000E94D38F0E94F30CC80135DE60E074E0CC
:105FC000681B790B4AE0CE0107960E94E39A6DE1C7
:105FD00076E0CE0101960E94189ABE01695F7F4F5C
:105FE000CE0101960E943F9CBC0180EC9CE00E9487
:105FF000829ACE0101960E94AD99CE0107960E9429
:10600000AD9940E067E082EE9DE00E94C86F66EBCC
:1060100077E0CE0101960E94B69B42E350E068E033
:1060200070E0CE0101960E94A00ACE0101960E9466
:10603000AD9960EC7CE0CE0101960E94979A42E314
:1060400050E06FEF7FEFCE0101960E942C0CCE0145
:1060500001960E94AD9964E276E0CE0101960E941D
:10606000189A60EC7CE0CE0101960E943F9CBC0136
:1060700080EC9CE00E94829ACE0101960E94AD992C
:106080008091B10C882331F060E273E080E090E011
:106090000E94D38F2C960FB6F894DEBF0FBECDBFF3
:1060A000DF91CF911F910F9108950F9390E0BBDD89
:1060B000BC01882777FD8095982F0E94CB9F2DE00B
:1060C00038E643E55BE30E945FA106E021E532E0AC
:1060D00049E652E079DC20E030E048EC52E40E94EE
:1060E0005FA120E030E048EA51E40E945FA12091E6
:1060F0004D0230914E0240914F02509150020E9449
:10610000FF9E0F910895CF92DF92EF92FF92CF936F
:10611000DF93CDB7DEB72C970FB6F894DEBF0FBE76
:10612000CDBFC3DF6B017C0168EF72E08AEB9CE0BE
:106130000E94969B6AEB7CE0CE0101960E94979AA2
:1061400042E350E060E070E0CE0101960E94A00AB8
:10615000CE0101960E94AD9922E0B701A601CE01C1
:1061600007960E943A9B69EF75E0CE0101960E9466
:10617000189ABE01695F7F4FCE0101960E943F9C35
:106180006EE276E00E94509CBC0180EC9CE00E9494
:10619000829ACE0101960E94AD99CE0107960E9487
:1061A000AD9960EC7CE0CE0101960E94979A42E3A3
:1061B00050E06FEF7FEFCE0101960E942C0CCE01D4
:1061C00001960E94AD998091B10C882331F060E274
:1061D00073E080E090E00E94D38F2C960FB6F89485
:1061E000DEBF0FBECDBFDF91CF91FF90EF90DF906C
:1061F000CF900895CF92DF92EF92FF920F9390E0AD
:1062000012DDBC01882777FD8095982F0E94CB9FD7
:106210002DE038E643E55BE30E945FA106E021E55F
:1062200032E049E652E0D0DB20E030E048EC52E4D6
:106230000E945FA16B017C0120E030E0A9010E9477
:10624000FB9E181634F0C12CD12C08EAE02E01E494
:10625000F02EC0924D02D0924E02E0924F02F09288
:1062600050020F91FF90EF90DF90CF9008952F9202
:106270003F924F925F926F927F928F929F92AF92D6
:10628000BF92CF92DF92EF92FF920F931F93CF9323
:10629000DF9300D01F92CDB7DEB76C0148EA54E01F
:1062A00086E994E09A83898305EC1BE0EE24E3946D
:1062B000F12C66246394712C22E1222E312C33E1DF
:1062C000432E512C60E1A62EB12C71E1872E912C2A
:1062D00080919404909195048E159F050CF4EDC067
:1062E00091E0C916D10431F4F80180819181E981EE
:1062F000FA8109C0F2E0CF16D10439F4E981FA81BC
:1063000080819181F80191838083E981FA81808184
:106310009181009741F4FA01808191819093B904B1
:106320008093B80429C08130910541F4FA0180813D
:1063300091819093C7048093C6041EC0823091055A
:1063400041F4FA01808191819093C5048093C40443
:1063500013C0039789F4FA01808191819093BB0463
:106360008093BA046AE37BE088E19DE04B835C8321
:106370000E94B59A5C814B81E981FA81819191916A
:10638000FA83E9838430910541F4FA012081318157
:1063900030938202209381022CC08530910541F414
:1063A000FA01208131813093C3042093C20421C0BB
:1063B0008630910541F4FA01208131813093BF0488
:1063C0002093BE0421C08730910541F4FA01208159
:1063D00031813093BD042093BC044AC08A309105BA
:1063E00041F4FA01208131813093C1042093C0042B
:1063F0003FC08531910541F4FA012081318130930C
:10640000C9042093C80434C08631910541F4FA01CF
:10641000208131813093E5042093E40429C0873141
:10642000910531F5FA01208131812830310549F497
:10643000B092E904A092E8049092E7048092E60406
:1064400017C02730310549F43092E9042092E8045E
:106450005092E7044092E6040BC02630310541F427
:106460007092E9046092E8041092E7041092E60446
:106470009C012B5031092A303105B8F4FA012081F2
:1064800031813093BB042093BA04F7E1F89FB00147
:10649000F99F700D11246D577D4F88E19DE04B836E
:1064A0005C830E94B59A5C814B812FEFE21AF20A5D
:1064B0004E5F5F4F0E5F1F4F0BCF0F900F900F90EF
:1064C0000F90DF91CF911F910F91FF90EF90DF9090
:1064D000CF90BF90AF909F908F907F906F905F9084
:1064E0004F903F902F90089581E08093FA0480911F
:1064F000FB04882321F082EE9DE00C94776F0895D1
:1065000082EE9DE00E94736F1092FA0408958091CC
:10651000FB0481110AC081E08093FB048093FA049C
:1065200082EE9DE00E94FA6F0CC08091FA048823ED
:1065300041F0E6DF82EE9DE00E94F46F1092FB04D2
:106540000895D2CF4F925F926F927F92AF92BF9297
:10655000CF92DF92EF92FF920F931F93CF93DF932F
:10656000CDB7DEB7EA970FB6F894DEBF0FBECDBF4A
:10657000182F6AE37BE0CE01C5960E94189A612F1E
:10658000CE0145960E948B8EBE016B5E7F4FCE0181
:1065900001960E949D7FCE0101960E94FC80CE0153
:1065A00001960E9490826CE0CE0101960E94EC81DF
:1065B000CE0101960E94A67F082F10E0033011053E
:1065C00009F46FC162E672E0CE01C5960E94969B07
:1065D0006AE37BE080EC9CE00E94B59ABE016B5CB4
:1065E0007F4FCE0183960E94979A4AE050E060E088
:1065F00070E0CE0183960E94A00ACE0183960E948D
:10660000AD9941E060E082EE9DE00E94C86F62E4D7
:1066100076E0CE01C5960E94B59AE9E1AE2EECE097
:10662000BE2ECC24C394D12CE12CF12CE016F10623
:106630000CF0EDC06E2DCE0101960E941D83F50178
:1066400021913191419151915F010E94359E2B0121
:106650003C0120E030E04CEF52EC0E94FB9E87FFB3
:1066600025C04AE0B601CE0189960E94E39A62E70E
:1066700077E0CE0183960E94189ABE01675D7F4F36
:10668000CE0183960E943F9C63E376E00E94509C7B
:10669000BC0180EC9CE00E94E99BCE0183960E94A5
:1066A000AD99CE0189960E94AD9949C022E0B3010F
:1066B000A201CE0183960E943A9B4AE0B601CE0128
:1066C0008F960E94E39A62E777E0CE0189960E9456
:1066D000189ABE01615D7F4FCE0189960E943F9C52
:1066E0006BE278E00E94509CBE016D5D7F4F0E947E
:1066F0003F9CBC0184EB9CE00E94829ACE0189966B
:106700000E94AD99CE018F960E94AD99CE018396DD
:106710000E94AD9964EB7CE0CE0183960E94979A2B
:1067200061E475E0CE0183960E94509CBC0180EC30
:106730009CE00E94E99BCE0183960E94AD990130B6
:10674000110559F4E114F10409F05AC060EC7CE041
:10675000CE01C5960E94829A53C00230110511F5F0
:1067600022E0B301A201CE0189960E943A9BBE01AC
:10677000675D7F4FCE0183960E94979A61E475E032
:10678000CE0183960E94509CBC01CE01C5960E940A
:10679000E99BCE0183960E94AD99CE0189960E9415
:1067A000AD992EC064EB7CE0CE0183960E94979A4F
:1067B00044E150E06FEF7FEFCE0183960E942C0CF6
:1067C000CE0183960E94AD9968E875E0CE0183966C
:1067D0000E94189ACE0183960E94D50CCE01839612
:1067E0000E94AD998091FB04882351F08091FA04B6
:1067F000882331F060ED77E080E090E00E94D38F55
:10680000FFEFEF1AFF0A8FEFC81AD80A0FCFCE0199
:10681000C5960E94B29D80EC9CE00E94B29D01153D
:106820001105C9F46FE472E080EC9CE00E94969B35
:1068300064E472E0CE0183960E94B69B4AE050E089
:106840006FEF7FEFCE0183960E942C0CCE018396D2
:106850000E94AD99EEC0043011050CF003C1BE01D9
:106860006B5C7F4FCE0183960E94979A4AE050E07E
:106870006FEF7FEFCE0183960E942C0CCE018396A2
:106880000E94AD9968E875E0CE0183960E94189A3F
:10689000CE0183960E94D50CCE0183960E94AD99BD
:1068A000E1C06FE376E0CE01C5960E94B59ABE01C5
:1068B0006B5C7F4FCE0183960E94979A4AE050E02E
:1068C00060E070E0CE0183960E94A00ACE0183961C
:1068D0000E94AD996AE37BE080EC9CE00E94B59A4F
:1068E00060EC7CE0CE01C5960E94829A00E010E048
:1068F000602FCE0101960E941D836B017C0122E076
:10690000AB01BC01CE010115110569F483960E940B
:106910003A9BBE016D5D7F4F82EE9DE00E945096D6
:10692000CE0183961BC089960E943A9BBE01675D8B
:106930007F4FCE0183960E94979A61E475E0CE0165
:1069400083960E94509CBC01CE01C5960E94E99B93
:10695000CE0183960E94AD99CE0189960E94AD9991
:1069600022E0B701A601CE0189960E943A9BBE01A2
:10697000675D7F4FCE0183960E94979A61E475E030
:10698000CE0183960E94509CBC0180EC9CE00E944A
:10699000E99BCE0183960E94AD99CE0189960E9413
:1069A000AD990F5F1F4F0330110509F0A1CFCE0144
:1069B000C5960E94B29DBE016B5C7F4FCE0183964F
:1069C0000E94979A4AE050E06FEF7FEFCE018396E6
:1069D0000E942C0CCE0183960E94AD9968E875E068
:1069E000CE0183960E94189ACE0183960E94D50C00
:1069F000CE0183960E94AD9980EC9CE00E94B29DEE
:106A000065E476E0CE0183960E94189A60EC7CE003
:106A1000CE0183960E943F9C6FE476E00E94509CDA
:106A2000BC0180EC9CE00E94829ACE0183960E9479
:106A3000AD99CE01C5960E94AD99EA960FB6F8942D
:106A4000DEBF0FBECDBFDF91CF911F910F91FF90A1
:106A5000EF90DF90CF90BF90AF907F906F905F905E
:106A60004F9008956FE476E080EC9CE00E94EF9BED
:106A7000E0CF8F929F92AF92BF92CF92DF92EF9230
:106A8000FF920F931F93CF93DF93CDB7DEB7A297FB
:106A90000FB6F894DEBF0FBECDBF5C016A017B016B
:106AA000122F8091AF0C8823D9F060E372E08EE85A
:106AB0009FE00E942D964AE050E0B5018EE89FE0ED
:106AC0000E94489761E475E08EE89FE00E945E9620
:106AD00022E030E0B701A6018EE89FE00E94829894
:106AE000612FCE0145960E948B8EBE016B5E7F4F5B
:106AF000CE0101960E949D7FCE0101960E94FC80EE
:106B0000CE0101960E9490826CE0CE0101960E9417
:106B1000EC81CE0101960E94A67F082F10E00B3079
:106B2000110514F00AE010E08BE5A816B10408F492
:106B30004FC099E1892E9CE0992EC12CD12C760171
:106B4000A12CB12CA016B106BCF46A2DCE01019681
:106B50000E941D839B01AC01F401619371938193A9
:106B600091934F01C701B6010E94359E6B017C01D4
:106B7000FFEFAF1ABF0AE6CFB801882777FD8095EF
:106B8000982F0E94CB9F9B01AC01C701B6010E94C8
:106B9000FF9E6B017C0189E1882E8CE0982EA12C50
:106BA000B12CA016B1060CF052C0F4012081318145
:106BB00042815381C701B6010E94349EF401619362
:106BC0007193819391934F01FFEFAF1ABF0AE9CF01
:106BD000A114B10439F4B9E18B2EBCE09B2EA12C99
:106BE000B12C1DC00A151B050CF0850101501109BF
:106BF000602FCE0101960E941D839B01AC01000F06
:106C0000111F000F111F075E134FC701B6010E942D
:106C1000349EF801608371838283938318C0A01629
:106C2000B106ACF46A2DCE0101960E941D839B0132
:106C3000AC01C701B6010E94349EF40161937193C7
:106C4000819391934F01FFEFAF1ABF0AE8CFA2964D
:106C50000FB6F894DEBF0FBECDBFDF91CF911F916D
:106C60000F91FF90EF90DF90CF90BF90AF909F90EB
:106C70008F900895CF93DF93C8EED4E060E08881D1
:106C80000E941B9182E090E00E94F98F61E0888170
:106C90000E941B918AE090E00E94F98F60E0888159
:106CA0000E941B9120E432E44FE050E061E08091CB
:106CB000E6040E9478910E94C99F20E030E048ECF1
:106CC00052E40E94FF9E2091C40D3091C50D409169
:106CD000C60D5091C70D0E945FA120E030E44CE149
:106CE00056E40E94FF9E20E030E040E05FE30E9417
:106CF0005FA1DF91CF910895CF92DF92EF92FF9243
:106D0000B9DF6B017C0120E030E040E050E40E94FC
:106D1000A0A018161CF4AEDF6B017C0120E030E06F
:106D200040E050E4C701B6010E94A0A018161CF470
:106D3000A1DF6B017C0120E030E040E050E4C701BE
:106D4000B6010E94A0A018161CF494DF6B017C0110
:106D500020E030E040E050E4C701B6010E94A0A06E
:106D600018162CF4FF90EF90DF90CF9083CFC701DF
:106D7000B601FF90EF90DF90CF9008954F925F9211
:106D80006F927F928F929F92AF92BF92CF92DF923B
:106D9000EF92FF92CF93DF9300D01F92CDB7DEB773
:106DA000ABDF9B01AC0169833A834B835C830E9418
:106DB000B08F2B013C016EE170E080E090E00E941A
:106DC000D38F9ADF6B017C010E94B08F4B015C0175
:106DD00084189508A608B70829813A814B815C81FF
:106DE00081ED881687E09806A104B1040CF43DC03B
:106DF000C701B6010E94349E6B017C0120E030E0A7
:106E0000A9010E94A0A018165CF426EA3BE944EC14
:106E10005BE3C701B6010E94FB9E87FF0BC025C044
:106E200026EA3BE944EC5BEBC701B6010E94A0A057
:106E30001816DCF0C501B40128EE33E040E050E064
:106E40000E94C4A2CA01B9010E94CB9F4B015C0100
:106E500020E030E04AE754E4C701B6010E945FA198
:106E6000A50194010E94FF9E03C060E070E0CB0189
:106E70000F900F900F900F90DF91CF91FF90EF90B8
:106E8000DF90CF90BF90AF909F908F907F906F904A
:106E90005F904F90089523E333E948E853E40E945C
:106EA000FF9E20E030E040E85FE30E94359E0E94B4
:106EB00012A226E636EA45EA53E40E945FA16093F7
:106EC000C40D7093C50D8093C60D9093C70D0895A2
:106ED0004F925F926F927F928F929F92AF92BF92EA
:106EE000CF92DF92EF92FF92CF93DF93CDB7DEB7D1
:106EF0006C970FB6F894DEBF0FBECDBF6B017C015F
:106F00000E94A48F6D8B7E8B8F8B988F88EC90E185
:106F10000E94129361E08091E8040E94E29060E098
:106F20008091E6040E94E29082EE9CE00E94A269B9
:106F30006093C00D7093C10D8093C20D9093C30DEB
:106F4000AADFDADE6D877E878F87988B0E94B08FED
:106F5000698B7A8B8B8B9C8B6AE070E080E090E091
:106F60000E94D38F62E676E080EC9CE00E94B59AA6
:106F700020E030E04AE754E4C701B6010E945FA177
:106F8000698F7A8F8B8F9C8F412C512C3201C12CB1
:106F9000D12C7601C701B6010E94CB9F298D3A8D75
:106FA0004B8D5C8D0E94FB9E87FF87C10E94A48F42
:106FB0002D893E894F89588D621B730B840B950B6D
:106FC0000E94C99F20E030E04AE754E40E94FF9EFF
:106FD000AB01BC0123E0CE0101960E943A9BBE01A9
:106FE0006F5F7F4F8AEB9CE00E949F9ACE010196D3
:106FF0000E94AD9981DE6B017C010E94B08F4B0134
:107000005C0189899A89AB89BC89881A990AAA0A7C
:10701000BB0A91ED891697E09906A104B1040CF41E
:1070200041C020E030E0A901C701B6010E94A0A044
:1070300018165CF426EA3BE944EC5BE3C701B601B1
:107040000E94FB9E87FF0BC02DC026EA3BE944EC63
:107050005BEBC701B6010E94A0A018161CF1C50188
:10706000B40128EE33E040E050E00E94C4A2CA011F
:10707000B9010E94CB9F4B015C012D853E854F8558
:107080005889C701B6010E94349E20E030E04AE7EB
:1070900054E40E945FA1A50194010E94FF9E4B0150
:1070A0005C0103C0812C912C54016AEB7CE0CE0181
:1070B00001960E94979A66E876E0CE0101960E94BA
:1070C000509CBC018AEB9CE00E94829ACE01019602
:1070D0000E94AD9923E0B701A601CE0107960E9458
:1070E0003A9BBE01695F7F4FCE0101960E94979A3D
:1070F00068E175E0CE0101960E94509CBC0184EBD2
:107100009CE00E94829ACE0101960E94AD99CE0128
:1071100007960E94AD9922E0B501A401CE01019627
:107120000E943A9B69E675E0CE0107960E94189A84
:107130006AEB7CE0CE0107960E943F9C60E876E017
:107140000E94509C64EB7CE00E943F9C69E876E0E2
:107150000E94509CBE016F5F7F4F0E943F9C64E87D
:1071600076E00E94509CBC0180EC9CE00E94E99B70
:10717000CE0107960E94AD99CE0101960E94AD996D
:1071800020E030E0A901C501B4010E94A0A087FD64
:1071900006C061E475E084EB9CE00E94EF9B22E076
:1071A000B501A401CE0107960E943A9BBE01695F1A
:1071B0007F4FCE0101960E94979A64E876E0CE0157
:1071C00001960E94509CBC0184EB9CE00E94E99BCC
:1071D000CE0101960E94AD99CE0107960E94AD990D
:1071E00060EC7CE0CE0101960E94979ACE01019658
:1071F0000E949E11CE0101960E94AD99C301B20179
:1072000025E030E040E050E00E94C4A2672B682BEC
:10721000692B21F569E272E0CE0101960E94B69BCE
:1072200045E050E060E070E0CE0101960E94A00AC7
:10723000CE0101960E94AD9964EB7CE0CE010196EF
:107240000E94979A45E050E06FEF7FEFCE010196E4
:107250000E942C0CCE0101960E94AD996AE37BE05E
:1072600080EC9CE00E94B59A65E070E080E090E0E0
:107270000E94D38F0E94A48F6B017C012D893E89CF
:107280004F89588DC21AD30AE40AF50A35DD6D8795
:107290007E878F87988B0E94B08F698B7A8B8B8BC0
:1072A0009C8B6AE070E080E090E00E94D38F3FEF1B
:1072B000431A530A630A730A6DCE60E08091E804B2
:1072C0000E94E2906C960FB6F894DEBF0FBECDBF61
:1072D000DF91CF91FF90EF90DF90CF90BF90AF9074
:1072E0009F908F907F906F905F904F9008950F9335
:1072F0001F93CF93DF93CDB7DEB72C970FB6F894DB
:10730000DEBF0FBECDBF88EC90E10E94129308EE65
:1073100014E061E0F80180810E94E29060E08091D9
:10732000E6040E94E29082EE9CE00E94A2696093D3
:10733000C00D7093C10D8093C20D9093C30DABDD52
:10734000DBDCAB01BC0123E0CE0107960E943A9B37
:10735000BE01695F7F4FCE0101960E94979A60E05F
:1073600077E0CE0101960E94509CBC018AEB9CE024
:107370000E94829ACE0101960E94AD99CE01079695
:107380000E94AD9961E876E0CE0101960E94189ABC
:107390006AEB7CE0CE0101960E943F9CBC0180EC30
:1073A0009CE00E94829ACE0101960E94AD99E6DC93
:1073B000AB01BC0122E0CE0107960E943A9BBE01C0
:1073C000695F7F4FCE0101960E94979A64E876E04C
:1073D000CE0101960E94509CBC0184EB9CE00E946F
:1073E000829ACE0101960E94AD99CE0107960E9425
:1073F000AD9968E876E0CE0101960E94189A64EB98
:107400007CE0CE0101960E943F9CBC0180EC9CE098
:107410000E94E99BCE0101960E94AD9961E475E05E
:10742000CE0101960E94189A64EB7CE0CE01019691
:107430000E943F9CBC018AEB9CE00E94E99BCE012C
:1074400001960E94AD9962E272E0CE0101960E941F
:10745000B69B4AE050E060E070E0CE0101960E94E9
:10746000A00ACE0101960E94AD996AEB7CE0CE01A4
:1074700001960E94979A45E050E06FEF7FEFCE01B2
:1074800001960E942C0CCE0101960E94AD996CE8E9
:1074900076E080EC9CE00E94EF9B60E0F801808148
:1074A0000E94E2902C960FB6F894DEBF0FBECDBFBF
:1074B000DF91CF911F910F910895EF920F9320E0EC
:1074C00044E064E182EE9DE00E94E86E6FE976E0C0
:1074D00084ED9DE00E94189A64ED7DE08EEC9DE0C5
:1074E0000E94979A65EA76E088EC9DE00E94189ADF
:1074F0006AE58FEB9DE00E948F7020E141E168E139
:107500008CEB9DE00E94867E24E0E22E04E02AECD3
:1075100034E04EEC54E062ED74E08DE49DE00E94B6
:10752000EF6B89E39DE00E94B7881092380D6AE303
:107530007BE088E19DE00E94189A8091BE049091C2
:10754000BF049093170D8093160D20914102309146
:107550004202409143025091440260914502709171
:10756000460280914702909148020E94349E6093A7
:10757000120D7093130D8093140D9093150D4FEF12
:107580005FEFBA0189EF9CE00E94A08382EE9CE04D
:107590000E9483686AE37BE088ED9CE00E94189A71
:1075A0006AE37BE082ED9CE00E94189A6AE37BE04C
:1075B0008CEC9CE00E94189A6AE37BE086EC9CE0ED
:1075C0000E94189A6AE37BE080EC9CE00E94189A83
:1075D0006AE37BE08AEB9CE00E94189A6AE37BE016
:1075E00084EB9CE00E94189A609132027091330201
:1075F0008AE89BE00F91EF900C94587284EB9CE02A
:107600000E94AD998AEB9CE00E94AD9980EC9CE0D1
:107610000E94AD9986EC9CE00E94AD998CEC9CE0B8
:107620000E94AD9982ED9CE00E94AD9988ED9CE0AE
:107630000E94AD998FE59AE09093FA0C8093F90C33
:1076400088E19DE00E94AD9988EC9DE00E94AD9993
:107650008EEC9DE00E94AD9984ED9DE00C94AD9977
:107660008F929F92AF92BF92CF92DF92EF92FF9252
:107670000F931F93CF93DF93CDB7DEB72C970FB641
:10768000F894DEBF0FBECDBF61E08091FC040E9484
:10769000E29061E08091FC040E941B9182EE9DE0EB
:1076A0000E94F66E82EE9DE00E9440704EEE54E025
:1076B00060E082EE9DE00E9401700E94F30C0E9447
:1076C00074328EED93E09093420C8093410C0E94B3
:1076D0007BA68093F20D8FED93E00E947BA68093B2
:1076E000F30D8091F20D9091F30D1816190654F4D4
:1076F00010920005019731F41092F30D1092F20DE3
:107700000E94500A64E97DE0CE0101960E94B69B7A
:107710004AE050E06FEF7FEFCE0101960E94A00A91
:10772000CE0101960E94AD9940E052EC61E070E01C
:107730008EE89FE00E94FD0980910005882331F0CA
:1077400068EE73E080E090E00E94D38F8EE89FE0C7
:107750000E94BD91182F823709F493C11092420CF8
:107760001092410C7BE8C72E7BE0D72EE12CF12C48
:10777000C7010E947BA6D6018D936D01BFEFEB1A66
:10778000FB0AE6E8EE16F10499F780918B0B9091D5
:107790008C0BA0918D0BB0918E0B85369105A105B8
:1077A000B1050CF46EC18093380290933902A09316
:1077B0003A02B0933B0280918F0B9091900BA09175
:1077C000910BB091920B8093340290933502A09369
:1077D0003602B09337028091930B9091940BA09155
:1077E000950BB091960B80932E0290932F02A0934D
:1077F0003002B093310267EA7BE0CE0101960E942D
:10780000189ABE016F5F7F4F84ED9DE00E949F9AA2
:10781000CE0101960E94AD9965E07CE0CE01019613
:107820000E94189ABE016F5F7F4F8EEC9DE00E9410
:107830009F9ACE0101960E94AD9923E030E040E08E
:1078400050E064ED7DE0CE0101960E946F9D23E043
:1078500030E040E050E06EEC7DE0CE0107960E9403
:107860006F9DBE016F5F7F4FCE0107960E94989C6F
:10787000082FCE0107960E94AD99CE0101960E9475
:10788000AD99011106C064ED7DE08EEC9DE00E9493
:10789000829A8091970B9091980BA091990BB0913F
:1078A0009A0B8093220290932302A0932402B09318
:1078B000250280919B0B90919C0BA0919D0BB09108
:1078C0009E0B80931E0290931F02A0932002B09300
:1078D000210280919F0B9091A00BA091A10BB091E0
:1078E000A20B80931A0290931B02A0931C02B093E8
:1078F0001D028091A30B9091A40BA091A50BB091B8
:10790000A60B8093160290931702A0931802B093CF
:1079100019028091AF0B9091B00BA091B10BB09177
:10792000B20B8093450290934602A0934702B09316
:1079300048028091B30B9091B40BA091B50BB0911C
:10794000B60B8093410290934202A0934302B093FE
:1079500044028091B70B9091B80BA091B90BB091F4
:10796000BA0B8093490290934A02A0934B02B093C2
:107970004C028091BB0B9091BC0BA091BD0BB091C0
:10798000BE0B80933D0290933E02A0933F02B093C2
:1079900040028091BF0B9091C00BA091C10BB091A0
:1079A000C20B80934D0290934E02A0934F02B0936E
:1079B0005002C090D50BD090D60BE090D70BF09032
:1079C000D80BA7019601C701B6010E9453A28111ED
:1079D00008C0C0921202D0921302E0921402F092F8
:1079E00015026091010C7091020C882777FD80953B
:1079F000982F0E94CB9F9B01AC010E9453A2882329
:107A000021F01092020C1092010CE090030CF09007
:107A1000040CB701882777FD8095982F0E94CB9F93
:107A20009B01AC010E9453A2811104C0F092FF049B
:107A3000E092FE0459EDA52E5BE0B52E69E1862E9D
:107A40006CE0962ED501CD90DD90ED90FD905D011E
:107A5000A7019601C701B6010E9453A2811105C07A
:107A6000F401C082D182E282F382F4E08F0E911C95
:107A700081E0A8168CE0B80629F781E090E00E942A
:107A800037310EE8010F023080F01E3671F0809120
:107A90008B0B90918C0BA0918D0BB0918E0B85363A
:107AA0009105A105B1050CF057C180913802909164
:107AB0003902A0913A02B0913B0280938B0B9093D4
:107AC0008C0BA0938D0BB0938E0B80913402909110
:107AD0003502A0913602B091370280938F0B9093BC
:107AE000900BA093910BB093920B80912E029091EA
:107AF0002F02A0913002B09131028093930B9093AA
:107B0000940BA093950BB093960B1337A1F020E044
:107B100030E048E050E067EA7BE084ED9DE00E94C1
:107B2000EE9C20E030E04CE050E065E07CE08EEC44
:107B30009DE00E94EE9C8091220290912302A091F0
:107B40002402B09125028093970B9093980BA093F9
:107B5000990BB0939A0B80911E0290911F02A091F5
:107B60002002B091210280939B0B90939C0BA093D9
:107B70009D0BB0939E0B80911A0290911B02A091D5
:107B80001C02B0911D0280939F0B9093A00BA093B9
:107B9000A10BB093A20B8091160290911702A091B5
:107BA0001802B09119028093A30B9093A40BA09399
:107BB000A50BB093A60B8091450290914602A0912F
:107BC0004702B09148028093AF0B9093B00BA09303
:107BD000B10BB093B20B8091410290914202A091FF
:107BE0004302B09144028093B30B9093B40BA093E3
:107BF000B50BB093B60B8091490290914A02A091C7
:107C00004B02B0914C028093B70B9093B80BA093AA
:107C1000B90BB093BA0B80913D0290913E02A091B6
:107C20003F02B09140028093BB0B9093BC0BA0939A
:107C3000BD0BB093BE0B80914D0290914E02A0916E
:107C40004F02B09150028093BF0B9093C00BA09352
:107C5000C10BB093C20B8091120290911302A091BC
:107C60001402B09115028093D50B9093D60BA0937C
:107C7000D70BB093D80B8091FE049091FF049093A2
:107C8000040C8093030CE9E1FCE029ED3BE0419119
:107C9000519161917191D9014D935D936D937D9354
:107CA0009D01BCE0E134FB0791F76EE77DE0CE017A
:107CB00001960E94B69BCE0101960E94740ACE01E5
:107CC00001960E94AD9934E9C32E34E0D32E43ECE3
:107CD000A42E4BE0B42EE12CF12C809194049091D1
:107CE00095048E159F0574F1F60180819181D5016F
:107CF0008D939D935D018091AF0C8823E1F061EB42
:107D000076E08EE89FE00E945E964AE050E0B70180
:107D10008EE89FE00E9448976EEA76E08EE89FE04A
:107D20000E945E96F601608171814AE050E08EE823
:107D30009FE00E944F97FFEFEF1AFF0A82E0C80E04
:107D4000D11CCBCF023040F41092420C1092410C67
:107D500080E090E00E94270A8091010C9091020C33
:107D6000892B41F440E855E260E070E085E691E15E
:107D70000E94FD098091010C9091020C019741F441
:107D800040E052EC61E070E085E691E10E94FD097F
:107D900064E670E080E090E00E94D38F8091010C57
:107DA0009091020C892B09F0B7C01E3671F08091BA
:107DB0008B0B90918C0BA0918D0BB0918E0B853617
:107DC0009105A105B1050CF0A7C06AE37BE0CE01E7
:107DD00007960E94189A63EB76E0CE0101960E9406
:107DE000189A6EEC7DE0CE0101960E943F9CBC018A
:107DF000CE0107960E94829ACE0101960E94AD990B
:107E0000BE01695F7F4F85E691E10E94509668EB65
:107E10007BE080E090E00E94D38FBE01695F7F4FDE
:107E2000CE0101960E94979ACE0101960E94740A93
:107E3000CE0101960E94AD996CE271E080E090E085
:107E40000E94D38F4091D20D5091D30D42505109D1
:107E50006EEC7DE0CE0101960E94F109BE016F5FDC
:107E60007F4FCE0107960E949F9ACE0101960E94F5
:107E7000AD99BE01695F7F4FCE0101960E94979A2E
:107E8000BE01695F7F4FCE0101960E943F9CBC01FD
:107E9000CE0107960E94829ACE0101960E94AD996A
:107EA0006BEB76E0CE0101960E94189ABE01695FE5
:107EB0007F4FCE0101960E943F9CBC01CE010796E8
:107EC0000E94829ACE0101960E94AD99BE01695F1F
:107ED0007F4F85E691E10E94509668EB7BE080E061
:107EE00090E00E94D38FBE01695F7F4FCE01019663
:107EF0000E94979ACE0101960E94740ACE010196C3
:107F00000E94AD996CE271E080E090E00E94D38F16
:107F1000CE0107960E94AD9964E670E080E090E0A3
:107F20000E94D38F8AE89BE00E945D726EE67DE03E
:107F3000CE0101960E94B69B4AE050E06FEF7FEFC2
:107F4000CE0101960E94A00ACE0101960E94AD9931
:107F50008091010C9091020C892B09F56BE175E081
:107F6000CE0107960E94189A6EEC7DE0CE0107962E
:107F70000E943F9CBC01CE0101960E94979A4AE064
:107F800050E06FEF7FEFCE0101960E942C0CCE01E6
:107F900001960E94AD99CE0107960E94AD998091FD
:107FA000010C9091020C019709F56FE175E0CE018B
:107FB00007960E94189A6EEC7DE0CE0107960E940B
:107FC0003F9CBC01CE0101960E94979A4AE050E086
:107FD0006FEF7FEFCE0101960E942C0CCE0101962F
:107FE0000E94AD99CE0107960E94AD9961EB76E0B3
:107FF000CE0107960E94189A6EEC7DE0CE0107969E
:108000000E943F9C62EC76E00E94509CBC01CE0135
:1080100001960E94979ACE0101960E949E11CE0170
:1080200001960E94AD99CE0107960E94AD9964E633
:1080300070E080E090E00E94D38F85EC9EE00E948B
:10804000178664E670E080E090E00E94D38F63E2E0
:1080500070E085EC9EE00E942A8661E070E085EC8D
:108060009EE00E94000A85EC9EE00E949E8683E0CE
:1080700090E09093F10D8093F00D60E070E08CEB58
:108080009DE00E947D7F6B017C0162E370E080E0F7
:1080900090E00E94D38FA7019601C701B6010E940C
:1080A00053A2882309F44CC060E070E08CEB9DE0A3
:1080B0000E947B7F6B017C0162E370E080E090E0D6
:1080C0000E94D38FA7019601C701B6010E9453A257
:1080D0008823B1F11092F10D1092F00D88EC90E12F
:1080E0000E94129364E670E080E090E00E94D38FDB
:1080F00040E855E260E070E088EC90E10E94FD0904
:1081000088EC90E10E94A491892BD1F064E57DE098
:10811000CE0101960E94B69BCE0101960E94740A80
:10812000CE0101960E94AD9982E090E09093F10D0E
:108130008093F00D64E670E080E090E00E94D38FC1
:108140008091F00D9091F10D039779F46FE37DE04C
:10815000CE0101960E94B69BCE0101960E94740A40
:10816000CE0101960E94AD9912C08FEB9DE00E9456
:10817000D47020E030E048E453E40E94FB9E87FF87
:1081800006C082E090E09093E3048093E20463E011
:1081900082EE9CE00E944369811111C069E17DE09B
:1081A000CE0101960E94B69BCE0101960E949E11BF
:1081B000CE0101960E94AD9910923C02A3C066E0E8
:1081C0007DE080EC9CE00E94969B40E050E0BA018C
:1081D00082EE9CE00E94646B0E94CB9F20E030E026
:1081E00048EC52E40E94FF9EAB01BC0122E0CE01AC
:1081F00007960E943A9BBE01695F7F4FCE010196B0
:108200000E94979A61EE78E0CE0101960E94509C00
:10821000BC0180EC9CE00E94E99BCE0101960E948B
:10822000AD99CE0107960E94AD9960EC7CE0CE013D
:1082300001960E94979ACE0101960E94740ACE017F
:1082400001960E94AD9960EF7CE080EC9CE00E947A
:10825000969B609138027091390280913A02909118
:108260003B020E94CB9F20E030E048EC52E40E94A9
:10827000FF9EAB01BC0122E0CE0107960E943A9B13
:10828000BE01695F7F4FCE0101960E94979A61EE11
:1082900078E0CE0101960E94509CBC0180EC9CE0ED
:1082A0000E94E99BCE0101960E94AD99CE010796EE
:1082B0000E94AD9960EC7CE0CE0101960E94979AF5
:1082C000CE0101960E94740ACE0101960E94AD99DA
:1082D000113629F481E00E94211D81E011C08EE851
:1082E0009FE00E94BD91182F64E670E080E090E06E
:1082F0000E94D38F113671F380E00E94211D80E02F
:108300000E94B41164E670E080E090E00E94D38F98
:108310008091F00D9091F10D892BE1F488EC90E1C2
:108320000E94129361E08091E8040E94E29060E074
:108330008091E6040E94E29082EE9CE00E94A26995
:108340006093C00D7093C10D8093C20D9093C30DC7
:108350000E944B3780910005882331F068EE73E06E
:1083600080E090E00E94D38F6FE477E08CEC9CE09B
:108370000E94B59A82E090E09093AE0C8093AD0C91
:108380008091000581110E942A1B2C960FB6F8944B
:10839000DEBF0FBECDBFDF91CF911F910F91FF9038
:1083A000EF90DF90CF90BF90AF909F908F90089507
:1083B0006F927F928F929F92AF92BF92CF92DF92F5
:1083C000EF92FF920F931F93CF93DF93CDB7DEB75A
:1083D000E8970FB6F894DEBF0FBECDBF4B015C012E
:1083E00088EC90E10E94129364E670E080E090E0F7
:1083F0000E94D38F40E855E260E070E088EC90E1A5
:108400000E94FD0964E670E080E090E00E94D38F56
:108410006CEE72E08AEB9CE00E94969B6AEB7CE03B
:10842000CE0101960E94979A42E350E06FEF7FEFF2
:10843000CE0101960E94A00ACE0101960E94AD993C
:1084400061EE72E08AEB9CE00E94969B6AEB7CE016
:10845000CE0101960E94979A42E350E06FEF7FEFC2
:10846000CE0101960E942C0CCE0101960E94AD997E
:108470008091F00D9091F10D8D7F712CC12CD12C3C
:10848000E12CF12C00E010E0019709F459C0B2E4AE
:108490006B2E0E94A48F681979098A099B09683B91
:1084A0007B408105910508F04BC088EC90E10E946B
:1084B000A491892BF1F14CED55E060E070E088EC7F
:1084C00090E10E94C09868AE41E050E0BE01685C57
:1084D0007F4F88EC90E10E94A799882351F14FE1EA
:1084E00050E0BE016F5F7F4F88EC90E10E94C6981C
:1084F00089818D34F1F46FE1CE0101960E94EB2D5C
:108500008823B9F00C8110E0102F00278D81080F0F
:10851000111DEE80F12CFE2CEE248F81E80EF11C53
:10852000C884D12CDC2CCC248985C80ED11C77249E
:10853000739462E370E080E090E00E94D38FA9CF53
:108540000E94A48F681979098A099B09683B7B40BE
:108550008105910510F47110C1C00E94F30C6AEB03
:108560007CE0CE0180960E94979A42E350E066E05C
:1085700070E0CE0180960E94A00ACE0180960E94F3
:10858000AD99772009F4CFC082E090E09093F10D8F
:108590008093F00D4AE0B601CE0180960E94E39AE6
:1085A0004AE0B701CE0186960E94E39A4AE0B801FC
:1085B000CE01C2960E94E39ABE016E5C7F4FCE014F
:1085C0008C960E94979A6BE979E0CE018C960E9476
:1085D000509CBE016A5D7F4F0E943F9C6BE979E031
:1085E0000E94509CBE01605E7F4F0E943F9CBC0178
:1085F00080EC9CE00E94829ACE018C960E94AD99FC
:10860000CE01C2960E94AD99CE0186960E94AD9988
:10861000CE0180960E94AD9960EC7CE0CE01809600
:108620000E94979A4AE050E06FEF7FEFCE0180966C
:108630000E942C0CCE0180960E94AD996BED72E0E9
:1086400082EE9DE00E942D964AE0B601CE01809612
:108650000E94E39A4AE0B701CE0186960E94E39A0F
:108660004AE0B801CE01C2960E94E39A64EE76E039
:10867000CE018C960E94189ABE016E5C7F4FCE018F
:108680008C960E943F9C61E475E00E94509CBE0164
:108690006A5D7F4F0E943F9C61E475E00E94509CA0
:1086A000BE01605E7F4F0E943F9C64EF76E00E94B7
:1086B000509CBC0180EC9CE00E94829ACE018C967A
:1086C0000E94AD99CE01C2960E94AD99CE018696C8
:1086D0000E94AD99CE0180960E94AD9962E370E050
:1086E00080E090E00E94D38F88EC90E10E9412938A
:1086F00062E370E080E090E00E94D38FE8960FB6CE
:10870000F894DEBF0FBECDBFDF91CF911F910F91C7
:10871000FF90EF90DF90CF90BF90AF909F908F90A1
:108720007F906F90089560ED72E080EC9CE00E9475
:10873000969B60EC7CE0CE0180960E94979A4AE07E
:1087400050E060E070E0CE0180960E942C0CCE01DB
:1087500080960E94AD996DEB72E080EC9CE00E94E7
:10876000969B8091F00D9091F10D029709F0B6CF94
:108770001092F10D1092F00DB1CF7F928F929F92D7
:10878000AF92BF92CF92DF92EF92FF920F931F931F
:10879000CF93DF9300D000D0CDB7DEB74C018BE292
:1087A00090E10E94129340E052EC61E070E08BE2B5
:1087B00090E10E94FD094CED55E060E070E08BE235
:1087C00090E10E94C09864E670E080E090E00E9432
:1087D000D38FA12CB12C712CA814B9040CF051C06A
:1087E00065E070E080E090E00E94D38F00E010E050
:1087F000C12CD12C760171100FC08BE290E10E9448
:10880000A491892B31F485E1C816D104E104F10467
:108810001CF40330110554F08FEFA81AB80A64E66F
:1088200070E080E090E00E94D38FD6CF8BE290E1A1
:108830000E94A491892B69F08BE290E10E94BD9186
:10884000E1E0F0E0EC0FFD1FE00FF11F80830F5F10
:108850001F4F65E070E080E090E00E94D38F02300F
:1088600011054CF089818B3B31F4772473948A8114
:108870008A3A09F0712C8FEFC81AD80AE80AF80A68
:10888000BACF872D26960FB6F894DEBF0FBECDBFA8
:10889000DF91CF911F910F91FF90EF90DF90CF90DC
:1088A000BF90AF909F908F907F9008952F923F92AE
:1088B0004F925F926F927F928F929F92AF92BF92F0
:1088C000CF92DF92EF92FF920F931F93CF93DF939C
:1088D000CDB7DEB72B970FB6F894DEBF0FBECDBF76
:1088E0001C018BEB8F838AEA888781E0898784E685
:1088F000829D9001839D300D11243B872A87E12CB6
:10890000F12CC12CD12C812C912C5401C214D304F4
:1089100094F1C501B4010E94CB9F20E030E040E219
:1089200051E40E94FF9E6B017C01B101882777FD15
:108930008095982F0E94CB9F9B01AC01C701B60187
:108940000E94FF9E2B960FB6F894DEBF0FBECDBFE0
:10895000DF91CF911F910F91FF90EF90DF90CF901B
:10896000BF90AF909F908F907F906F905F904F904F
:108970003F902F9008952A853B85E216F3064CF62A
:10898000C7016AE070E00E948FA2892B79F4E09120
:108990002B10F0912C100280F381E02D43E050E089
:1089A000BE01695F7F4F8BE290E1199565E070E051
:1089B00080E090E00E94D38F3FEFE31AF30A00E0DB
:1089C00010E0412C512C32018BE290E10E94A491E5
:1089D000892B39F424E042165104610471040CF02F
:1089E00095CF063011050CF091CF8BE290E10E94FB
:1089F000A491892B69F08BE290E10E94BD91E1E0A6
:108A0000F0E0EC0FFD1FE00FF11F80830F5F1F4FA1
:108A100065E070E080E090E00E94D38F06301105A1
:108A200001F599818F8198131CC09A8188859813CC
:108A300018C09B818985981314C02C818D8190E08A
:108A4000A0E0B0E0BA2FA92F982F8827820F911DA0
:108A5000A11DB11D880E991EAA1EBB1E8FEFC81A3C
:108A6000D80A9FEF491A590A690A790AADCFCF92FD
:108A7000DF92EF92FF92CF93DF93CDB7DEB72C97C3
:108A80000FB6F894DEBF0FBECDBF8BE290E10E941F
:108A9000129340E052EC61E070E08BE290E10E94C2
:108AA000FD094CED55E060E070E08BE290E10E9442
:108AB000C09864E670E080E090E00E94D38F8091DF
:108AC000EE0D9091EF0D019751F483E090E055DEAB
:108AD00081111AC01092EF0D1092EE0D15C081E0B9
:108AE00090E04BDE81110AC083E090E046DE811108
:108AF00005C083E090E041DE882331F081E090E022
:108B00009093EF0D8093EE0D8091EE0D9091EF0D0F
:108B10000197D9F061EB72E08AEB9CE00E94969B92
:108B20006AEB7CE0CE0101960E94979A44E150E006
:108B30006FEF7FEFCE0101960E942C0CCE010196C3
:108B40000E94AD9965EA72E079C069E972E080EC53
:108B50009CE00E94969B60EC7CE0CE0101960E9416
:108B6000979ACE0101960E94740ACE0101960E9446
:108B7000AD9962E370E080E090E00E94D38F60ECFA
:108B80007CE0CE0101960E94979A42E350E06FEF9D
:108B90007FEFCE0101960E94A00ACE0101960E94AD
:108BA000AD996DE872E08AEB9CE00E94969B6AEBBF
:108BB0007CE0CE0101960E94979A44E150E06FEF6D
:108BC0007FEFCE0101960E942C0CCE0101960E94EF
:108BD000AD9984E090E06ADE6B017C0120E030E03A
:108BE00040EA51E40E94A0A0181634F521E0B70134
:108BF000A601CE0107960E943A9B60E679E0CE017D
:108C000001960E94189ABE01695F7F4FCE010196BE
:108C10000E943F9C6AEF76E00E94509CBC0180EC71
:108C20009CE00E94829ACE0101960E94AD99CE01ED
:108C300007960E94AD9906C061E872E080EC9CE066
:108C40000E94969B60EC7CE0CE0101960E94979A70
:108C50004AE050E060E070E0CE0101960E94A00A78
:108C6000CE0101960E94AD9960EC7CE0CE010196A8
:108C70000E94979A61E475E0CE0101960E94509C93
:108C80006AEB7CE00E943F9CBC0180EC9CE00E946F
:108C9000829ACE0101960E94AD998BE290E10E94EA
:108CA00012938091B10C882331F060E273E080E090
:108CB00090E00E94D38F2C960FB6F894DEBF0FBEC3
:108CC000CDBFDF91CF91FF90EF90DF90CF900895CF
:108CD0002F923F924F925F926F927F928F929F92CC
:108CE000AF92BF92CF92DF92EF92FF920F931F93BA
:108CF000CF93DF93CDB7DEB766970FB6F894DEBF9C
:108D00000FBECDBF6C018BE290E10E94129340E850
:108D100055E260E070E08BE290E10E94FD0964E6BC
:108D200070E080E090E00E94D38F4CED55E060E071
:108D300070E08BE290E10E94C09864E670E080E011
:108D400090E00E94D38F8FEF898381E08A8386E849
:108D50008B831C821D821E821F82188689E7898769
:108D6000C601880F991F9E8B8D8B212C312CE12CF5
:108D7000F12C812C912C5401EC14FD044CF08BE26D
:108D800090E10E941293E114F104B9F1670135C03A
:108D90008D899E892816390694F78BE290E10E940E
:108DA000349308977CF0E0912B10F0912C10028006
:108DB000F381E02D49E050E0BE016F5F7F4F8BE211
:108DC00090E1199565E070E080E090E00E94D38F1B
:108DD00000E010E0412C512C32018BE290E10E9426
:108DE000A491892B31F4E4E04E165104610471041E
:108DF00084F5023011056CF530C0C501B4010E9444
:108E0000CB9F4B015C01B601882777FD8095982F99
:108E10000E94CB9F9B01AC01C501B4010E94FF9E43
:108E200066960FB6F894DEBF0FBECDBFDF91CF912F
:108E30001F910F91FF90EF90DF90CF90BF90AF9078
:108E40009F908F907F906F905F904F903F902F906A
:108E50000895FFEF2F1A3F0A8FCF8BE290E10E9417
:108E6000A491892B69F08BE290E10E94BD91EAE028
:108E7000F0E0EC0FFD1FE00FF11F80830F5F1F4F2D
:108E800065E070E080E090E00E94D38F0230110531
:108E900069F59A858981981329C09B858B819813E0
:108EA00025C0FE013C96FC8BEB8B8BE290E10E948F
:108EB000A491892B31F4F4E04F165104610471043C
:108EC000DCF409301105E1F42D858C8590E0982FB4
:108ED0008827820F911DAA2797FDA095BA2F880E8B
:108EE000991EAA1EBB1E8FEFE81AF80A9FEF491AB7
:108EF000590A690A790A71CF04301105A4F3E4CF45
:108F00008BE290E10E94BD91EB89FC898193FC8BFF
:108F1000EB8B0F5F1F4FC9CF8091FB04882349F073
:108F20008091FA04882329F060E082EE9DE00C94A1
:108F30003B7008952F923F924F925F926F927F9273
:108F40008F929F92AF92BF92CF92DF92EF92FF9259
:108F50000F931F93CF93DF93CDB7DEB763970FB611
:108F6000F894DEBF0FBECDBF8B8B60E00E94E29015
:108F70008091B10C811105C08FE090E0A0E0B0E0DD
:108F800004C082E090E0A0E0B0E08F87988BA98BCE
:108F9000BA8B64E772E080EC9CE00E94969B60ECE8
:108FA0007CE0CE0101960E94979A4AE050E06FEF74
:108FB0007FEFCE0101960E94A00ACE0101960E9489
:108FC000AD99C12CD12C7601312C1D861E86212C09
:108FD00002E310E0412C512C32018B890E946990F0
:108FE000AA2797FDA095BA2F480E591E6A1E7B1E10
:108FF00065E070E080E090E00E94D38F015011099D
:1090000061F78090120290901302A0901402B09029
:109010001502C301B2010E94CB9F20E030E040EA7C
:1090200050E40E945FA120E030E040E85AE30E9453
:109030005FA120E030E048E452E40E94FF9EA501D9
:1090400094010E94349E20E030E040E751E40E9409
:109050005FA12B013C01A50194016AE979E989E34B
:1090600090E40E94349E9B01AC01C301B2010E94B6
:10907000FF9E20E030E0A9010E94359E20E030E014
:1090800040E251E40E945FA15B018C01232D3D85EC
:109090004E85522D0E94A0A0181624F43A2CBD86AD
:1090A0000E87212E20E030E0A901B501C8010E9401
:1090B000FB9E87FF04C0A12CB12C00E010E022E051
:1090C000A501B801CE0107960E943A9BBE01695FD7
:1090D0007F4FCE0101960E94979A6DEF76E0CE0108
:1090E00001960E94509CBC018AEB9CE00E94829AEF
:1090F000CE0101960E94AD99CE0107960E94AD99CE
:109100006AEB7CE0CE0101960E94979A4AE050E01B
:1091100060E070E0CE0101960E942C0CCE01019619
:109120000E94AD990E94A48F8090EA049090EB0475
:10913000A090EC04B090ED040091DA0D1091DB0DDD
:109140002091DC0D3091DD0D800E911EA21EB31E0C
:1091500086169706A806B90608F4E9C00E94A48FEF
:109160000E94C99F4B015C016091EA047091EB047D
:109170008091EC049091ED040E94CB9F20E030E0C0
:1091800040E85EE30E945FA12B013C016091DA0D93
:109190007091DB0D8091DC0D9091DD0D0E94CB9FD5
:1091A0009B01AC01C301B2010E94359E9B01AC0141
:1091B000C501B4010E94FB9E87FDB9C06CE370E05D
:1091C00080E090E00E94D38F9FEFC91AD90AE90A84
:1091D000F90A8F859889A989BA898C159D05AE05EC
:1091E000BF050CF0F5CE64E670E080E090E00E94F0
:1091F000D38F0E94F30C64E670E080E090E00E9460
:10920000D38F6CE672E08AEB9CE00E94969B6AEB3F
:109210007CE0CE0101960E94979A44E150E060E024
:1092200070E0CE0101960E94A00ACE0101960E9434
:10923000AD9922E0432D5D856E85722DCE01079696
:109240000E943A9BBE01695F7F4FCE0101960E944A
:10925000979A6DEF76E0CE0101960E94509CBC017A
:109260008AEB9CE00E94829ACE0101960E94AD9901
:10927000CE0107960E94AD996AEB7CE0CE01019683
:109280000E94979A42E350E06FEF7FEFCE01019684
:109290000E942C0CCE0101960E94AD9964E170E011
:1092A00080E090E00E94D38F37DE6EE170E080E0D6
:1092B00090E00E94D38F6EE170E080E090E00E9429
:1092C000D38F62E077E0CE0101960E94189A6AEB94
:1092D0007CE0CE0101960E943F9C66E077E00E9410
:1092E000509C60EC7CE00E943F9CBC0180EC9CE0C8
:1092F0000E94829ACE0101960E94AD9963960FB6A4
:10930000F894DEBF0FBECDBFDF91CF911F910F91BB
:10931000FF90EF90DF90CF90BF90AF909F908F9095
:109320007F906F905F904F903F902F900895F4DD65
:1093300045CFFF920F931F93CF93DF93CDB7DEB747
:109340002C970FB6F894DEBF0FBECDBF1092B20CB3
:109350006AE37BE088ED9CE00E94B59A11E08EE81C
:109360009FE00E94A4912091B20C18161906C4F532
:10937000211136C08EE89FE00E94BD918093B30C0E
:109380008A3041F08D3031F0682F88ED9CE00E94EA
:10939000FE9B1FC01093B20C6AE077E0CE010796E7
:1093A0000E94189A68ED7CE0CE0107960E943F9CCF
:1093B000BC01CE0101960E94979ACE0101960E94AF
:1093C000740ACE0101960E94AD99CE0107960E94C3
:1093D000AD996AE070E080E090E00E94D38FBFCF4B
:1093E000222361F02091B20C8091DC0C9091DD0C75
:1093F000211174C0009709F071C0B8C000E010E0FE
:10940000FF24F39485E691E10E94A49118161906B1
:10941000A4F585E691E10E94BD918093B30C8A305A
:1094200071F08D3061F09091B20C911108C0682FED
:1094300088ED9CE00E94FE9B0F5F1F4F17C080913C
:10944000DC0C9091DD0C892B89F0F092B20C85E652
:1094500091E10E94A4911816190644F46AE37BE096
:1094600088ED9CE00E94B59A1092B20C6FE070E01B
:1094700080E090E00E94D38FC5CF62E370E080E08F
:1094800090E00E94D38F012B09F4ACCF63E177E029
:10949000CE0107960E94189A68ED7CE0CE010796EF
:1094A0000E943F9CBC01CE0101960E94979ACE017A
:1094B00001960E94740ACE0101960E94AD99CE01D8
:1094C00007960E94AD9985E691E10E942B9264E691
:1094D00070E080E090E00E94D38F84CF019709F084
:1094E00069C066E876E0CE0107960E94189ABE0130
:1094F000695F7F4F88ED9CE00E94CE9C811115C072
:1095000069E177E0CE0101960E94189ABE016F5F73
:109510007F4F88ED9CE00E94CE9C11E0811110E00D
:10952000CE0101960E94AD9901C010E0CE010796D0
:109530000E94AD99112399F040E050E068ED7CE085
:10954000CE0101960E94F109BE016F5F7F4F8CEC46
:109550009CE00E949F9ACE0101960E94AD9964E121
:1095600070E080E090E00E94D38F24C064E670E059
:1095700080E090E00E94D38F0E94A48FCB0168EE20
:1095800073E00E948FA2CB0164E670E00E948FA27C
:10959000823691057CF08091B10C81110BC08CEC6E
:1095A0009CE00E940E9E613071058105910511F4C9
:1095B0000E942A1B2C960FB6F894DEBF0FBECDBFBB
:1095C000DF91CF911F910F91FF900895BF92CF929D
:1095D000DF92EF92FF920F931F93CF93DF93CDB75C
:1095E000DEB72B970FB6F894DEBF0FBECDBF6C0170
:1095F0008BE290E10E94129340E855E260E070E057
:109600008BE290E10E94FD0964E670E080E090E06A
:109610000E94D38F4CED55E060E070E08BE290E16A
:109620000E94C09864E670E080E090E00E94D38FD2
:109630008FEF898381E08A8386E88B831C821D8279
:109640001E821F82188689E789878BE290E10E943B
:109650002B9262E370E080E090E00E94D38F8BE277
:1096600090E10E94349308977CF0E0912B10F091E8
:109670002C100280F381E02D49E050E0BE016F5FC5
:109680007F4F8BE290E1199562E370E080E090E01B
:109690000E94D38FE12CF12CB12CEC14FD040CF0C2
:1096A0005BC08BE290E10E94A491892B21F18BE2B7
:1096B00090E10E94349308977CF0E0912B10F09198
:1096C0002C100280F381E02D49E050E0BE016F5F75
:1096D0007F4F8BE290E1199565E070E080E090E0CB
:1096E0000E94D38F00E010E08BE290E10E94A491F1
:1096F0000230110554F062E370E080E090E00E94D7
:10970000D38F8FEFE81AF80AC8CF8BE290E10E945E
:10971000A491892B69F08BE290E10E94BD91EAE06F
:10972000F0E0EC0FFD1FE00FF11F80830F5F1F4F74
:1097300065E070E080E090E00E94D38F0230110578
:1097400099F69A8589819813CFCF9B858B81981341
:10975000CBCFBB24B394C8CF8BE290E10E9412938D
:109760008B2D2B960FB6F894DEBF0FBECDBFDF91C9
:10977000CF911F910F91FF90EF90DF90CF90BF900E
:109780000895CF92DF92EF92FF920F931F93CF93A2
:10979000DF93CDB7DEB72C970FB6F894DEBF0FBEC0
:1097A000CDBF0E94F30C6CE273E080EC9CE00E9461
:1097B000969B60EC7CE0CE0101960E94979A4AE06D
:1097C00050E060E070E0CE0101960E94A00ACE0158
:1097D00001960E94AD9963E273E08AEB9CE00E94DF
:1097E000969B6AEB7CE0CE0101960E94979A44E139
:1097F00050E06FEF7FEFCE0101960E942C0CCE015E
:1098000001960E94AD998091EE0D9091EF0D8230FE
:10981000910551F481E090E0D9DE81111CC01092D5
:10982000EF0D1092EE0D17C0892BA9F481E090E0A6
:10983000CDDE81110AC081E090E0C8DE811105C053
:1098400081E090E0C3DE882331F082E090E09093E5
:10985000EF0D8093EE0D8091EE0D9091EF0D02973C
:1098600091F167E173E080EC9CE00E94969B60ECD4
:109870007CE0CE0101960E94979A4AE050E060E0B9
:1098800070E0CE0101960E94A00ACE0101960E94CE
:10989000AD9960EC7CE0CE0101960E94979A61E45C
:1098A00075E0CE0101960E94509C6AEB7CE00E941C
:1098B0003F9CBC0180EC9CE00E94829ACE01019604
:1098C0000E94AD9997C08AE090E002DA6B017C01BA
:1098D00020E030E0A9010E94FB9E18162CF08AE0DF
:1098E00090E0F6D96B017C010BE010E020E030E065
:1098F00042ED53E4C701B6010E94FB9E181684F4A2
:1099000020E030E0A901C701B6010E94FB9E1816B5
:10991000B4F069E073E080EC9CE00E94969B40C04C
:109920000150110969F368EC70E080E090E00E945A
:10993000D38F83E090E0CCD96B017C01D7CF20E0BE
:1099400030E048EC52E4C701B6010E94FB9E87FF5D
:1099500002C021E001C020E0B701A601CE010796B8
:109960000E943A9B68EF75E0CE0101960E94189A1A
:10997000BE01695F7F4FCE0101960E943F9C6DEF53
:1099800075E00E94509CBC0180EC9CE00E94829A91
:10999000CE0101960E94AD99CE0107960E94AD9925
:1099A00060EC7CE0CE0101960E94979A42E350E081
:1099B0006FEF7FEFCE0101960E942C0CCE01019635
:1099C0000E94AD9960E073E08AEB9CE00E94969B58
:1099D0006AEB7CE0CE0101960E94979A42E350E048
:1099E00060E070E0CE0101960E94A00ACE010196CF
:1099F0000E94AD998091B10C882331F060E273E050
:109A000080E090E00E94D38F2C960FB6F894DEBFD2
:109A10000FBECDBFDF91CF911F910F91FF90EF90BF
:109A2000DF90CF9008954F925F926F927F928F92C6
:109A30009F92AF92BF92CF92DF92EF92FF92CF931D
:109A4000DF93CDB7DEB760970FB6F894DEBF0FBED9
:109A5000CDBF8091B10C811105C08EE190E0A0E0F6
:109A6000B0E004C082E090E0A0E0B0E08D879E8787
:109A7000AF87B88B69EA73E080EC9CE00E94969B0C
:109A800060EC7CE0CE0101960E94979A4AE050E09B
:109A90006FEF7FEFCE0101960E942C0CCE01019654
:109AA0000E94AD99812C912C5401C12CD12C7601AE
:109AB00063E270E085EC9EE00E942A8667E070E039
:109AC00085EC9EE00E94000A85EC9EE00E949E8646
:109AD00066E970E080E090E00E94D38F63E270E07E
:109AE00085EC9EE00E942A8660E270E085EC9EE0B4
:109AF0000E94000A85EC9EE00E949E8666E970E066
:109B000080E090E00E94D38F42E050E063E270E09A
:109B100085EC9EE00E949C86412C512C320185EC04
:109B20009EE00E948285181619066CF485EC9EE072
:109B30000E948A85762C652C542C4424480E511C96
:109B4000611C711CECCFC301B2010E94CB9F2AE9BA
:109B500039E949E95FE30E94FF9E0E94989FAB01AB
:109B6000BC01C416D506E606F70614F46A017B01AB
:109B70002AE0CE0107960E940E9BBE01695F7F4FCF
:109B8000CE0101960E94979A6BE177E0CE01019693
:109B90000E94509CBC018AEB9CE00E94829ACE01FC
:109BA00001960E94AD99CE0107960E94AD996AEB8D
:109BB0007CE0CE0101960E94979A4EE150E060E071
:109BC00070E0CE0101960E94550BCE0101960E94D5
:109BD000AD999FEF891A990AA90AB90A8D859E85C0
:109BE000AF85B88988159905AA05BB050CF060CF2B
:109BF0002AE0B701A601CE0107960E940E9BBE0186
:109C0000695F7F4FCE0101960E94979A6BE177E0E2
:109C1000CE0101960E94509CBC018AEB9CE00E9400
:109C2000829ACE0101960E94AD99CE0107960E94BC
:109C3000AD996AEB7CE0CE0101960E94979A4AE0CA
:109C400050E060E070E0CE0101960E94A00ACE01D3
:109C500001960E94AD992AE0B701A601CE010796B0
:109C60000E940E9B6FE177E0CE0101960E94189A48
:109C7000BE01695F7F4FCE0101960E943F9C62E268
:109C800077E00E94509C60EC7CE00E943F9CBC010D
:109C900080EC9CE00E94829ACE0101960E94AD99D0
:109CA000CE0107960E94AD9962E370E080E090E0FB
:109CB0000E94D38F60960FB6F894DEBF0FBECDBF63
:109CC000DF91CF91FF90EF90DF90CF90BF90AF905A
:109CD0009F908F907F906F905F904F9008958F929C
:109CE0009F92AF92BF92CF92DF92EF92FF920F932B
:109CF0001F93CF93DF93CDB7DEB72C970FB6F894B1
:109D0000DEBF0FBECDBF8C01E090AD0CF090AE0C6D
:109D10008091AF0C882369F06FE379E08EE89FE0D3
:109D20000E942D964AE050E0B8018EE89FE00E9424
:109D30004F97C8010596059708F18091AD0C909159
:109D4000AE0C8017910709F10E94F30C0E94743247
:109D50001093AE0C0093AD0C4AE0B801CE01019611
:109D60000E94E39ABE016F5F7F4F8CEC9CE00E94E3
:109D70009F9ACE0101960E94AD9907C00E3F8FEFCA
:109D80001807A9F40E9487324FC261E475E0CE0142
:109D900001960E94189A4AE050E06FEF7FEFCE01E3
:109DA00001960E94550BCE0101960E94AD99F801D3
:109DB0007996E533F10508F0D6C1EE58FF4F0C94C3
:109DC000E0A28091B10C882319F00E947739F9C183
:109DD00060910A0270910B0280910C0290910D0229
:109DE0000E946837EEC18091E4049091E5040E94DE
:109DF000A232E7C18091C8049091C9049BD8E1C107
:109E00008091BC049091BD040E948330DAC180919E
:109E1000BE049091BF04B5DCD4C10E94A48F0E94FF
:109E2000D841CFC160E070E08091C2049091C3043A
:109E30000E94402AC6C18091B8049091B9040E9442
:109E4000372EBFC18091B00C91E089278093B00C70
:109E50008091B10C882331F060EC7CE085E691E1E3
:109E60000E94799668EC70E080E090E00E94D38FC9
:109E7000A8C11092B10CA5C181E08093B10C6CEC2B
:109E80007CE082ED9CE00E94829A8091AD0C9091E2
:109E9000AE0C9093AC0C8093AB0C93C10E94E50D7B
:109EA00090C10E9437458DC10E9449198AC1809195
:109EB0003C02882309F485C16AE37BE0CE01019668
:109EC0000E94189A4AE050E061E070E0CE010196ED
:109ED0000E94A00ACE0101960E94AD990E94361000
:109EE00070C1A1DD6EC18091C4049091C5040E942F
:109EF000C42F67C18091BA049091BB040E94CE2EFA
:109F000060C180913C02882309F45BC18091B10C4F
:109F1000882329F082E090E00E94811252C183E000
:109F200090E00E94B0164DC10E94432885E691E161
:109F30000E942B9246C180918102909182020E94E0
:109F4000692C3FC180913C02882309F43AC1809179
:109F5000B10C811127C0C0900A02D0900B02E09092
:109F60000C02F0900D0220E030E04AE754E4C70113
:109F7000B6010E945FA10E94989F4B015C0120E006
:109F800030E040EA50E4C701B6010E945FA120E042
:109F900030E040EA50E40E94359E0E94989FA5015F
:109FA000940108C021E030E040E050E06AE070E059
:109FB00080E090E00E947C2204C18091010C90918D
:109FC000020C892BF1F581E090E09093020C8093D4
:109FD000010C67E277E0CE0101960E94189ACE014B
:109FE00001960E94740ACE0101960E94AD996FE11C
:109FF00075E0CE0107960E94189A6EEC7DE0CE01C6
:10A0000007960E943F9CBC01CE0101960E94979A40
:10A0100048EC50E06FEF7FEFCE0101960E94A00A5E
:10A02000CE0101960E94AD99CE0107960E94AD998E
:10A0300085E691E10E94129340E052EC61E070E00D
:10A040003BC01092020C1092010C60E377E0CE014D
:10A0500001960E94189ACE0101960E94740ACE01C0
:10A0600001960E94AD996BE175E0CE0107960E94C2
:10A07000189A6EEC7DE0CE0107960E943F9CBC01D1
:10A08000CE0101960E94979A48EC50E06FEF7FEF67
:10A09000CE0101960E94A00ACE0101960E94AD99C0
:10A0A000CE0107960E94AD9985E691E10E94129338
:10A0B00040E855E260E070E085E691E10E94FD092C
:10A0C0001092420C1092410C80E090E00E94270A0E
:10A0D00065E275E0CE0107960E94189A68EC7DE073
:10A0E000CE0107960E943F9CBC01CE0101960E94C2
:10A0F000979A40ED57E06FEF7FEFCE0101960E94F7
:10A100002C0CCE0101960E94AD99CE0107960E94BB
:10A11000AD9957C08091F20D9091F30D892BA1F468
:10A1200081E090E09093F30D8093F20D8EED93E03B
:10A130009093420C8093410C0E94500A68EC70E0AE
:10A1400080E090E00E94D38FE091680BF091690B62
:10A15000199537C082EE9DE00E9440700E94F30C7A
:10A160000E9474322EC0F092AE0CE092AD0C62E30D
:10A1700079E080EC9CE00E94969B6AE37BE0CE0154
:10A1800001960E94189A4AE050E060E070E0CE012B
:10A1900001960E94A00ACE0101960E94AD9960EC42
:10A1A0007CE0CE0101960E94979A4AE050E06FEF62
:10A1B0007FEFCE0101960E942C0CCE0101960E94E9
:10A1C000AD998091C40C9091C50C009799F041977E
:10A1D00018F402301105ACF460EC7CE0CE0101967D
:10A1E0000E94979ACE0101960E949E11CE0101967F
:10A1F0000E94AD9964E670E080E090E00E94D38F09
:10A2000013C060EC7CE0CE0101960E94979A4AE070
:10A2100050E06FEF7FEFCE0101960E942C0CCE0133
:10A2200001960E94AD99D8CF2C960FB6F894DEBF58
:10A230000FBECDBFDF91CF911F910F91FF90EF9097
:10A24000DF90CF90BF90AF909F908F900895FF9236
:10A250000F931F93CF93DF9300D000D0CDB7DEB71D
:10A26000823409F441C0CCF4803309F45DC07CF43D
:10A27000833209F450C08A3209F075C061E577E095
:10A2800088ED9CE00E94B59A8FEF9FEF6AC0813302
:10A2900009F459C08134E9F066C08136D1F02CF45C
:10A2A000833469F1843439F05EC0833641F1E4F0DF
:10A2B000843609F058C08091D00C9091D10C892B34
:10A2C00009F4E3C08CEC9CE00E940E9E97FF68C0EE
:10A2D000DCC065E477E088ED9CE00E94B59A80914F
:10A2E000AD0C9091AE0C3DC068E477E088ED9CE049
:10A2F0000E94B59A1092B10C8CEF9FEF32C06BE4C4
:10A3000077E088ED9CE00E94B59A81E08093B10CE3
:10A310008DEF9FEF26C06EE477E088ED9CE00E9411
:10A32000B59A8EEF9FEF1DC064E677E08CEC9CE061
:10A330000E94B59A64E677E088ED9CE00E94B59AA9
:10A3400080E090E00EC062E577E08CEC9CE00E943B
:10A35000B59A62E577E088ED9CE00E94B59A81E0CD
:10A3600090E0BDDC9AC0682FCE0101960E94CB9A86
:10A37000BE016F5F7F4F8CEC9CE00E949F9ACE01E4
:10A3800001960E94AD998CEC9CE00E940E9ECB0140
:10A39000A6DC64E670E080E090E00E94D38F7DC090
:10A3A0008091AF0C882361F06EE377E08EE89FE048
:10A3B0000E945E966CEC7CE08EE89FE00E947996AD
:10A3C0008CEC9CE00E940E9EDC01CB014AEF5FEF1B
:10A3D0006FEF7FEF481B590B6A0B7B0B2AE0CE0116
:10A3E00001960E940E9BBE016F5F7F4F8CEC9CE03C
:10A3F0000E949F9ACE0101960E94AD998CEC9CE040
:10A4000040C00F5F1F4F093E83E0180769F06EE1FF
:10A4100070E080E090E00E94D38F8DE49DE00E9488
:10A42000C86EF82EFF2069F36AE270E06F197109B7
:10A43000F7FC73954AE0CE0101960E94E39ABE01B3
:10A440006F5F7F4F88ED9CE00E949F9ACE0101963E
:10A450000E94AD9968ED7CE08CEC9CE00E94829AB1
:10A460008091AF0C882359F06EE377E08EE89FE08F
:10A470000E945E966F2D8EE89FE00E94999688ED6F
:10A480009CE00E940E9ECB016CCF8DE49DE00E946B
:10A49000C86EF82E00E010E0C5CF26960FB6F894EF
:10A4A000DEBF0FBECDBFDF91CF911F910F91FF9007
:10A4B00008950F931F93CF93DF9300D000D0CDB7B3
:10A4C000DEB78091AF0C8823A1F064E577E08EE8D9
:10A4D0009FE00E945E9640917E0B50917F0B6091B1
:10A4E000800B7091810B20E130E08EE89FE00E94AC
:10A4F000969780917E0B90917F0BA091800BB091ED
:10A50000810B883025E09207A105B10509F4FCC153
:10A5100008F08DC0893421E09207A105B10509F446
:10A52000F6C1E0F5843421E09207A105B10509F4F4
:10A53000DFC1E8F4813421E09207A105B10509F4F7
:10A54000C8C138F480349140A105B10509F4B2C105
:10A55000E1C1823421E09207A105B10509F4C2C12D
:10A5600083349140A105B10509F4BFC1D3C186343C
:10A5700021E09207A105B10509F4C0C108F4BBC1EF
:10A58000873421E09207A105B10509F4BAC18834E6
:10A590009140A105B10509F4B7C1BCC1823025E0E5
:10A5A0009207A105B10509F49DC1E8F4843721E0C3
:10A5B0009207A105B10509F448C138F482379140EA
:10A5C000A105B10509F44CC1A5C1811525E092078B
:10A5D000A105B10509F46EC181309540A105B10511
:10A5E00009F477C197C1853025E09207A105B1052F
:10A5F00009F481C170F4833025E09207A105B1050B
:10A6000009F473C184309540A105B10509F470C106
:10A6100081C1863025E09207A105B10509F46EC11C
:10A6200087309540A105B10509F46BC173C18D3B1D
:10A6300022E492072FEFA207B10509F42CC108F01C
:10A640004BC08F3E20E192072FEFA207B10509F41E
:10A6500058C118F5823325E09207A105B10509F428
:10A66000FFC038F489309540A105B10509F44FC108
:10A6700051C1843325E09207A105B10509F4E5C075
:10A680008D3F9240AF4FB10509F044C165E477E0DA
:10A6900088ED9CE00E94B59AE0C08D3D22E29207D1
:10A6A0002FEFA207B10509F4D0C038F4873E9841D6
:10A6B000AF4FB10509F41FC12DC18F3C20E39207B4
:10A6C0002FEFA207B10509F413C1873C9843AF4FA0
:10A6D000B10509F419C11EC1873928E692072FEF89
:10A6E000A207B10509F4F5C048F58D3A22E59207B5
:10A6F0002FEFA207B10509F4BFC038F4853B9A4497
:10A70000AF4FB10509F4D6C005C1853A2AE59207D5
:10A710002FEFA207B10509F4FAC08D399246AF4F69
:10A72000B10509F0F7C068E477E088ED9CE00E948D
:10A73000B59A1092B10C8CEF9FEF85C0873528EA4F
:10A7400092072FEFA207B105F9F078F485382AE7D0
:10A7500092072FEFA207B10509F4D0C087369849B8
:10A76000AF4FB10509F4BEC0D5C08F3420EB9207BE
:10A770002FEFA207B10509F4B8C08D33924CAF4F4B
:10A78000B10509F46DC0C6C08AE89BE00E947472EE
:10A7900000E010E06AE67BE08AE89BE00E94297313
:10A7A000892B39F40F5F1F4F093E83E0180709F02A
:10A7B0009DC18091AF0C8823A1F06FE179E08EE814
:10A7C0009FE00E942D9640916E0B50916F0B60910F
:10A7D000700B7091710B2AE030E08EE89FE00E94D0
:10A7E000969780916E0B90916F0BA091700BB0912A
:10A7F000710B853025E09207A105B10509F461C10F
:10A8000008F0E1C0873421E09207A105B10509F401
:10A8100064C108F0B8C0833421E09207A105B105F6
:10A8200009F43DC108F0A5C0813421E09207A105DB
:10A83000B10509F097C069E577E08CEC9CE00E94D7
:10A84000B59A89EF9FEF4BDA7EC065E477E088ED3B
:10A850009CE00E94B59A1092B10C8BEF9FEFF3CF62
:10A860006BE477E088ED9CE00E94B59A81E08093EC
:10A87000B10C8DEF9FEFE7CF6EE477E08CEC9CE0BE
:10A880000E94B59A6EE477E088ED9CE00E94B59A4C
:10A890008EEF9FEFD8CF61E577E08CEC9CE00E94D3
:10A8A000B59A61E577E088ED9CE00E94B59A8FEF5C
:10A8B0009FEFC9CF64E677E08CEC9CE00E94B59AEC
:10A8C00064E677E088ED9CE00E94B59A80E090E035
:10A8D000BACF62E577E08CEC9CE00E94B59A81E00B
:10A8E00090E0B1CF82E090E0AECF83E090E0ABCFDC
:10A8F00084E090E0A8CF85E090E0A5CF86E090E0EE
:10A90000A2CF87E090E09FCF88E090E09CCF89E0E5
:10A9100090E099CF40E050E068ED7CE0CE010196F8
:10A920000E94F109BE016F5F7F4F8CEC9CE00E949A
:10A930009F9ACE0101960E94AD9964E670E080E096
:10A9400090E00E94D38F8AE89BE00E947472269662
:10A950000FB6F894DEBF0FBECDBFDF91CF911F9130
:10A960000F91089582349140A105B10509F48EC07C
:10A97000E4CF853421E09207A105B10509F4A1C017
:10A9800008F496C0A7C0813025E09207A105B10563
:10A9900009F451CF70F4883421E09207A105B10584
:10A9A00009F49EC089349140A105B10509F49BC00A
:10A9B000C4CF833025E09207A105B10509F46FC02B
:10A9C00008F464C075C08F3C20E392072FEFA20704
:10A9D000B10509F46DC068F5883025E09207A1053E
:10A9E000B10509F47DC070F4863025E09207A10519
:10A9F000B10509F46FC087309540A105B10509F490
:10AA00006CC09BCF8F3E20E192072FEFA207B105CC
:10AA100009F463C0873E28E192072FEFA207B10532
:10AA200009F44FC089309540A105B10509F085CFE3
:10AA30005AC0873928E692072FEFA207B10509F41B
:10AA4000FACE78F4873C28E392072FEFA207B105EE
:10AA500009F446C0853A9A45AF4FB10509F443C0A1
:10AA60006CCF873628E992072FEFA207B10571F066
:10AA70008F3420EB92072FEFA207B10581F08538C4
:10AA80009A47AF4FB10509F058CF24C06CE577E085
:10AA90008CEC9CE00E94B59A88EF9FEFD4CE6FE5D6
:10AAA00077E08CEC9CE00E94B59A87EF9FEFCBCECD
:10AAB00062E677E08CEC9CE00E94B59A86EF9FEF0F
:10AAC000C2CE66E677E08CEC9CE00E94B59A85EFFA
:10AAD0009FEFB9CE84EF9FEFB6CE83EF9FEFB3CE5B
:10AAE00082EF9FEFB0CE81EF9FEFADCE6EE170E0D1
:10AAF00080E090E00E94D38F4DCE8F929F92AF92D4
:10AB0000BF92CF92DF92EF92FF920F931F93CF935A
:10AB1000DF93CDB7DEB7A6970FB6F894DEBF0FBEB2
:10AB2000CDBF6AE77BE08AE89BE00E942973892B0E
:10AB300019F0BFDC0C94FB676AE37BE088ED9CE0D6
:10AB40000E94B59A0E9499496AE070E080E090E026
:10AB50000E94D38F8091DC0C9091DD0C009711F452
:10AB60000C94DD67019709F046C061E076E0CE0104
:10AB70000F960E94189ABE01615F7F4F88ED9CE09E
:10AB80000E94CE9C81112AC06BEF76E0CE0109961F
:10AB90000E94189ABE01675F7F4F88ED9CE00E947B
:10ABA000CE9C811115C068E875E0CE0101960E9427
:10ABB000189ABE016F5F7F4F88ED9CE00E94CE9C8B
:10ABC00011E0811110E0CE0101960E94AD9901C003
:10ABD00010E0CE0109960E94AD9901C010E0CE01AF
:10ABE0000F960E94AD99112331F068ED7CE08CEC5A
:10ABF0009CE00E94829A8091DC0C9091DD0C04977D
:10AC0000F0F56AE677E0CE0101960E94189ABE013F
:10AC10006F5F7F4F88ED9CE00E94CE9C182FCE0185
:10AC200001960E94AD99112351F141E050E068ED89
:10AC30007CE0CE0109960E94F109CE0109960E949E
:10AC40000E9EDC01CB014AEF5FEF6FEF7FEF481BF9
:10AC5000590B6A0B7B0B2AE0CE0101960E940E9BDA
:10AC6000BE016F5F7F4F8CEC9CE00E949F9ACE01EB
:10AC700001960E94AD99CE0109960E94AD996CE6AD
:10AC800077E0CE0109960E94189ABE01675F7F4F58
:10AC900088ED9CE00E94CE9C811116C060E777E0B1
:10ACA000CE0101960E94189ABE016F5F7F4F88ED1A
:10ACB0009CE00E94CE9C11E0811101C010E0CE0109
:10ACC00001960E94AD9901C011E0CE0109960E9443
:10ACD000AD99112309F442C364E777E0CE010196F0
:10ACE0000E94189ACE0101960E949E11CE010196F3
:10ACF0000E94AD9960E877E0CE0109960E94189A0B
:10AD00006EEC7DE0CE0109960E943F9CBC01CE0115
:10AD100001960E94979ACE0101960E949E11CE0143
:10AD200001960E94AD99CE0109960E94AD9960915D
:10AD300038027091390280913A0290913B020E9450
:10AD4000CB9F20E030E048EC52E40E94FF9EAB0134
:10AD5000BC0122E0CE010F960E943A9B66E977E0A3
:10AD6000CE0109960E94189ABE01615F7F4FCE0105
:10AD700009960E943F9C61EE78E00E94509CBC01C5
:10AD8000CE0101960E94979ACE0101960E949E11D3
:10AD9000CE0101960E94AD99CE0109960E94AD990F
:10ADA000CE010F960E94AD99409134025091350228
:10ADB000609136027091370224E0CE010F960E9416
:10ADC0003A9B6BEA77E0CE0109960E94189ABE0181
:10ADD000615F7F4FCE0109960E943F9CBC01CE016E
:10ADE00001960E94979ACE0101960E949E11CE0173
:10ADF00001960E94AD99CE0109960E94AD99CE01AF
:10AE00000F960E94AD9940911E0250911F026091D1
:10AE100020027091210222E0CE0109960E943A9B05
:10AE20004091160250911702609118027091190218
:10AE300023E0CE010F960E943A9B4091220250914E
:10AE40002302609124027091250222E0CE014596F2
:10AE50000E943A9B40911A0250911B0260911C0281
:10AE600070911D0223E0CE0181960E943A9B68EC0E
:10AE700077E0CE014B960E94189ABE016F5D7F4F1E
:10AE8000CE014B960E943F9C6DED77E00E94509C56
:10AE9000BE016B5E7F4F0E943F9C60EE77E00E9498
:10AEA000509CBE01615F7F4F0E943F9C6DED77E03B
:10AEB0000E94509CBE01675F7F4F0E943F9C66EEE0
:10AEC00077E00E94509CBC01CE0101960E94979AA7
:10AED000CE0101960E949E11CE0101960E94AD996D
:10AEE000CE014B960E94AD99CE0181960E94AD99FC
:10AEF000CE0145960E94AD99CE010F960E94AD9964
:10AF0000CE0109960E94AD994091450250914602AA
:10AF1000609147027091480223E0CE0109960E9499
:10AF20003A9B2091490230914A0240914B02509144
:10AF30004C0260E070E080E291E40E94C2A1AB01AB
:10AF4000BC0121E0CE0145960E94689B6BEE77E044
:10AF5000CE010F960E94189ABE016B5E7F4FCE0104
:10AF60000F960E943F9C6EEF77E00E94509CBE01BE
:10AF7000675F7F4F0E943F9C63E076E00E94509C99
:10AF8000BC01CE0101960E94979ACE0101960E94C3
:10AF90009E11CE0101960E94AD99CE010F960E949E
:10AFA000AD99CE0145960E94AD99CE0109960E94B9
:10AFB000AD994091410250914202609143027091DB
:10AFC000440223E0CE0109960E943A9B20913D0263
:10AFD00030913E0240913F025091400260E070E0AB
:10AFE00080E291E40E94C2A1AB01BC0121E0CE014C
:10AFF00045960E94689B64E078E0CE010F960E941F
:10B00000189ABE016B5E7F4FCE010F960E943F9C47
:10B010006EEF77E00E94509CBE01675F7F4F0E94F9
:10B020003F9C63E076E00E94509CBC01CE010196FB
:10B030000E94979ACE0101960E949E11CE01019620
:10B040000E94AD99CE010F960E94AD99CE01459612
:10B050000E94AD99CE0109960E94AD9940914D0292
:10B0600050914E0260914F027091500222E0CE0149
:10B070000F960E943A9B67E178E0CE0109960E9404
:10B08000189ABE01615F7F4FCE0109960E943F9CD6
:10B090006DE278E00E94509CBC01CE0101960E94B6
:10B0A000979ACE0101960E949E11CE0101960E94B0
:10B0B000AD99CE0109960E94AD99CE010F960E94DE
:10B0C000AD99409112025091130260911402709157
:10B0D000150222E0CE010F960E943A9B64E378E0CD
:10B0E000CE0109960E94189ABE01615F7F4FCE0182
:10B0F00009960E943F9C63E076E00E94509CBC0150
:10B10000CE0101960E94979ACE0101960E949E114F
:10B11000CE0101960E94AD99CE0109960E94AD998B
:10B12000CE010F960E94AD9916E9C12E14E0D12EE2
:10B1300001E010E087E1E82E80919404909195045D
:10B14000801791070CF44FC0D601AD90BD906D01F2
:10B150004AE0B501CE0109960E94E39A4AE0B8019F
:10B16000CE0145960E94E39A67E478E0CE010F96FF
:10B170000E94189ABE016B5E7F4FCE010F960E940F
:10B180003F9C64E178E00E94509CBE01675F7F4F66
:10B190000E943F9C6FE478E00E94509CEA9CB001C2
:10B1A000EB9C700D11246D577D4F0E94509CBC018B
:10B1B000CE0101960E94979ACE0101960E949E119F
:10B1C000CE0101960E94AD99CE010F960E94AD99D5
:10B1D000CE0145960E94AD99CE0109960E94AD9987
:10B1E0000F5F1F4FA9CF8091010C9091020C892B0A
:10B1F00071F465E578E0CE0101960E94189ACE01BF
:10B2000001960E949E11CE0101960E94AD998091F7
:10B21000010C9091020C019771F464E678E0CE0184
:10B2200001960E94189ACE0101960E949E11CE01AD
:10B2300001960E94AD996091FE047091FF044AE06E
:10B24000CE010F960E94E39A6EE678E0CE01099651
:10B250000E94189ABE01615F7F4FCE0109960E943D
:10B260003F9CBC01CE0101960E94979ACE010196A7
:10B270000E949E11CE0101960E94AD99CE010996C1
:10B280000E94AD99CE010F960E94AD9940910E0299
:10B2900050910F02609110027091110222E0CE01D4
:10B2A0000F960E943A9B6AE878E0CE0109960E94C8
:10B2B000189ABE01615F7F4FCE0109960E943F9CA4
:10B2C00066E876E00E94509CBC01CE0101960E9487
:10B2D000979ACE0101960E949E11CE0101960E947E
:10B2E000AD99CE0109960E94AD99CE010F960E94AC
:10B2F000AD9940910A0250910B0260910C0270913D
:10B300000D0222E0CE010F960E943A9B6AE978E096
:10B31000CE0109960E94189ABE01615F7F4FCE014F
:10B3200009960E943F9C66E876E00E94509CBC0112
:10B33000CE0101960E94979ACE0101960E949E111D
:10B34000CE0101960E94AD99CE0109960E94AD9959
:10B35000CE010F960E94AD9910E001C011E08091DE
:10B36000DC0C9091DD0C039708F08EC00E947432C3
:10B370000E94F30C61E475E0CE0101960E94189AD8
:10B380004AE050E060E070E0CE0101960E94550B6B
:10B39000CE0101960E94AD998091DC0C9091DD0C5C
:10B3A000019739F460E070E088ED9CE00E94ED9C2C
:10B3B000F82E8091DC0C9091DD0C029709F055C0BD
:10B3C0006AE677E0CE0101960E94189ABE016F5F8F
:10B3D0007F4F88ED9CE00E94CE9C182FCE010196F5
:10B3E0000E94AD99112309F440C061E070E088ED3E
:10B3F0009CE00E94ED9C682FCE0101960E94CB9AA2
:10B40000BE016F5F7F4F8CEC9CE00E94AA9ACE0138
:10B4100001960E94AD9960E070E088ED9CE00E948A
:10B42000ED9CF82E8091AF0C8823F9F06AEA78E061
:10B43000CE0101960E94189A68ED7CE0CE0101963B
:10B440000E943F9C61E475E00E94509CBC018EE824
:10B450009FE00E945096CE0101960E94AD996CEC3F
:10B460007CE08EE89FE00E9479968F2D0E94275104
:10B470000E94A48F6093DE0C7093DF0C8093E00C2D
:10B480009093E10C0C94FB6721E030E040E050E049
:10B4900068ED7CE0CE0101960E946F9DBE016F5F5A
:10B4A0007F4F8AEB9CE00E949F9ACE0101960E94FA
:10B4B000AD996DED78E0CE0109960E94189ABE0113
:10B4C000675F7F4F88ED9CE00E94CE9C811116C083
:10B4D0006DED75E0CE0101960E94189ABE016F5F76
:10B4E0007F4F88ED9CE00E94CE9C01E0811101C05D
:10B4F00000E0CE0101960E94AD9901C001E0CE01AD
:10B5000009960E94AD99002309F4DCC042E050E0A6
:10B5100068ED7CE0CE0101960E94F109BE016F5FEB
:10B520007F4F8AEB9CE00E949F9ACE0101960E9479
:10B53000AD996AEB7CE0CE0101960E94979ACE010C
:10B5400001960E94740ACE0101960E94AD998AEB81
:10B550009CE00E94189E20E030E048EC52E40E94FB
:10B560005FA10E94989FAB01BC01409338025093A9
:10B57000390260933A0270933B022AE0CE010196B1
:10B580000E940E9BCE0101960E94740ACE01019684
:10B590000E94AD99609138027091390280913A020F
:10B5A00090913B028B019C0100591F4521403109BC
:10B5B00001341C4921053105D0F060EB78E0CE0163
:10B5C00001960E94189A6AEB7CE0CE0101960E94D7
:10B5D0003F9C63EC78E00E94509CBC0180EC9CE0B6
:10B5E0000E94829ACE0101960E94AD994DC01982A7
:10B5F0001A821B821C821D821E821F8218860E9454
:10B60000CB9F20E030E048EC52E40E94FF9E8E0188
:10B610000F5F1F4F22E047E00E9440A3BC0180EC77
:10B620009CE00E94B59A63ED78E0CE0109960E94F5
:10B63000189A60EC7CE0CE0109960E943F9C60EE77
:10B6400078E00E94509CBC0180EC9CE00E94829AB1
:10B65000CE0109960E94AD991092420C1092410CB5
:10B660008091380290913902A0913A02B0913B0248
:10B6700080938B0B90938C0BA0938D0BB0938E0BC0
:10B6800080E090E00E94270A61EB76E0CE01099607
:10B690000E94189A60EC7CE0CE0109960E943F9CC3
:10B6A000BC01CE0101960E94979ACE0101960E949C
:10B6B0009E11CE0101960E94AD99CE0109960E947D
:10B6C000AD99F3C065EE78E0CE0109960E94189A14
:10B6D000BE01675F7F4F88ED9CE00E94CE9C811188
:10B6E00016C06BEE78E0CE0101960E94189ABE015A
:10B6F0006F5F7F4F88ED9CE00E94CE9C01E081113E
:10B7000001C000E0CE0101960E94AD9901C001E0A8
:10B71000CE0109960E94AD99002309F475C026E078
:10B7200030E045E050E068ED7CE0CE0101960E94FB
:10B730006F9DBE016F5F7F4F8AEB9CE00E949F9AD6
:10B74000CE0101960E94AD998AEB9CE00E940E9E6C
:10B750006B017C016BE278E0CE0109960E94189A99
:10B76000BE01675F7F4F88ED9CE00E94669DAC0143
:10B770004F5F5F4F68ED7CE0CE0101960E94F109BA
:10B78000BE016F5F7F4F8AEB9CE00E949F9ACE01C3
:10B7900001960E94AD99CE0109960E94AD998AEB5F
:10B7A0009CE00E940E9EDB01E6E9F4E021E030E03F
:10B7B0004091940450919504421753075CF04081E6
:10B7C00051814A175B0711F4118210822F5F3F4F9E
:10B7D0003296EECFF601EE0FFF1FEC56FB4F718352
:10B7E000608382E090E00E94373168ED7CE0CE011A
:10B7F00001960E94979ACE0101960E94740ACE018A
:10B8000001960E94AD9949C061EF78E0CE0109969A
:10B810000E94189ABE01675F7F4F88ED9CE00E94EE
:10B82000CE9C811116C067EF78E0CE0101960E9490
:10B83000189ABE016F5F7F4F88ED9CE00E94CE9CFE
:10B8400001E0811101C000E0CE0101960E94AD9996
:10B8500001C001E0CE0109960E94AD99002331F1AB
:10B86000E6E9F4E081E090E02091940430919504C1
:10B870002817390774F0863091051CF49183808372
:10B8800005C09C012E5F3F4F318320830196329685
:10B89000EBCF82E090E00E9437311092420C109280
:10B8A000410C80E090E00E94270A10E06DEF78E004
:10B8B000CE0109960E94189ABE01675F7F4F88EDFE
:10B8C0009CE00E94CE9C811116C065E079E0CE011B
:10B8D00001960E94189ABE016F5F7F4F88ED9CE031
:10B8E0000E94CE9C01E0811101C000E0CE010196D2
:10B8F0000E94AD9901C001E0CE0109960E94AD9968
:10B90000002349F06DE079E0CE0101960E94189A7B
:10B9100068EC7DE034C067E179E0CE0109960E94D1
:10B92000189ABE01675F7F4F88ED9CE00E94CE9C15
:10B93000811116C06EE179E0CE0101960E94189A3D
:10B94000BE016F5F7F4F88ED9CE00E94CE9C01E0BE
:10B95000811101C000E0CE0101960E94AD9901C0A5
:10B9600001E0CE0109960E94AD990023A1F168E89B
:10B9700077E0CE0101960E94189A6EEC7DE0CE0130
:10B9800001960E943F9CBC0180EC9CE00E94829A40
:10B99000CE0101960E94AD9961EB76E0CE01099649
:10B9A0000E94189A60EC7CE0CE0109960E943F9CB0
:10B9B000BC01CE0101960E94979ACE0101960E9489
:10B9C0009E11CE0101960E94AD99CE0109960E946A
:10B9D000AD990C94FB6765E279E0CE0109960E946F
:10B9E000189ABE01675F7F4F88ED9CE00E94CE9C55
:10B9F000811116C06AE279E0CE0101960E94189A80
:10BA0000BE016F5F7F4F88ED9CE00E94CE9C01E0FD
:10BA1000811101C000E0CE0101960E94AD9901C0E4
:10BA200001E0CE0109960E94AD990023D9F16BE2A5
:10BA300078E0CE0109960E94189ABE01675F7F4F99
:10BA400088ED9CE00E94669DAC014F5F5F4F68ED02
:10BA50007CE0CE0101960E94F109BE016F5F7F4F2D
:10BA60008AEB9CE00E949F9ACE0101960E94AD99BC
:10BA7000CE0109960E94AD998AEB9CE00E940E9E31
:10BA80006115710521F481E08093FB0407C06130EA
:10BA9000710511F00C94FB671092FB040E94873231
:10BAA0000C94FB676FE279E0CE0109960E94189A28
:10BAB000BE01675F7F4F88ED9CE00E94CE9C8111A4
:10BAC00016C063E379E0CE0101960E94189ABE0188
:10BAD0006F5F7F4F88ED9CE00E94CE9C01E081115A
:10BAE00001C000E0CE0101960E94AD9901C001E0C5
:10BAF000CE0109960E94AD99002309F474C043E079
:10BB000050E068ED7CE0CE0101960E94F109BE0193
:10BB10006F5F7F4F8AEB9CE00E949F9ACE01019657
:10BB20000E94AD996AEB7CE0CE0101960E94979A43
:10BB3000CE0101960E94740ACE0101960E94AD9931
:10BB40001092420C1092410C6AEB7CE084ED9DE077
:10BB50000E94829A6AEB7CE08EEC9DE00E94829AC1
:10BB600020E030E048E050E067EA7BE084ED9DE0D3
:10BB70000E94EE9C20E030E04CE050E065E07CE08C
:10BB80008EEC9DE00E94EE9C8091410C9091420CC5
:10BB90000E94270A63EB76E0CE0101960E94189A74
:10BBA0006EEC7DE0CE0101960E943F9CBC01CE016F
:10BBB00009960E94979ACE0101960E94AD99BE0106
:10BBC000675F7F4F85E691E10E94509668EB7BE0CE
:10BBD00080E090E00E94D38F67EA7BE0CE0101967F
:10BBE0000E94189A69C067E379E0CE0109960E9425
:10BBF000189ABE01675F7F4F88ED9CE00E94CE9C43
:10BC0000811116C06CE379E0CE0101960E94189A6A
:10BC1000BE016F5F7F4F88ED9CE00E94CE9C01E0EB
:10BC2000811101C000E0CE0101960E94AD9901C0D2
:10BC300001E0CE0109960E94AD99002309F448C0A5
:10BC400044E050E068ED7CE0CE0101960E94F109ED
:10BC5000BE016F5F7F4F8AEB9CE00E949F9ACE01EE
:10BC600001960E94AD996BEB76E0CE0101960E94A1
:10BC7000189A6AEB7CE0CE0101960E943F9CBC01C1
:10BC8000CE0109960E94979ACE0101960E94AD9925
:10BC9000BE01675F7F4F85E691E10E94509668EB99
:10BCA0007BE080E090E00E94D38FBE01675F7F4F12
:10BCB000CE0101960E94979ACE0101960E94740AC5
:10BCC000CE0101960E94AD99CE0109960C94DA67D7
:10BCD00061E479E0CE0109960E94189ABE01675F7F
:10BCE0007F4F88ED9CE00E94CE9C811116C066E4D7
:10BCF00079E0CE0101960E94189ABE016F5F7F4FD6
:10BD000088ED9CE00E94CE9C01E0811101C000E022
:10BD1000CE0101960E94AD9901C001E0CE010996C5
:10BD20000E94AD990023F1F025E030E044E050E0BE
:10BD300068ED7CE0CE0101960E946F9DBE016F5FB1
:10BD40007F4F8AEB9CE00E949F9ACE0101960E9451
:10BD5000AD998AEB9CE00E940E9E7093020C60935A
:10BD6000010C4DC06BE479E0CE0109960E94189A4F
:10BD7000BE01675F7F4F88ED9CE00E94CE9C8111E1
:10BD800016C060E579E0CE0101960E94189ABE01C6
:10BD90006F5F7F4F88ED9CE00E94CE9C01E0811197
:10BDA00001C000E0CE0101960E94AD9901C001E002
:10BDB000CE0109960E94AD990023C9F126E030E03A
:10BDC00044E050E068ED7CE0CE0101960E946F9D5A
:10BDD000BE016F5F7F4F8AEB9CE00E949F9ACE016D
:10BDE00001960E94AD998AEB9CE00E940E9E709392
:10BDF000040C6093030C7093FF046093FE0468EDE1
:10BE00007CE0CE0101960E94979ACE0101960E9495
:10BE1000740ACE0101960E94AD991092420C1092C4
:10BE2000410C80E090E00E94270A0C94FB6765E5D6
:10BE300079E0CE0109960E94189ABE01675F7F4F94
:10BE400088ED9CE00E94CE9C811116C06CE579E0E3
:10BE5000CE0101960E94189ABE016F5F7F4F88ED58
:10BE60009CE00E94CE9C01E0811101C000E0CE0167
:10BE700001960E94AD9901C001E0CE0109960E9491
:10BE8000AD99002321F127E030E046E050E068ED75
:10BE90007CE0CE0101960E946F9DBE016F5F7F4FD7
:10BEA0008AEB9CE00E949F9ACE0101960E94AD9978
:10BEB0008AEB9CE00E940E9E672B21F41092AF0C3F
:10BEC0000C94CE6781E08093AF0C0C94CE6763E650
:10BED00079E0CE010F960E94189ABE01615F7F4FF4
:10BEE00088ED9CE00E94CE9C81112BC066E679E033
:10BEF000CE0109960E94189ABE01675F7F4F88EDB8
:10BF00009CE00E94CE9C811116C069E679E0CE01CA
:10BF100001960E94189ABE016F5F7F4F88ED9CE0EA
:10BF20000E94CE9C01E0811101C000E0CE0101968B
:10BF30000E94AD9901C001E0CE0109960E94AD9921
:10BF400001C001E0CE010F960E94AD99002309F4D3
:10BF50002DC1FAE0AF2EB12CC12CD12C7601882452
:10BF60008A94A3E09A2E6EE170E080E090E00E9457
:10BF7000D38F809181020E946990B4010E948FA2A8
:10BF8000882777FD8095982F0E94CB9F20E030E096
:10BF900040EA50E40E945FA19B01AC01C701B601D9
:10BFA0000E94359E6B017C01E1E0AE1AB108D9F622
:10BFB00020E030E040E251E40E94FF9E6B017C01F2
:10BFC0006CE679E0CE0109960E94189ABE01675F7F
:10BFD0007F4F88ED9CE00E94CE9C811116C060E7E7
:10BFE00079E0CE0101960E94189ABE016F5F7F4FE3
:10BFF00088ED9CE00E94CE9C01E0811101C000E030
:10C00000CE0101960E94AD9901C001E0CE010996D2
:10C010000E94AD99002309F43FC020E030E040E6E3
:10C0200050E4C701B6010E945FA19B01AC0160E032
:10C0300070E080E890E40E94349EAB01BC01409324
:10C040002A0250932B0260932C0270932D0222E05F
:10C05000CE0101960E943A9BBE016F5F7F4F80EC3C
:10C060009CE00E949F9ACE0101960E94AD9964E7E0
:10C0700079E0CE0101960E94189A60EC7CE0CE0136
:10C0800001960E943F9CBC0180EC9CE00E94829A39
:10C09000CE0101960E94AD9963E879E0CE01099640
:10C0A0000E94189ABE01675F7F4F88ED9CE00E9456
:10C0B000CE9C811116C068E879E0CE0101960E94FD
:10C0C000189ABE016F5F7F4F88ED9CE00E94CE9C66
:10C0D00001E0811101C000E0CE0101960E94AD99FE
:10C0E00001C001E0CE0109960E94AD99002309F438
:10C0F0003FC020E030E040E650E4C701B6010E94B6
:10C100005FA19B01AC0160E070E080E291E40E94DD
:10C11000349EAB01BC0140932602509327026093EA
:10C1200028027093290222E0CE0101960E943A9BD8
:10C13000BE016F5F7F4F80EC9CE00E949F9ACE0112
:10C1400001960E94AD996DE879E0CE0101960E94BA
:10C15000189A60EC7CE0CE0101960E943F9CBC01E5
:10C1600080EC9CE00E94829ACE0101960E94AD99DB
:10C1700061EB76E0CE0109960E94189A60EC7CE0B3
:10C18000CE0109960E943F9CBC01CE0101960E94FF
:10C19000979ACE0101960E949E11CE0101960E94AF
:10C1A000AD99CE0109960E94AD99F6C66DE979E088
:10C1B000CE0101960E94189ABE016F5F7F4F88EDF5
:10C1C0009CE00E94CE9C082FCE0101960E94AD9962
:10C1D000002309F46EC08091DC0C9091DD0C079770
:10C1E00008F4DAC646E050E068ED7CE0CE01019646
:10C1F0000E94F109BE016F5F7F4F8AEB9CE00E94B5
:10C200009F9ACE0101960E94AD998AEB9CE00E9414
:10C21000189EAB01BC0140930E0250930F02609335
:10C2200010027093110221E0CE0109960E943A9B00
:10C230006AE878E0CE0101960E94189ABE01675F15
:10C240007F4FCE0101960E943F9C66E876E00E94F7
:10C25000509CBC0180EC9CE00E94829ACE01019629
:10C260000E94AD99CE0109960E94AD9960EC7CE0E8
:10C27000CE0101960E94979ACE0101960E949E11CE
:10C28000CE0101960E94AD990E94A48F28EE33E062
:10C2900040E050E00E94A2A2CA01B9010E94C99FD9
:10C2A0006093150C7093160C8093170C9093180CD8
:10C2B00073C664EA79E0CE0101960E94189ABE0125
:10C2C0006F5F7F4F88ED9CE00E94CE9C082FCE01CF
:10C2D00001960E94AD990023E9F18091DC0C9091C8
:10C2E000DD0C079708F458C646E050E068ED7CE0A6
:10C2F000CE0101960E94F109BE016F5F7F4F8AEB6C
:10C300009CE00E949F9ACE0101960E94AD998AEB13
:10C310009CE00E94189EAB01BC0140930A0250931E
:10C320000B0260930C0270930D0221E0CE0109967E
:10C330000E943A9B6AE978E0CE0101960E94189A21
:10C34000BE01675F7F4FCE0101960E943F9C66E869
:10C3500076E0F5C16BEA79E0CE0109960E94189A61
:10C36000BE01675F7F4F88ED9CE00E94CE9C8111EB
:10C3700016C06FEA79E0CE0101960E94189ABE01BC
:10C380006F5F7F4F88ED9CE00E94CE9C01E08111A1
:10C3900001C000E0CE0101960E94AD9901C001E00C
:10C3A000CE0109960E94AD99002309F45AC08091EC
:10C3B000C2049091C3040E94152A60931A027093DC
:10C3C0001B0280931C0290931D0260939F0B70933D
:10C3D000A00B8093A10B9093A20B80E090E0A0E8CB
:10C3E000BFE38093220290932302A0932402B09390
:10C3F00025028093970B9093980BA093990BB09381
:10C400009A0B8091AF0C8823A1F064ED7CE08EE85C
:10C410009FE00E942D9640911A0250911B0260915C
:10C420001C0270911D0222E030E08EE89FE00E9425
:10C4300082981092420C1092410C80E090E00E9491
:10C44000270A40911A0250911B0260911C027091C0
:10C450001D0222E0CE0109960E943A9B63EB79E02F
:10C4600078C56CEB79E0CE0109960E94189ABE015E
:10C47000675F7F4F88ED9CE00E94CE9C811116C0C3
:10C4800062EC79E0CE0101960E94189ABE016F5FBE
:10C490007F4F88ED9CE00E94CE9C01E0811101C09D
:10C4A00000E0CE0101960E94AD9901C001E0CE01ED
:10C4B00009960E94AD99002309F469C08091DC0CB3
:10C4C0009091DD0C0797F8F046E050E068ED7CE0D5
:10C4D000CE0101960E94F109BE016F5F7F4F8AEB8A
:10C4E0009CE00E949F9ACE0101960E94AD998AEB32
:10C4F0009CE00E94189E60934D0270934E028093C0
:10C500004F02909350028091BC040E94FA308091B7
:10C510004D0290914E02A0914F02B0915002809333
:10C52000BF0B9093C00BA093C10BB093C20B809133
:10C53000AF0C8823A1F062EC7CE08EE89FE00E94C3
:10C540002D9640914D0250914E0260914F02709194
:10C55000500222E030E08EE89FE00E948298109224
:10C56000420C1092410C80E090E00E94270A40911A
:10C570004D0250914E0260914F027091500222E0A4
:10C58000CE0109960E943A9B68EC79E0E2C462ED24
:10C5900079E0CE0109960E94189ABE01675F7F4F2D
:10C5A00088ED9CE00E94CE9C811116C067ED79E079
:10C5B000CE0101960E94189ABE016F5F7F4F88EDF1
:10C5C0009CE00E94CE9C01E0811101C000E0CE0100
:10C5D00001960E94AD9901C001E0CE0109960E942A
:10C5E000AD99002309F4AEC08091DC0C9091DD0C74
:10C5F000069708F145E050E068ED7CE0CE01019639
:10C600000E94F109BE016F5F7F4F8AEB9CE00E94A0
:10C610009F9ACE0101960E94AD998AEB9CE00E9400
:10C62000189E0E94E1A06093490270934A02809391
:10C630004B0290934C028091BE049091BF040E94E3
:10C64000A82D20E030E048E051E40E94FF9E609376
:10C65000450270934602809347029093480260938C
:10C66000AF0B7093B00B8093B10B9093B20B809192
:10C67000490290914A02A0914B02B0914C028093E2
:10C68000B70B9093B80BA093B90BB093BA0B8091F2
:10C69000AF0C882381F161EB7CE08EE89FE00E9483
:10C6A0002D962091490230914A0240914B025091BF
:10C6B0004C0260E070E080E291E40E94C2A1AB0114
:10C6C000BC0121E030E08EE89FE00E9481986CED93
:10C6D00079E08EE89FE00E945E964091450250917D
:10C6E0004602609147027091480222E030E08EE8F5
:10C6F0009FE00E9482981092420C1092410C80E0C0
:10C7000090E00E94270A40914502509146026091B4
:10C7100047027091480223E0CE0109960E943A9B9D
:10C7200063EE79E0CE0101960E94189ABE01675F20
:10C730007F4FCE0101960E943F9C62EF75E00E9400
:10C74000509C12C46CEE79E0CE0109960E94189AB2
:10C75000BE01675F7F4F88ED9CE00E94CE9C8111F7
:10C7600016C061EF79E0CE0101960E94189ABE01D1
:10C770006F5F7F4F88ED9CE00E94CE9C01E08111AD
:10C7800001C000E0CE0101960E94AD9901C001E018
:10C79000CE0109960E94AD99002309F49FC08091B3
:10C7A000DC0C9091DD0C069708F145E050E068ED57
:10C7B0007CE0CE0101960E94F109BE016F5F7F4FC0
:10C7C0008AEB9CE00E949F9ACE0101960E94AD994F
:10C7D0008AEB9CE00E94189E0E94E1A060933D02BB
:10C7E00070933E0280933F02909340028091BE047A
:10C7F0009091BF040E94A82D20E030E048E051E471
:10C800000E94FF9E60934102709342028093430214
:10C81000909344026093B30B7093B40B8093B50B69
:10C820009093B60B80913D0290913E02A0913F0201
:10C83000B09140028093BB0B9093BC0BA093BD0BB7
:10C84000B093BE0B8091AF0C882381F161EA7CE04C
:10C850008EE89FE00E942D9620913D0230913E028D
:10C8600040913F025091400260E070E080E291E42C
:10C870000E94C2A1AB01BC0121E030E08EE89FE044
:10C880000E9481986CED79E08EE89FE00E945E96B0
:10C8900040914102509142026091430270914402E2
:10C8A00022E030E08EE89FE00E9482981092420CD5
:10C8B0001092410C80E090E00E94270A40914102D2
:10C8C00050914202609143027091440223E0CE01F4
:10C8D00009960E943A9B66EF79E024CF6FEF79E0EA
:10C8E000CE0109960E94189ABE01675F7F4F88EDBE
:10C8F0009CE00E94CE9C811116C063E07AE0CE01DC
:10C9000001960E94189ABE016F5F7F4F88ED9CE0F0
:10C910000E94CE9C01E0811101C000E0CE01019691
:10C920000E94AD9901C001E0CE0109960E94AD9927
:10C93000002309F46FC060E08091C8040E94E29077
:10C9400009E110E0C12CD12C76018091C8040E942D
:10C950006990BC01882777FD8095982F0E94CB9F16
:10C960009B01AC01C701B6010E94359E6B017C01A1
:10C970006AE070E080E090E00E94D38F01501109DE
:10C9800021F720E030E040EA50E4C701B6010E9400
:10C990005FA120E030E040E85AE30E945FA120E080
:10C9A00030E048EC51E40E94FF9E609312027093C5
:10C9B000130280931402909315026093D50B709329
:10C9C000D60B8093D70B9093D80B1092420C1092F9
:10C9D000410C80E090E00E94270A409112025091A1
:10C9E0001302609114027091150222E0CE010996A3
:10C9F0000E943A9B64E378E0CE0101960E94189A67
:10CA0000BE01675F7F4FCE0101960E943F9C63E0AD
:10CA100076E095CE67E07AE0CE0109960E94189AFA
:10CA2000BE01675F7F4F88ED9CE00E94CE9C811124
:10CA300016C06BE07AE0CE0101960E94189ABE0102
:10CA40006F5F7F4F88ED9CE00E94CE9C01E08111DA
:10CA500001C000E0CE0101960E94AD9901C001E045
:10CA6000CE0109960E94AD99002309F473C026E017
:10CA700030E044E050E068ED7CE0CE0101960E9499
:10CA80006F9DBE016F5F7F4F8AEB9CE00E949F9A73
:10CA9000CE0101960E94AD998AEB9CE00E940E9E09
:10CAA0006B017C016BE278E0CE0109960E94189A36
:10CAB000BE01675F7F4F88ED9CE00E94669DAC01E0
:10CAC0004F5F5F4F68ED7CE0CE0101960E94F10957
:10CAD000BE016F5F7F4F8AEB9CE00E949F9ACE0160
:10CAE00001960E94AD99CE0109960E94AD990091E0
:10CAF000E4041091E5048AEB9CE00E94189EAB01CF
:10CB0000BC019801C6010E943935E9E1FCE029ED3C
:10CB10003BE04191519161917191D9014D935D93A8
:10CB20006D937D939D01BCE0E134FB0791F710927A
:10CB3000420C1092410C80E090E00E94270A44E0F1
:10CB400050E068ED7CE0CE0109960E94F1096FE0AB
:10CB50007AE0FFC160E37AE0CE0109960E94189A5C
:10CB6000BE01675F7F4F88ED9CE00E94CE9C8111E3
:10CB700016C064E37AE0CE0101960E94189ABE01C5
:10CB80006F5F7F4F88ED9CE00E94CE9C01E0811199
:10CB900001C000E0CE0101960E94AD9901C001E004
:10CBA000CE0109960E94AD99002309F45AC08091E4
:10CBB000C2049091C3040E94152A609316027093D8
:10CBC000170280931802909319026093A30B70933D
:10CBD000A40B8093A50B9093A60B80E090E5A3ECAB
:10CBE000B7E480931E0290931F02A0932002B0939B
:10CBF000210280939B0B90939C0BA0939D0BB09371
:10CC00009E0B8091AF0C8823A1F063E87CE08EE856
:10CC10009FE00E942D96409116025091170260915C
:10CC200018027091190222E030E08EE89FE00E9425
:10CC300082981092420C1092410C80E090E00E9489
:10CC4000270A4091160250911702609118027091C4
:10CC5000190222E0CE0109960E943A9B68E37AE02D
:10CC600078C163E47AE0CE0109960E94189ABE0169
:10CC7000675F7F4F88ED9CE00E94CE9C811116C0BB
:10CC800067E47AE0CE0101960E94189ABE016F5FB8
:10CC90007F4F88ED9CE00E94CE9C01E0811101C095
:10CCA00000E0CE0101960E94AD9901C001E0CE01E5
:10CCB00009960E94AD99002309F48CC08091DC0C88
:10CCC0009091DD0C0497F8F044E050E068ED7CE0D2
:10CCD000CE0101960E94F109BE016F5F7F4F8AEB82
:10CCE0009CE00E949F9ACE0101960E94AD998AEB2A
:10CCF0009CE00E94189E609322027093230280930E
:10CD00002402909325028091220290912302A09107
:10CD10002402B09125028093970B9093980BA093D7
:10CD2000990BB0939A0B8091AF0C8823A1F06AE61F
:10CD30007CE08EE89FE00E942D9640912202509167
:10CD40002302609124027091250222E030E08EE8F7
:10CD50009FE00E9481988091C2049091C3040E9438
:10CD6000152A60931A0270931B0280931C02909301
:10CD70001D0260939F0B7093A00B8093A10B909367
:10CD8000A20B8091AF0C8823A1F060E67CE08EE8D6
:10CD90009FE00E942D9640911A0250911B026091D3
:10CDA0001C0270911D0222E030E08EE89FE00E949C
:10CDB00082981092420C1092410C80E090E00E9408
:10CDC000270A40911A0250911B0260911C02709137
:10CDD0001D02B8C063E57AE0CE0109960E94189A58
:10CDE000BE01675F7F4F88ED9CE00E94CE9C811161
:10CDF00016C067E57AE0CE0101960E94189ABE013E
:10CE00006F5F7F4F88ED9CE00E94CE9C01E0811116
:10CE100001C000E0CE0101960E94AD9901C001E081
:10CE2000CE0109960E94AD99002309F4B5C0809106
:10CE3000DC0C9091DD0C0497F8F044E050E068EDD4
:10CE40007CE0CE0101960E94F109BE016F5F7F4F29
:10CE50008AEB9CE00E949F9ACE0101960E94AD99B8
:10CE60008AEB9CE00E94189E60931E0270931F0242
:10CE7000809320029093210280911E0290911F02C4
:10CE8000A0912002B091210280939B0B90939C0B68
:10CE9000A0939D0BB0939E0B8091AF0C8823A1F0C3
:10CEA00067E47CE08EE89FE00E942D9640911E0290
:10CEB00050911F02609120027091210222E030E027
:10CEC0008EE89FE00E9481988091C2049091C304F3
:10CED0000E94152A6093160270931702809318021D
:10CEE000909319026093A30B7093A40B8093A50BEE
:10CEF0009093A60B8091AF0C8823A1F06DE37CE0AA
:10CF00008EE89FE00E942D964091160250911702E4
:10CF1000609118027091190222E030E08EE89FE0E3
:10CF20000E9482981092420C1092410C80E090E096
:10CF30000E94270A40911602509117026091180230
:10CF40007091190222E0CE0109960E943A9B6BE48F
:10CF50007AE0CE0101960E94189ABE01675F7F4F6A
:10CF6000CE0101960E943F9CBC0180EC9CE00E9497
:10CF7000829ACE0101960E94AD99CE0109960E9437
:10CF8000AD9960EC7CE0CE0101960E94979ACE01AB
:10CF900001960E949E110CC0112369F168ED7CE09E
:10CFA000CE0101960E94979ACE0101960E94740AC2
:10CFB000CE0101960E94AD991EC08DE49DE0E8D699
:10CFC000182F882319F16AE37BE08CEC9CE00E9427
:10CFD000B59A8091AF0C882359F067E37CE08EE826
:10CFE0009FE00E942D96612F8EE89FE00E94999607
:10CFF000812F0E9427510E94A48F6093DE0C7093B2
:10D00000DF0C8093E00C9093E10C49C08091B10C4F
:10D01000882309F44FC00E94A48FE8EECE2EE3E0EF
:10D02000DE2EE12CF12CA70196010E94A2A2CA01DA
:10D03000B9010E94C99F2091150C3091160C4091A6
:10D04000170C5091180C0E94349E20910E023091C2
:10D050000F0240911002509111020E94A0A01816D8
:10D060004CF50E94A48FA70196010E94A2A2CA01BA
:10D07000B9010E94C99F6093150C7093160C8093A0
:10D08000170C9093180C8091AB0C9091AC0C0E94F3
:10D090006F4E64E170E080E090E00E94D38F809159
:10D0A000B10C8823E9F064E670E080E090E00E9433
:10D0B000D38F16C00E94A48FC090DE0CD090DF0CDE
:10D0C000E090E00CF090E10C6C197D098E099F094D
:10D0D00068347E4E8105910510F30E948032DFCFC7
:10D0E000A6960FB6F894DEBF0FBECDBFDF91CF91ED
:10D0F0001F910F91FF90EF90DF90CF90BF90AF9076
:10D100009F908F9008950895CF92DF92EF92FF92B3
:10D11000FC0185899689481B590B61097109A3890E
:10D12000B4899A01AB010E94E6A26B017C018FE0F9
:10D13000F594E794D794C7948A95D1F76585768559
:10D14000882777FD8095982F2BE0660F771F881F23
:10D15000991F2A95D1F727853089442737FD4095B7
:10D16000542F2C0D3D1D4E1D5F1D0E94C4A22C0D81
:10D170003D1D4E1D5F1DCA01B901FF90EF90DF906C
:10D18000CF9008951F93CF93DF931F92CDB7DEB753
:10D19000162F67E770E085EC9EE049830E942A869F
:10D1A000612F85EC9EE00E94D9854981642F85EC32
:10D1B0009EE00E94D98585EC9EE00F90DF91CF9193
:10D1C0001F910C949E86CF93C62F67E770E085EC85
:10D1D0009EE00E942A866C2F85EC9EE00E94D985F5
:10D1E00085EC9EE00E949E8667E770E085EC9EE0FD
:10D1F0000E942A8641E050E067E770E085EC9EE0FF
:10D200000E949C8685EC9EE00E948A85C82F85EC52
:10D210009EE00E949E868C2FCF910895CF93DF933E
:10D22000C62F67E770E085EC9EE00E942A866C2F8F
:10D2300085EC9EE00E94D98585EC9EE00E949E864A
:10D2400067E770E085EC9EE00E942A8642E050E0AD
:10D2500067E770E085EC9EE00E949C8685EC9EE08E
:10D260000E948A85D82F80E0C82F85EC9EE00E941E
:10D270008A85C82BD92B85EC9EE00E949E86CE0124
:10D28000DF91CF910895CF93DF93EC01643008F0E4
:10D2900063E0688385EC9EE00E94178660EDCE0116
:10D2A00092DF853509F039C06AEACE01B7DF9A838B
:10D2B00089836CEACE01B2DF9C838B836EEACE0158
:10D2C000ADDF9E838D8360EBCE01A8DF9A8B898BC7
:10D2D00062EBCE01A3DF9C8B8B8B64EBCE019EDFD8
:10D2E0009E8B8D8B66EBCE0199DF98878F8368EBE1
:10D2F000CE0194DF9A8789876AEBCE018FDF9C8706
:10D300008B876CEBCE018ADF9E878D876EEBCE011B
:10D3100085DF988B8F8781E001C080E0DF91CF911E
:10D320000895CF93DF93EC014EE264EF2BDF65E0CD
:10D3300070E080E090E00E94D38F66EFCE01DF9135
:10D34000CF916CCFCF93DF93EC01EBDFAC0160E0CA
:10D3500070E0CE01D9DE685F7F4F8F4F9F4F34E082
:10D3600095958795779567953A95D1F70E94CB9FCC
:10D3700020E030E040E251E40E94FF9EDF91CF9137
:10D380000895CF92DF92EF92FF92CF93DF93EC015B
:10D3900048814295440F440F407C4C5C64EFF2DEC0
:10D3A0008881811105C065E070E080E090E012C0E6
:10D3B000813029F468E070E080E090E00BC08230BA
:10D3C00029F46EE070E080E090E004C06AE170E073
:10D3D00080E090E00E94D38F66EFCE011FDF6C01EA
:10D3E000E12CF12CFE2CED2CDC2CCC2468EFCE01B2
:10D3F000EADEA7019601282BCA01B901488128E07D
:10D4000030E0241B310904C0969587957795679580
:10D410002A95D2F7DF91CF91FF90EF90DF90CF90D8
:10D4200008952F923F924F925F926F927F928F92C8
:10D430009F92AF92BF92CF92DF92EF92FF920F93A3
:10D440001F93CF93DF93CDB7DEB72A970FB6F8942B
:10D45000DEBF0FBECDBF9A87898763DF8C018985C8
:10D460009A858FDF6D837E838F839887A80160E024
:10D4700070E089859A8548DE4B015C0180EA881A54
:10D480008FE0980AA108B108A5019401C501B40173
:10D490000E946CA22B013C010CE075946794579498
:10D4A00047940A95D1F7A985BA8511962D903C909D
:10D4B00012971C9115960D90BC91A02D0E94F0A280
:10D4C0006B017C018DE0F594E794D794C7948A951D
:10D4D000D1F7E985FA85A781B085A30192010E9461
:10D4E000F0A2BB2797FDB095AB2FC80ED91EEA1E40
:10D4F000FB1EF2E0CF0ED11CE11CF11C32E0F594D2
:10D50000E794D794C7943A95D1F780E8D80EE11CF8
:10D51000F11CE985FA85A189B289A70196010E94CB
:10D52000E6A2DC01CB014FE0B695A79597958795CC
:10D530004A95D1F789839A83AB83BC836101EE243A
:10D54000D7FCE094FE2C52E0CC0CDD1CEE1CFF1C42
:10D550005A95D1F7A185B285A30192010E94F0A24C
:10D560002B013C016BE075946794579447946A953E
:10D57000D1F7A381B481A50194010E94F0A2EBE050
:10D580009595879577956795EA95D1F7460E571E3D
:10D59000681E791EC40CD51CE61CF71C012E04C0A5
:10D5A000CC0CDD1CEE1CFF1C0A94D2F792E0C90ED5
:10D5B000D11CE11CF11CC701B60124E030E040E0C1
:10D5C00050E00E94C4A28D819E81AF81B885821BEC
:10D5D000930BA40BB50B9C01AD0160E573EC80E0EF
:10D5E00090E004C096958795779567951A95D2F740
:10D5F0000E946CA297FD0DC0660F771F881F991FB0
:10D6000029813A814B815C810E94A2A249015A0181
:10D610000CC029813A814B815C810E94A2A2490100
:10D620005A01880C991CAA1CBB1C9927B7FC9A9517
:10D630008B2D7A2D692D9B01AC010E946CA29B0160
:10D64000AC01AEEDBBE00E94E6A26C01FF24D7FC6A
:10D65000F094EF2CA3E4B3EEA50194010E94F2A292
:10D66000BB2797FDB095AB2FC80ED91EEA1EFB1E37
:10D670009FECC90E9EE0D91EE11CF11CA4E0F594BC
:10D68000E794D794C794AA95D1F7C80CD91CEA1C83
:10D69000FB1CC701B6012A960FB6F894DEBF0FBE79
:10D6A000CDBFDF91CF911F910F91FF90EF90DF9051
:10D6B000CF90BF90AF909F908F907F906F905F9032
:10D6C0004F903F902F9008958F929F92AF92BF926C
:10D6D000CF92DF92EF92FF92CF93DF9300D01F9211
:10D6E000CDB7DEB74A015B019CDE6B017C0120E017
:10D6F0003AE24DE257E4C501B4010E94FF9E9B014E
:10D70000AC0160E070E080E89FE30E94349E26EF69
:10D7100038E248EA50E40E94C2A19B01AC01C70173
:10D72000B60129833A834B835C830E94CB9F298176
:10D730003A814B815C810E94FF9E0E94989F0F90CE
:10D740000F900F900F90DF91CF91FF90EF90DF90AF
:10D75000CF90BF90AF909F908F900895CF93DF931D
:10D7600000D01F92CDB7DEB79A01AB0129833A836F
:10D770004B835C8356DE0E94CB9F29813A814B818B
:10D780005C810E94FF9E21E03EED42E45EE30E9448
:10D79000C2A19B01AC0160E070E080E89FE30E94C1
:10D7A000349E20E03AE24DE257E40E945FA10F90E0
:10D7B0000F900F900F90DF91CF910895FC01108290
:10D7C0001482138215820895862F642F0C94E290A0
:10D7D000862F642F0C941B91862F0C9450914F929E
:10D7E0005F926F927F928F929F92AF92BF92CF92F1
:10D7F000DF92EF920F93CF93DF93EC014B013A014D
:10D8000059010296DBDF8DE69AE0998388836E01E9
:10D810008CE1C80ED11C26018CE3480E511CC601B8
:10D82000CDDF86E0C80ED11CC414D504C1F7FE01BB
:10D83000EE59FF4F718260823296B182A082329699
:10D8400000833196E08237979182808238968AE011
:10D8500090E091838083329684EF91E0918380837E
:10D860003396118210827197108211821282138274
:10D87000C459DF4F1882DF91CF910F91EF90DF9065
:10D88000CF90BF90AF909F908F907F906F905F9060
:10D890004F9008952F923F924F925F926F927F9296
:10D8A0008F929F92AF92BF92CF92DF92EF92FF92B0
:10D8B0000F931F93CF93DF93CDB7DEB728970FB6A3
:10D8C000F894DEBF0FBECDBF98878F83F12C4C013B
:10D8D00086E6880E911C0F8118850E591F4FD401C2
:10D8E0008C91F816A0F4AF81B8858D919C91F801C8
:10D8F000A081B181AF0DB11DFC012081318142E0D9
:10D900006C918F819885F9011995F394E8CF512C8A
:10D91000EF81F885E959FF4FFA83E9830F81188574
:10D920000C591F4FC12CD12C7601C3948F8198853F
:10D930008E599F4F9C838B83A981BA818C915816F5
:10D9400008F088C0A52CB12CAF81B8858D919C9131
:10D95000F801A081B181AA0DBB1DFC01208131819C
:10D9600041E06C918F819885F9011995AF81B88557
:10D970008D919C91F801A081B181AA0DBB1DFC0184
:10D980002281338140E06C918F819885F90119954E
:10D99000D701C601052C04C0880F991FAA1FBB1F01
:10D9A0000A94D2F79C011C0120943094412CD4019C
:10D9B0008C91EF81F88540815181481648F5642C9F
:10D9C000712CEB81FC81A081B181A60DB71DFA01FC
:10D9D000448155816C918F8198852D833E83FA0116
:10D9E0001995660C771C2D813E81EF81F885E60D37
:10D9F000F71D892B29F480859185822B932B04C0F8
:10DA00008085918582219321918780874394CFCF10
:10DA1000F801A081B181AA0DBB1DFA0122813381D9
:10DA200041E06C918F819885F9011995AF81B88596
:10DA30008D919C91F801A081B181AA0DBB1DFC01C3
:10DA40002081318140E06C918F819885F901199591
:10DA5000539472CF28960FB6F894DEBF0FBECDBF99
:10DA6000DF91CF911F910F91FF90EF90DF90CF90BA
:10DA7000BF90AF909F908F907F906F905F904F90EE
:10DA80003F902F900895FC0180E090E0258D368D29
:10DA90002617370739F0019636968A309105B1F787
:10DAA0008FEF9FEF0895DC0126E0629FA00DB11D6E
:10DAB000112490965C934E935F9721E091962C935E
:10DAC0009197FC01E459FF4F208131960190F0813C
:10DAD000E02D222331F0309749F0611107C0DC01BD
:10DAE00002C0309719F05C968C9119940895CF92EA
:10DAF000DF92FF920F931F93CF93DF931F92CDB7C7
:10DB0000DEB76C01F62EFC0186E0689FE00DF11D8A
:10DB1000112411A2878D90A181309105E9F01CF4A8
:10DB2000892B51F044C08230910591F1039709F09F
:10DB30003EC040E050E030C04423C9F141E050E035
:10DB4000C601B1DF0E94A48FF601E85AFF4F60833F
:10DB50007183828393832BC049830E94A48FF60133
:10DB6000E85AFF4F0081118122813381601B710BC4
:10DB7000820B930B72960081118120E030E0498185
:10DB8000061717072807390718F442E050E004C0C9
:10DB900041110DC043E050E06F2DC6010F90DF91A1
:10DBA000CF911F910F91FF90DF90CF907CCF0F907E
:10DBB000DF91CF911F910F91FF90DF90CF9008954B
:10DBC0002F923F924F925F926F927F928F929F928D
:10DBD000AF92BF92CF92DF92EF92FF920F931F937B
:10DBE000CF93DF931F92CDB7DEB71C01FC014AE053
:10DBF0008FEF9FEF278D30A1232B21F4148E968F6A
:10DC0000858F11A2415036964111F4CF712C6101DC
:10DC100026E6C20ED11C510187E6A80EB11C4101B7
:10DC2000A0E68A0E911C46E0442ED6018C9178160F
:10DC300008F053C0612C8101070D111D070D111D46
:10DC4000085F1F4FF501E0806E1408F044C0F80132
:10DC500040815181062C02C0569547950A94E2F7FF
:10DC600041707E9C70011124E60CF11CD401ED91F1
:10DC7000FC91EE0DFF1D5080B701C101498303DF08
:10DC8000498197FD02C0682F1BC0019611F54423FE
:10DC900001F180E090E060E070E0F101E80FF91F31
:10DCA000248D211110C0469EF001479EF00D1124D5
:10DCB000E20DF31D548EF68EE58E10A2178E41E014
:10DCC000C10115DF06C06F5F7F4F06966A30710590
:10DCD00021F76394B7CF7394A8CF20E030E080E0C1
:10DCE000F101E20FF31F91A1911181E02A5F3F4FF3
:10DCF0002C333105A9F70F90DF91CF911F910F9130
:10DD0000FF90EF90DF90CF90BF90AF909F908F905B
:10DD10007F906F905F904F903F902F900895CF929B
:10DD2000DF92EF92FF920F931F93CF93DF938C01BB
:10DD30000E94A48FE801C45ADF4FC880D980EA80CE
:10DD4000FB806C197D098E099F09F801E859FF4F86
:10DD5000C080D180E12CF12CC616D706E806F90662
:10DD600060F4C80197DDC8012BDF182F0E94A48F33
:10DD7000688379838A839B8301C010E0812FDF91C0
:10DD8000CF911F910F91FF90EF90DF90CF9008956A
:10DD90000F931F93CF93DF93EC018C0104591F4F16
:10DDA00081E0F8018083CE01BADF882349F089A1A0
:10DDB000882331F08F8D98A1019711F48C8D03C0C9
:10DDC000F801108280E0DF91CF911F910F910895AB
:10DDD000FC011382128281EF9AE091838083148286
:10DDE00060874187228788E083870895FF920F9399
:10DDF0001F93CF93DF938C0185EC9EE00E941786E2
:10DE000063E77AE08EE89FE00E948996C0E0D0E068
:10DE100087E2F82E6F2D85EC9EE00E94208685EC2F
:10DE20009EE00E949E8681111EC06FE77AE08EE818
:10DE30009FE00E945E9640E150E06F2D8EE89FE0EB
:10DE40000E948197F801F4826BE97AE08EE89FE006
:10DE50000E945E9640E150E06F2D8EE89FE00E94A8
:10DE6000819721960FC0843069F465EB7AE08EE8E3
:10DE70009FE00E945E9640E150E06F2D8EE89FE0AB
:10DE80000E948197F394F0E4FF12C4CFCD2B19F4D4
:10DE900060ED7AE002C066EE7AE08EE89FE0DF9106
:10DEA000CF911F910F91FF900C9489961F93CF9360
:10DEB000DF93EC01162F6C8185EC9EE00E9420869A
:10DEC000E091C50EF091C60E6B85612B0190F0813B
:10DED000E02D85EC9EE0199585EC9EE0DF91CF91D9
:10DEE0001F910C949E86FC01138660E0DFCF28E032
:10DEF000FC01238760E0DACF1F93CF93DF93EC011F
:10DF0000162F6460D3DF81E090E00E94F98F612FCB
:10DF10006B7FCE01CBDF82E390E0DF91CF911F9149
:10DF20000C94F98F1F93CF93DF93EC01162FBEDF74
:10DF3000612FCE01DF91CF911F91DECFEF92FF9243
:10DF40001F93CF93DF931F92CDB7DEB77C01162FBF
:10DF5000607F642B4983E6DF80E1189FB0011124C4
:10DF60004981642BC7010F90DF91CF911F91FF90E2
:10DF7000EF90D8CF40E0E2CF61E0FCDF80ED97E0AA
:10DF80000C94F98F62E0F6DF80ED97E00C94F98F46
:10DF9000CF93DF93CDB7DEB728970FB6F894DEBFE7
:10DFA0000FBECDBF28E0EAE0F5E0DE01119601905A
:10DFB0000D922A95E1F7FC012185241710F44FEF0B
:10DFC000420FFE013196E40FF11DE40FF11D208197
:10DFD000260F2068622F28960FB6F894DEBF0FBE7A
:10DFE000CDBFDF91CF91C6CFFC0166816B7F668389
:10DFF0006860C0CFFC016681262F246026836C6098
:10E00000B9CFCF92DF92EF92FF920F931F93CF93EE
:10E01000DF931F921F92CDB7DEB78C01677088E047
:10E02000689FB00111246064C80149835A83A2DF4C
:10E030004981C42E5A81D52EE12CF12CD6016D9147
:10E040006D01D801ED91FC910190F081E02DC801A6
:10E050001995BFEFEB1AFB0AE8E0EE16F10471F731
:10E060000F900F90DF91CF911F910F91FF90EF9044
:10E07000DF90CF90089541E061DF81E090E0089566
:10E08000CF93DF93EC0185EC9EE00E9417861D8202
:10E090008985823010F098E09D839A85992329F034
:10E0A000813019F48D8184608D8362E370E080E0BB
:10E0B00090E00E94D38F6B85CE01F8DE68EE73E0AE
:10E0C00080E090E00E94D38F60E3CE012BDF84E9F3
:10E0D00091E10E94F98F60E3CE0124DF84E991E1B0
:10E0E0000E94F98F60E3CE011DDF86E990E00E9477
:10E0F000F98F60E2CE0116DF6D816062CE013ADFFA
:10E1000084E08E83CE0176DFCE0136DF82E08F831E
:10E1100066E0CE012FDFCE01DF91CF9133CFFC013E
:10E12000608308951F93CF93DF93EC01162F6881CE
:10E1300085EC9EE00E942086612F85EC9EE00E9487
:10E14000D98560E085EC9EE00E942B8643E06881E3
:10E1500085EC9EE00E949A8685EC9EE00E948A856E
:10E16000EC0185EC9EE00E948A8520E030E0382FAB
:10E17000C9018C2B9D2BDF91CF911F910895D2DF88
:10E18000BC0180E090E00E94C99F2AE037ED43EA9D
:10E190005CE30E945FA123E333E948E853E40C9475
:10E1A000349E089567E0EBCF66E0E9CFCF92DF922F
:10E1B000EF92FF92CF93DF93EC01882777FD809554
:10E1C000982F0E94CB9F6B017C0120E030E040E45F
:10E1D0005FE30E945FA120E030E048E452E40E9447
:10E1E000FF9E0E94989FC617D707ECF020E030E012
:10E1F00040EA5FE3C701B6010E945FA120E030E082
:10E2000048E452E40E94FF9E20E030E040E85FE3F3
:10E210000E94359E0E94989F21E06C177D070CF4A8
:10E2200020E0822F01C080E090E0DF91CF91FF904D
:10E23000EF90DF90CF900895CF92DF92EF92FF9210
:10E24000CF93DF93EC016C597F4F882777FD809542
:10E25000982F0E94CB9F6B017C0120E030E040E4CE
:10E260005FE30E945FA120E030E048E452E40E94B6
:10E27000FF9E0E94989FC617D707ECF020E030E081
:10E2800040EA5FE3C701B6010E945FA120E030E0F1
:10E2900048E452E40E94FF9E20E030E040E85FE363
:10E2A0000E94359E0E94989F21E06C177D070CF418
:10E2B00020E0822F01C080E090E0DF91CF91FF90BD
:10E2C000EF90DF90CF900895CF92DF92EF92FF9280
:10E2D000CF93DF93EC0164567109882777FD809511
:10E2E000982F0E94CB9F6B017C0120E030E040E43E
:10E2F0005FE30E945FA120E030E048E452E40E9426
:10E30000FF9E0E94989FC617D707ECF020E030E0F0
:10E3100040EA5FE3C701B6010E945FA120E030E060
:10E3200048E452E40E94FF9E20E030E040E85FE3D2
:10E330000E94359E0E94989F21E06C177D070CF487
:10E3400020E0822F01C080E090E0DF91CF91FF902C
:10E35000EF90DF90CF9008951F920F920FB60F921B
:10E3600011240BB60F922F933F934F935F936F93AC
:10E370007F938F939F93AF93BF93EF93FF9380917E
:10E38000F50D0E9450912091F80D3091F90D2F5FFD
:10E390003F4F3093F90D2093F80D9091F70D95367E
:10E3A00018F096E09093F40D9091F40D9430C9F12B
:10E3B00028F4923069F09330D1F05EC0953009F4C2
:10E3C00051C0963009F058C091E09093C40E51C0EE
:10E3D000811152C02091F80D3091F90D243631058C
:10E3E00008F442C01092C40E1092F70D1CC0813088
:10E3F00009F042C0E091F70D91E09E0F9093F70D68
:10E40000F0E02091F80D3091F90DEE0FFF1FE6506E
:10E41000F24F318320831092F90D1092F80D94E0A1
:10E4200029C0811117C0E091F70D91E09E0F9093E4
:10E43000F70DF0E02091F80D3091F90DEE0FFF1F70
:10E44000E650F24F318320831092F90D1092F80DAF
:10E4500093E010C02091F80D3091F90D253631056B
:10E4600058F007C0811108C01092F90D1092F80DF4
:10E4700003C095E09093F40D9091F60D992329F047
:10E48000811102C02F9A01C02F98FF91EF91BF9187
:10E49000AF919F918F917F916F915F914F913F913C
:10E4A0002F910F900BBE0F900FBE0F901F901895DD
:10E4B0006093F50D1092F60D0895F89482E0809324
:10E4C000B0008093B10094E69093B3001092B20034
:10E4D0008093700078948093F40D1092F70D8091E2
:10E4E000F50D60E00C94E29082E08093F40D1092C0
:10E4F000F70D08958F929F92AF92BF92CF92DF92C5
:10E50000EF92FF927B01BA0180E090E00E94C99FE8
:10E510004B015C01B70180E090E00E94C99F6B0154
:10E520007C012DEC3CEC4CE45FE30E945FA19B017D
:10E53000AC01C501B4010E94FB9E87FD17C02DEC04
:10E540003CEC4CE45FE3C501B4010E945FA19B0178
:10E55000AC01C701B6010E94FB9E992787FD9095EB
:10E560008827990F881F9927019602C080E090E0C4
:10E57000FF90EF90DF90CF90BF90AF909F908F90E3
:10E5800008958F929F92AF92BF92CF92DF92EF92B7
:10E59000FF920F931F93CF93DF936C01EB01EC84F9
:10E5A000FD8486E0E816F1040CF443C0EE0CFF1C79
:10E5B00006E010E045EC842E4DE9942E4CE1A42EAB
:10E5C00041E8B42E8A859B85FC01E00FF11F408154
:10E5D0005181F8013497E80FF91F60817181C601FC
:10E5E00089DFFC01A501940163E971E080E091E01D
:10E5F0000E946CA24F01AA2497FCA094BA2C8626F4
:10E600009726A826B9260E5F1F4F0E151F05D1F6B7
:10E610008C829D82AE82BF8280E290E0998788875B
:10E620008FEF9FEF9983888361E070E080E090E056
:10E6300003C060E070E0CB01DF91CF911F910F919B
:10E64000FF90EF90DF90CF90BF90AF909F908F9012
:10E6500008950F931F93CF93DF938C01EB018AEF03
:10E660009DE09B878A878091F70D90E09D878C873E
:10E670008091C40E90E09F878E878091F40D853045
:10E6800009F051C0C8011BD3882319F081E090E044
:10E690004CC0BE01C801B0D78111F8CFBE01C8017E
:10E6A00007D78111F3CFBE01C8017ED28111EECF11
:10E6B000BE01C801CCD48111E9CFBE01C80169D522
:10E6C0008111E4CFBE01C80192D38111DFCFBE0119
:10E6D000C801E3D18111DACFBE01C8012DD181116A
:10E6E000D5CFBE01C80145D68111D0CFBE01C8012A
:10E6F0000E94977B8111CACFBE01C8011BD0811136
:10E70000C5CFBE01C801A2D08111C0CFBE01C801D2
:10E7100038DF672B682B692B09F0B8CF82E0809334
:10E72000F40D1092F70D80E090E0DF91CF911F91F2
:10E730000F910895AF92BF92CF92DF92EF92FF9226
:10E740000F931F93CF93DF93EB018091F70D8835E3
:10E7500010F480E070C0EA85FB858281938160E6D9
:10E7600072E26ADD892BA9F3EA85FB8584819581B4
:10E7700064E971E1A9DD892B61F3BEE1CB2ED12CD7
:10E780001DE1E12EF12C00E010E08091F70D90E00A
:10E790000497E816F906ACF5EA85FB85C701880FF2
:10E7A000991FE80FF91F8081918164EF71E044DDCA
:10E7B000892B79F25601AA0CBB1CEA85FB85EA0D70
:10E7C000FB1D8081918168E572E07EDD892B21F05F
:10E7D000000F111F01600DC0EA85FB85EA0DFB1DCE
:10E7E0008081918164EA76E06FDD892B49F0000F2A
:10E7F000111F82E0E80EF11C82E0C80ED11CC5CFCB
:10E80000760181E0E81AF108F594E794F986E88644
:10E810008AE2E816F1040CF49CCFC801AA2797FD00
:10E82000A095BA2F8C839D83AE83BF8389E090E04F
:10E830009983888381E0DF91CF911F910F91FF90A1
:10E84000EF90DF90CF90BF90AF900895AF92BF92BE
:10E85000CF92DF92EF92FF920F931F93CF93DF93AC
:10E86000EB018091F70D803211F080E05AC0EA850B
:10E87000FB85828193816CE271E0DEDC892BA9F358
:10E88000EA85FB85848195816EEE72E01DDD892B22
:10E8900061F306E010E0C12CD12C7601EA85FB85FE
:10E8A000E00FF11F808191816CE271E0C5DC892B62
:10E8B000E1F2580182E0A80EB11CEA85FB85EA0D61
:10E8C000FB1D8081918168E077E0FEDC892B39F0C7
:10E8D000CC0CDD1CEE1CFF1C6894C0F810C0EA854F
:10E8E000FB85EA0DFB1D808191816EEE72E0ECDC10
:10E8F000892B09F4BACFCC0CDD1CEE1CFF1C0C5F7D
:10E900001F4F0E33110551F68EE090E099878887EE
:10E91000CC82DD82EE82FF828FE090E09983888353
:10E9200081E0DF91CF911F910F91FF90EF90DF90E9
:10E93000CF90BF90AF900895AF92BF92CF92DF92E9
:10E94000EF92FF920F931F93CF93DF93EB01809190
:10E95000F70D823251F5EA85FB858281938168E566
:10E9600072E06ADC892B09F18091F70D90E081500B
:10E970009048880F991FEA85FB85E80FF91F808171
:10E98000918168E572E058DC892B79F01986188648
:10E990008FEF9FEFDC018C839D83AE83BF8386E086
:10E9A00090E09983888381E06DC0EA85FB85828150
:10E9B000938160E47FE140DC892B21F08091F70DA9
:10E9C000813210F480E05EC0EA85FB858481958108
:10E9D00060EA7FE079DC892BA9F358E0A52EB12C01
:10E9E00003E010E0C12CD12C7601EA85FB85C8013B
:10E9F000880F991FE80FF91F8081918168E572E007
:10EA00001BDC892BF9F2EA85FB85EA0DFB1D808171
:10EA1000918160E476E058DC892B39F0CC0CDD1C68
:10EA2000EE1CFF1C6894C0F810C0EA85FB85EA0D57
:10EA3000FB1D8081918166E272E046DC892B09F43E
:10EA4000C1CFCC0CDD1CEE1CFF1C0E5F1F4F84E001
:10EA5000A80EB11C0332110541F6EA85FB85EA5B7D
:10EA6000FF4F8081918168E572E0E6DB892B09F434
:10EA7000A9CF80E190E099878887CC82DD82EE8201
:10EA8000FF828DCFDF91CF911F910F91FF90EF907B
:10EA9000DF90CF90BF90AF900895AF92BF92CF928A
:10EAA000DF92EF92FF920F931F93CF93DF93EB01CF
:10EAB0008091F70D893310F480E06BC0EA85FB8507
:10EAC0008281938160E47FE1B7DB892BA9F3EA853A
:10EAD000FB858481958160EA7FE0F6DB892B61F319
:10EAE00038E0A32EB12C03E010E0C12CD12C76012C
:10EAF000EA85FB85C801880F991FE80FF91F8081FF
:10EB0000918168E572E098DB892BB1F2EA85FB859B
:10EB1000EA0DFB1D8081918160E476E0D5DB892BD5
:10EB200039F0CC0CDD1CEE1CFF1C6894C0F810C042
:10EB3000EA85FB85EA0DFB1D8081918166E272E02A
:10EB4000C3DB892B09F4B8CFCC0CDD1CEE1CFF1CF9
:10EB50000E5F1F4F84E0A80EB11C0B33110541F668
:10EB6000EA85FB85EA58FF4F8081918168E572E074
:10EB700063DB892B09F4A0CF8CE190E0998788872B
:10EB8000CC82DD82EE82FF828AE090E099838883E6
:10EB900081E0DF91CF911F910F91FF90EF90DF9077
:10EBA000CF90BF90AF9008956F927F928F929F9277
:10EBB000AF92BF92CF92DF92EF92FF920F931F938B
:10EBC000CF93DF93EB018091F70D823208F45DC0A3
:10EBD000EA85FB85828193816EE571E02DDB892BCF
:10EBE00009F453C063E0A62EB12C02E010E0C12C62
:10EBF000D12C760135018091F70D90E0A816B90669
:10EC0000CCF54801880C991CEA85FB85E80DF91DB7
:10EC1000808191816EE977E00FDB892B39F0CC0C94
:10EC2000DD1CEE1CFF1C6894C0F80FC0EA85FB8554
:10EC3000E80DF91D808191816EEE72E0FDDA892B7D
:10EC400021F1CC0CDD1CEE1CFF1CC501880F991FA7
:10EC5000EA85FB85E80FF91F808191816EE571E0FF
:10EC600033DB22E0A20EB11C892B19F00E5F1F4F7F
:10EC7000C1CF8301015011091595079519870887A0
:10EC80000031110524F41986188680E009C0CC8271
:10EC9000DD82EE82FF828CE090E09983888381E0C0
:10ECA000DF91CF911F910F91FF90EF90DF90CF9068
:10ECB000BF90AF909F908F907F906F900895AF928C
:10ECC000BF92CF92DF92EF92FF920F931F93CF9359
:10ECD000DF93EB01EA85FB858281938168E273E231
:10ECE000ABDA892B11F480E077C08091F70D843086
:10ECF00009F5EA85FB85848195816AEC78E0E4DAA0
:10ED0000892BC1F0EA85FB858681978160E372E0FB
:10ED100093DA892B79F0198618868FEF9FEFDC0143
:10ED20008C839D83AE83BF8383E090E09983888347
:10ED300081E052C08091F70D8434A8F2EA85FB850A
:10ED40008481958164E971E1BFDA892B61F206E083
:10ED500010E0C12CD12C7601EA85FB85E00FF11F74
:10ED60008081918160E372E067DA892B09F4BBCF7F
:10ED7000580182E0A80EB11CEA85FB85EA0DFB1D57
:10ED8000808191816AE976E09FDA892B39F0CC0C99
:10ED9000DD1CEE1CFF1C6894C0F810C0EA85FB85E2
:10EDA000EA0DFB1D8081918160E372E08DDA892B91
:10EDB00009F499CFCC0CDD1CEE1CFF1C0C5F1F4F1F
:10EDC0000638110549F680E290E099878887CC8261
:10EDD000DD82EE82FF82A8CFDF91CF911F910F914C
:10EDE000FF90EF90DF90CF90BF90AF9008958F92FB
:10EDF0009F92AF92BF92CF92DF92EF92FF920F93CA
:10EE00001F93CF93DF9300D01F92CDB7DEB74B0196
:10EE1000DB011A96ED91FC911B97828193816EEA3A
:10EE20007DE00ADA892B11F480E08FC0D4011A96B4
:10EE3000ED91FC911B978481958166ED76E0FCD97C
:10EE4000892B91F3E6E0EE2EF12C20E030E040E05B
:10EE500050E0A12CB12CC12CD12CD4011A96ED91EB
:10EE6000FC911B97EE0DFF1D8081918166EF71E093
:10EE700029833A834B835C83DFD9892BA9F28701ED
:10EE80000E5F1F4FD4011A96ED91FC911B97E00F76
:10EE9000F11F808191816CED74E016DA29813A814D
:10EEA0004B815C81892B39F0B501C60101E00E94DC
:10EEB000FAA221601CC0D4011A96ED91FC911B9717
:10EEC000E00FF11F8081918160E971E029833A832D
:10EED0004B835C83F9D929813A814B815C81892BF1
:10EEE00009F4A2CFB501C60101E00E94FAA25B01BC
:10EEF0006C01B4E0EB0EF11CE6ECEE16F10409F047
:10EF0000ACCFD40114962C93149715963C93159777
:10EF100016964C93169717965C931797B501C601F2
:10EF200000E20E9415A312962C93129713963C931D
:10EF3000139785E090E011969C938E9380E390E088
:10EF400019969C938E93189781E00F900F900F90D5
:10EF50000F90DF91CF911F910F91FF90EF90DF9075
:10EF6000CF90BF90AF909F908F9008958F929F9277
:10EF7000AF92BF92CF92DF92EF92FF920F931F93C7
:10EF8000CF93DF937A016901DA01CD91DC91FB0126
:10EF900084859585C817D9070CF047C0CE01880F26
:10EFA000991F0284F385E02DE80FF91FA080B1803E
:10EFB000C170DD27F1E0CF27209719F484E690E0B7
:10EFC00002C08CE99FEF4801880E991EB401C5016B
:10EFD000EDD8892B89F4800E911EB401C501E6D8C5
:10EFE000892B69F4B401600F711FC501DFD8892B2B
:10EFF000F9F023E030E005C021E030E002C022E07B
:10F0000030E0D6018D919C9111970196821793075C
:10F0100044F0F60111821082D7018D919C911197D5
:10F0200001968D939C93CE0105C081E090E002C0D3
:10F030008FEF9FEFDF91CF911F910F91FF90EF9096
:10F04000DF90CF90BF90AF909F908F9008954F9298
:10F050005F926F927F928F929F92AF92BF92CF9268
:10F06000DF92EF92FF920F931F93CF93DF9300D025
:10F070001F92CDB7DEB76C017B011C821B8281E041
:10F0800090E09A8389838091F70D8D3010F480E0B1
:10F090006BC009E713E09E012D5F3F4FAE014F5F4C
:10F0A0005F4FC60163DF892B91F79E012D5F3F4FB4
:10F0B000AE014F5F5F4FB701C60158DF019739F7C7
:10F0C0009E012D5F3F4FAE014F5F5F4FB701C601FD
:10F0D0004DDF892BE1F6412C512C3201A12CB12CB2
:10F0E0008091F70D90E029813A81281739078CF536
:10F0F00009E713E09E012D5F3F4FAE014F5F5F4F69
:10F10000B701C60133DF4C019E012D5F3F4FAE01B9
:10F110004F5F5F4FB701C60129DF21E082169104DE
:10F1200051F4892B09F0B3CF440C551C661C771C95
:10F13000689440F80AC0892809F0A9CF019709F01E
:10F14000A6CF440C551C661C771C8FEFA81AB80A72
:10F15000C7CFF701B186A086448255826682778246
:10F1600081E090E0918380830F900F900F900F903B
:10F17000DF91CF911F910F91FF90EF90DF90CF9093
:10F18000BF90AF909F908F907F906F905F904F90C7
:10F1900008952F923F924F925F926F927F928F923B
:10F1A0009F92AF92BF92CF92DF92EF92FF920F9316
:10F1B0001F93CF93DF9300D01F92CDB7DEB76C01C2
:10F1C0007B011C821B82DB011C968D919C911D97FB
:10F1D0001816190614F080E0B5C0DB011A96ED91FF
:10F1E000FC911B9782E090E09A83898382819381CE
:10F1F0006AE67AE021D8892B71F3D7011A96ED914E
:10F20000FC911B9789819A819C012F5F3F4F3A8324
:10F210002983880F991FE80FF91F8081918169E781
:10F2200073E052D8892BB9F20CEB11E09E012D5FEF
:10F230003F4FAE014F5F5F4FB701C60197DE892B8D
:10F2400051F69E012D5F3F4FAE014F5F5F4FB701FB
:10F25000C6018CDE019709F0BECF212C312C210193
:10F26000A12CB12C29813A81F70184859585281735
:10F2700039070CF05CC00CEB11E09E012D5F3F4F95
:10F28000AE014F5F5F4FB701C60170DE3C01B3E0D6
:10F29000AB16B10489F00CEB11E09E012D5F3F4FDE
:10F2A000AE014F5F5F4FB701C60160DE4C01E3E086
:10F2B000AE16B104F9F40FC00CEB11E09E012D5F06
:10F2C0003F4FAE014F5F5F4FB701C6014FDE68167B
:10F2D000790609F380CF0CEB11E09E012D5F3F4FC3
:10F2E000AE014F5F5F4FB701C60140DE8816990639
:10F2F00009F071CF6114710459F48A94892809F0D6
:10F300006ACF220C331C441C551C689420F80BC097
:10F310006A94672809F05FCF892809F05CCF220C36
:10F32000331C441C551CAFEFAA1ABA0A9BCFB186F6
:10F33000A086248235824682578282E090E09183C3
:10F34000808381E00F900F900F900F90DF91CF910D
:10F350001F910F91FF90EF90DF90CF90BF90AF90F3
:10F360009F908F907F906F905F904F903F902F90E5
:10F370000895AF92BF92CF92DF92EF92FF920F93D8
:10F380001F93CF93DF93EB01EA85FB858281938105
:10F3900068E873E10E941C71892B11F480E07DC044
:10F3A0008091F70D843019F5EA85FB85848195817C
:10F3B0006AEC78E00E946471892BC9F0EA85FB85CC
:10F3C0008681978160E372E00E941C71892B79F03D
:10F3D000198618868FEF9FEFDC018C839D83AE83A7
:10F3E000BF8387E090E09983888381E056C0809155
:10F3F000F70D843498F2EA85FB858481958168E86D
:10F4000073E10E946471892B49F206E010E0C12C7F
:10F41000D12C7601EA85FB85E00FF11F8081918177
:10F4200060E372E00E941C71892B09F4B7CF580188
:10F4300082E0A80EB11CEA85FB85EA0DFB1D8081E8
:10F44000918160E476E00E946471892B39F0CC0CE4
:10F45000DD1CEE1CFF1C6894C0F811C0EA85FB851A
:10F46000EA0DFB1D8081918160E372E00E9464716E
:10F47000892B09F493CFCC0CDD1CEE1CFF1C0C5F18
:10F480001F4F0638110531F680E290E09987888792
:10F49000CC82DD82EE82FF82A4CFDF91CF911F91DB
:10F4A0000F91FF90EF90DF90CF90BF90AF900895B5
:10F4B0008F929F92AF92BF92CF92DF92EF92FF9284
:10F4C0000F931F93CF93DF93EB018091F70D8A3158
:10F4D00008F47AC0EA85FB8580819181803293406F
:10F4E00050F4198618868FEF9FEFDC018C839D8383
:10F4F000AE83BF836FC0828193816CEA7DE00E94FE
:10F500001C71892B09F460C0EA85FB858481958193
:10F510006CEA7DE00E941C71892B09F455C054E00F
:10F52000A52EB12C03E010E0C12CD12C76018091E6
:10F53000F70D90E0A816B906E4F5EA85FB85C80149
:10F54000880F991FE80FF91F8081918166EB73E0A6
:10F550000E946471892B61F14501880C991CEA8530
:10F56000FB85E80DF91D8081918160E679E00E94BC
:10F570001C71892B39F0CC0CDD1CEE1CFF1C68942F
:10F58000C0F810C0EA85FB85E80DF91D80819181E6
:10F590006CEB72E00E941C71892BB1F0CC0CDD1C6D
:10F5A000EE1CFF1C0E5F1F4F82E0A80EB11CBFCFE8
:10F5B00085010150110915950795198708870C30A9
:10F5C000110524F41986188680E009C0CC82DD82FA
:10F5D000EE82FF828BE090E09983888381E0DF9167
:10F5E000CF911F910F91FF90EF90DF90CF90BF9040
:10F5F000AF909F908F9008958F929F92AF92BF92FD
:10F60000CF92DF92EF92FF920F931F93CF93DF93EE
:10F61000EB018091F70D8A3108F471C0EA85FB8512
:10F6200080819181843F914060F4198618868FEF24
:10F630009FEFDC018C839D83AE83BF838BE090E0E2
:10F6400066C08281938160E679E00E941C71892BFB
:10F6500009F455C073E0A72EB12C02E010E0C12CD4
:10F66000D12C76018091F70D90E0A816B906E4F54B
:10F67000EA85FB85C801880F991FE80FF91F808173
:10F68000918168E572E00E946471892B61F1450106
:10F69000880C991CEA85FB85E80DF91D8081918114
:10F6A00060EB74E00E941C71892B39F0CC0CDD1CDE
:10F6B000EE1CFF1C6894C0F810C0EA85FB85E80DBD
:10F6C000F91D8081918168E572E00E941C71892B8F
:10F6D000B1F0CC0CDD1CEE1CFF1C0E5F1F4F82E056
:10F6E000A80EB11CBFCF85010150110915950795D2
:10F6F000198708870C30110524F41986188680E0D4
:10F7000009C0CC82DD82EE82FF8284E090E09983A2
:10F71000888381E0DF91CF911F910F91FF90EF904F
:10F72000DF90CF90BF90AF909F908F900895AF9251
:10F73000BF92CF92DF92EF92FF920F931F93CF93DE
:10F74000DF93EB018091F70D863410F480E086C0E2
:10F75000EA85FB85828193816EEE72E00E941C71C6
:10F76000892BA1F3EA85FB85848195816EEE72E099
:10F770000E946471892B51F3EA85FB85868197810C
:10F7800062E27BE00E941C71892B01F3EA85FB8514
:10F790008085918562E27BE00E946471892BB1F2E1
:10F7A0005CE0A52EB12C05E010E0C12CD12C760137
:10F7B000EA85FB85C801880F991FE80FF91F808132
:10F7C00091816EEE72E00E941C71892B09F4BECF0C
:10F7D000EA85FB85EA0DFB1D8081918166E678E074
:10F7E0000E946471892B39F0CC0CDD1CEE1CFF1CCF
:10F7F0006894C0F811C0EA85FB85EA0DFB1D808185
:10F8000091816EEE72E00E946471892B09F49ECFA3
:10F81000CC0CDD1CEE1CFF1C0E5F1F4F84E0A80EFD
:10F82000B11C0534110521F6EA85FB85E657FF4F2B
:10F83000808191816EEE72E00E941C71892B09F427
:10F8400085CF80E290E099878887CC82DD82EE8246
:10F85000FF8288E090E09983888381E0DF91CF91F7
:10F860001F910F91FF90EF90DF90CF90BF90AF90DE
:10F8700008956F927F928F929F92AF92BF92CF9294
:10F88000DF92EF92FF920F931F93CF93DF931F921C
:10F89000CDB7DEB73C01B62EFC011086118612866C
:10F8A0001386148661E08B2D49830E94E29060E00C
:10F8B0008B2D0E941B914981642F70E080E090E0C5
:10F8C0000E94D38F60E08B2D0E94E29088E290E04E
:10F8D0000E94F98F00E911E08B2D0E945091892B35
:10F8E00021F401501109C1F71AC000E911E08B2D74
:10F8F0000E945091019721F401501109C1F70FC0E6
:10F9000098E2992E20E8A22E812C00E911E08B2D9F
:10F910000E945091892B31F401501109C1F78EEFEB
:10F920009FEF29C00E94B08F6B017C0100E911E0BC
:10F930008B2D0E945091019721F401501109C1F7BC
:10F94000EECF0E94B08F6C197D098E099F09693234
:10F9500071058105910530F0F301E80DF11D8085F9
:10F960008A298087A69419F4839480E8A82E9A9413
:10F9700061F680E090E00F90DF91CF911F910F91A1
:10F98000FF90EF90DF90CF90BF90AF909F908F90BF
:10F990007F906F900895AF92BF92CF92DF92EF92D7
:10F9A000FF920F931F93CF93DF93EC018D858823F4
:10F9B00009F0F89442E1CE015CDF2D85222309F0A5
:10F9C0007894009769F040E050EC69E774EC488364
:10F9D00059836A837B834C835D836E837F8358C0A6
:10F9E00018850985612F70E080E090E00E94CB9F30
:10F9F0006B017C01602F70E080E090E00E94CB9F63
:10FA00002DEC3CEC4CEC5DE30E945FA19B01AC0152
:10FA1000C701B6010E94359E688379838A839B83E0
:10FA2000BA84AB846B2D6F7770E080E090E00E9429
:10FA3000CB9F6B017C016A2D70E080E090E00E941A
:10FA4000CB9F2DEC3CEC4CEC5DE30E945FA19B0155
:10FA5000AC01C701B6010E94359EB7FC05C06C839E
:10FA60007D838E839F8307C0DC01CB01B0588C83DC
:10FA70009D83AE83BF83100F1B0D1A0D81E090E0B4
:10FA80002C85211302C080E090E091958195910929
:10FA9000DF91CF911F910F91FF90EF90DF90CF906A
:10FAA000BF90AF900895CF93DF93EC018D858823AD
:10FAB00009F0F89441E0CE01DCDE2D85222309F027
:10FAC0007894009769F040E050EC69E774EC488363
:10FAD00059836A837B834C835D836E837F8341C0BC
:10FAE000698588850E94A899BC0180E090E00E9409
:10FAF000C99F2DEC3CEC4CEC5DE30E945FA1688358
:10FB000079838A839B838A856B858F770E94A899E6
:10FB1000BC0180E090E00E94C99F2DEC3CEC4CECD5
:10FB20005DE30E945FA16C837D838E839F833A8512
:10FB300037FF07C0DC01CB01B0588C839D83AE83B7
:10FB4000BF832885230F8985280F8B85280F81E0A7
:10FB500090E03C85321302C080E090E09195819561
:10FB60009109DF91CF910895EF92FF920F931F9328
:10FB7000CF93DF937C016CE585EC9EE00E942086AC
:10FB8000E091C50EF091C60E0190F081E02D60E08D
:10FB900085EC9EE0199585EC9EE00E949E8645E0EE
:10FBA0006CE585EC9EE00E949A86C82FD0E02097F5
:10FBB00091F0C530D1058CF000E010E085EC9EE0BE
:10FBC000A9D7F701E00FF11F80870F5F1F4F0C17B8
:10FBD0001D07A4F305C085EF01C084EF9FEF01C0AE
:10FBE000CE01DF91CF911F910F91FF90EF9008957B
:10FBF000AF92BF92CF92DF92EF92FF920F931F933B
:10FC0000CF93DF93EC01B0DF97FD54C018850985D1
:10FC1000612F70E080E090E00E94CB9F6B017C013F
:10FC2000602F70E080E090E00E94CB9F2DEC3CECD8
:10FC30004CEC5DE30E945FA19B01AC01C701B601E2
:10FC40000E94359E688379838A839B83BA84AB84C0
:10FC50006B2D6F7770E080E090E00E94CB9F6B018E
:10FC60007C016A2D70E080E090E00E94CB9F2DEC3B
:10FC70003CEC4CEC5DE30E945FA19B01AC01C70131
:10FC8000B6010E94359EB7FC05C06C837D838E83D0
:10FC90009F8307C0DC01CB01B0588C839D83AE836A
:10FCA000BF83100F1B0D1A0D8C85811711F086EF85
:10FCB00001C080E0DF91CF911F910F91FF90EF90F5
:10FCC000DF90CF90BF90AF900895FB01618182815A
:10FCD00070E0762F6627680F711D882777FD809565
:10FCE000982F0E94CB9F20E030E040E85DE30E9427
:10FCF0005FA123E333E948E853E40C94349E08956C
:10FD000021E06227FC0180810C941B91CF93DF934B
:10FD1000EC01862F688349832A8361E00E94E29088
:10FD200061E088810E941B9160E089810E94E290DD
:10FD300060E08A810E94E29061E089810E941B91CB
:10FD400061E08A810E941B9160E0CE01DF91CF913A
:10FD5000D7CFFB0181819081890F9281890F938197
:10FD6000981304C081E094819D3009F080E00895EB
:10FD70002F923F924F925F926F927F928F929F92BB
:10FD8000AF92BF92CF92DF92EF92FF920F931F93A9
:10FD9000CF93DF9300D000D0CDB7DEB78C013B010D
:10FDA0004E830E94A48F1B012C0180ED280E87E05A
:10FDB000381E411C511C61E0C801A2DFFE013196D2
:10FDC0006F014E01F6E08F0E911CF60185E0119255
:10FDD0008A95E9F7760127E0A22EB12CF8018181FE
:10FDE0000E945091019739F40E94A48F6215730507
:10FDF0008405950598F3F80181810E945091892B23
:10FE000039F40E94A48F621573058405950598F353
:10FE1000F80182810E945091892B59F0F7012081CD
:10FE200081E090E00A2C01C0880F0A94EAF7282BA1
:10FE30002083F1E0AF1AB10888F69FEFE91AF90ABA
:10FE4000E814F90441F60E94A48F62157305840535
:10FE5000950540F060E0C80153DF20E030E040EC61
:10FE60005FE72EC08981EE818E13AFCFB601C80146
:10FE700070DF882309F4A9CF60E0C80141DFB60133
:10FE8000C80123DFFB01DC016A946728B9F420E094
:10FE900030E040E151E4BF01CD010E945FA120E0CC
:10FEA00030E040EA50E40E94FF9E20E030E040E075
:10FEB00052E40E94359E9B01AC0102C09F01AD013E
:10FEC000B901CA0126960FB6F894DEBF0FBECDBFAA
:10FED000DF91CF911F910F91FF90EF90DF90CF9026
:10FEE000BF90AF909F908F907F906F905F904F905A
:10FEF0003F902F90089546E63BCF4CE439CFFB016D
:10FF00008081883251F028F4803139F0823239F41E
:10FF100004C08B3311F0823411F481E0089580E045
:10FF20000895FC017783668314821582108289E02C
:10FF3000818381E0828383830895CF93DF93EC01F3
:10FF4000F0DF1B8A1A8ADF91CF910895FC01858129
:10FF50000895CF93DF93EB0167E0CE010E94448FB9
:10FF600091E02F81821390E0892FDF91CF91089546
:10FF7000EF92FF920F931F93CF93DF93EC018B01CE
:10FF8000E42E8E819F810E94798EF12C41E0B80190
:10FF90008E819F810E94AC8E882351F0FE1005C097
:10FFA000B801CE01D6DF811104C0F394EF1470F7CD
:10FFB00080E0DF91CF911F910F91FF90EF90089516
:10FFC000CF92DF92EF92FF920F931F93CF93DF9325
:10FFD0001F921F92CDB7DEB76C01F42EE52EFC0107
:10FFE0008681978169837A830E94618D69817A8194
:10FFF000882311F1F601868197810E94508E40E09E
:020000021000EC
:100000006EEBF601868197810E94F48D0F2D1E2DD7
:1000100089E0F82EF601868197810E94358EF801DD
:1000200081938F01FA94B1F7F601868197810E943E
:10003000618D91E0813009F090E0892F0F900F9051
:10004000DF91CF911F910F91FF90EF90DF90CF90B4
:100050000895CF93DF93EA01B3DF882351F068E07E
:10006000CE010E94448F91E02885821390E0892F71
:1000700001C080E0DF91CF910895EF92FF920F933E
:100080001F93CF93DF93EC018B017A018E819F81C7
:100090000E94618DB8018E819F810E94508E40E048
:1000A0006EE48E819F810E94F48D40E0F7016281B1
:1000B0008E819F810E94F48D40E0F70163818E81E3
:1000C0009F810E94F48DF8018081803139F040E0F9
:1000D000F70164818E819F810E94F48D8E819F81C2
:1000E0000E94618DB8018E819F810E94508E48814F
:1000F00068E48E819F810E94F48D64E170E080E06D
:1001000090E00E94D38F8881882331F06AE070E00C
:1001100080E090E00E94D38F8E819F81DF91CF910C
:100120001F910F91FF90EF900C94618DEF92FF92D1
:100130001F93CF93DF931F921F92CDB7DEB77C0141
:10014000FC018681978169837A830E94618D698130
:100150007A81F701868197810E94508E40E064EB9E
:10016000F701868197810E94F48DF701868197813E
:100170000E94CC8D182FF701868197810E94618D96
:1001800081E0111180E00F900F90DF91CF911F91CE
:10019000FF90EF900895CF93DF93CDB7DEB7299707
:1001A0000FB6F894DEBF0FBECDBFFB01208120311A
:1001B000C9F0AE014F5F5F4F4CDF882379F08D812E
:1001C0008F3351F020F48F3149F489E00CC08F3522
:1001D00039F08F3739F002C08AE005C080E003C0F3
:1001E0008BE001C08CE029960FB6F894DEBF0FBEFD
:1001F000CDBFDF91CF910895FF920F931F93CF93BF
:10020000DF93CDB7DEB728970FB6F894DEBF0FBEE9
:10021000CDBF8C01FC01868197810E94798EF80107
:100220001482158241E0BE016F5F7F4FF801868125
:1002300097810E94AC8E8823C1F1BE016F5F7F4F12
:10024000C80187DE882371F3F8018081811107C01E
:10025000BE016F5F7F4FC80169DF811122C0F801C5
:10026000F180BE016F5F7F4FC80195DF8F1518F4D5
:10027000F801818105C0BE016F5F7F4FC8018BDF30
:10028000F801818384818F5F8483BE016F5F7F4F1C
:10029000C80135DE882331F2F80185818F5F8583BF
:1002A000C1CF81E0F8018083DACF28960FB6F894A9
:1002B000DEBF0FBECDBFDF91CF911F910F91FF9099
:1002C0000895DF92EF92FF920F931F93CF93DF93E6
:1002D000CDB7DEB762970FB6F894DEBF0FBECDBFC5
:1002E0008C017B01D22E493028F0342F4D3018F08C
:1002F0003CE001C039E0B701C8013A8B4CDF3A89D4
:10030000831709F458C0AE014F5F5F4FB701C801B2
:100310003A8B9FDE3A89882309F44FC0F701808128
:10032000803109F448C03B3041F03C3021F03A3094
:1003300031F48FE305C08FE703C08FE501C08FE183
:100340008D83AE014F5F5F4FB701C8013A8B95DED9
:10035000F80191813A89832F391708F4892FF80120
:100360008183D11028C0381730F53183E12CF12C6E
:10037000F801848190E0E816F906ECF44E2DBE01F8
:10038000665F7F4FC801F4DDF801D180BE01665F72
:100390007F4FC80100DF8D1518F4F801818105C079
:1003A000BE01665F7F4FC801F6DEF8018183FFEF73
:1003B000EF1AFF0ADDCF81E001C080E062960FB640
:1003C000F894DEBF0FBECDBFDF91CF911F910F918B
:1003D000FF90EF90DF900895EF92FF920F931F939D
:1003E000CF93DF93CDB7DEB728970FB6F894DEBF73
:1003F0000FBECDBF8C01693020F06D3018F06CE07D
:1004000001C069E0F8016183E12CF12CF8018481DD
:1004100090E0E816F90694F44E2DBE016F5F7F4F11
:10042000C801A6DD21E0F8014181BE016F5F7F4F69
:10043000C80147DFFFEFEF1AFF0AE8CF28960FB693
:10044000F894DEBF0FBECDBFDF91CF911F910F910A
:10045000FF90EF900895FC01868197810E94CC8DDA
:1004600091E0813009F090E0892F08958F929F925A
:10047000AF92BF92CF92DF92EF92FF920F931F93B2
:10048000CF93DF93EC016950633048F4E62FF0E03E
:10049000EE0FFF1FEB50F54F0081118102C00EEEF1
:1004A00012E08B818823E1F08881811119C00E94BC
:1004B000A48F6B017C014801AA2497FCA094BA2C5C
:1004C000CE01C9DF81111FC00E94A48F681979096C
:1004D0008A099B096C157D058E059F05A0F4F0CF58
:1004E000B801882777FD8095982FDF91CF911F91D4
:1004F0000F91FF90EF90DF90CF90BF90AF909F90C3
:100500008F900C94D38FDF91CF911F910F91FF901B
:10051000EF90DF90CF90BF90AF909F908F90089515
:10052000CF93DF93EC018E819F810E94618D8E813C
:100530009F810E94768E488164E48E819F810E9413
:10054000F48D8A81882329F06981CE01DF91CF91D2
:100550008DCFDF91CF910895FA01208148E0249F4B
:1005600090011124818190E0982F8827990F990F8D
:10057000990F282B392BDB018C918031C1F46781D5
:1005800070E08681AB01481B5109CA019695982FEE
:100590008827979587950E948FA260517109207FC7
:1005A00053E0220F331F5A95E1F7260F371FC90179
:1005B0000895EF92FF920F931F93CF93DF93CDB7E0
:1005C000DEB729970FB6F894DEBF0FBECDBF8C0102
:1005D0007B01AE014F5F5F4F3CDD882339F0AE01F8
:1005E0004F5F5F4FB701C801B7DF02C080E894EEEC
:1005F00029960FB6F894DEBF0FBECDBFDF91CF9125
:100600001F910F91FF90EF900895813824EE92078B
:100610006CF0BC01882777FD8095982F0E94CB9FB6
:1006200020E030E040E05CE30C945FA160E070E02B
:100630008EEF92EC0895BDDFE8CF0F931F93CF9319
:10064000DF93CDB7DEB728970FB6F894DEBF0FBEA5
:10065000CDBF8C01462FBE016F5F7F4F89DC8823A1
:1006600031F0BE016F5F7F4FC801E5DF04C060E07D
:1006700070E08EEF92EC28960FB6F894DEBF0FBEB6
:10068000CDBFDF91CF911F910F9108952FE53AE0F3
:10069000FC013183208308952FE53AE0FC0131838A
:1006A00020830C94329E0F931F93CF93DF938C0182
:1006B000EB0188E2FB0111928A95E9F74BE050E0EB
:1006C0006BEF7AE0CE010E94D7A51B8641E050E097
:1006D00060E070E04C875D876E877F87F801458911
:1006E00056896789708D488B598B6A8B7B8B42E06A
:1006F00050E060E070E04C8B5D8B6E8B7F8B1CA2BA
:100700001DA21EA21FA240E050E068E474E4488FDE
:10071000598F6A8F7B8F40E050E068E474EC4C8F17
:100720005D8F6E8F7F8F4DEC5CEC6CE47EE348A3B5
:1007300059A36AA37BA3DF91CF911F910F910895D5
:1007400027E03BE0FC0131832083458B568B678B90
:10075000708F0895CF93DF931F921F92CDB7DEB7AE
:1007600085EC9EE02A8349836BD24981642F85EC16
:100770009EE01FD22A81622F85EC9EE01AD285EC82
:100780009EE00F900F90DF91CF91D8C20F931F93EF
:10079000CF93DF938C01EB01262F41E06EE1DADF8E
:1007A000F801D483C383C038D10509F45BC0DCF4FD
:1007B000C034D105A9F1C036D10509F442C0A097D3
:1007C00009F08AC080E090E8A9E8B4E480930505C8
:1007D00090930605A0930705B093080580E090E08C
:1007E000A5E7B4E471C0C03CD10509F44CC0C03EDB
:1007F000D10509F459C0C03AD10509F06DC080E0B7
:1008000090E0A8ECB3E48093050590930605A093CF
:100810000705B093080580E090E0AFE7B3E454C06B
:1008200080E090ECA5E5B4E480930505909306057F
:10083000A0930705B093080580E090E0AEE3B4E430
:1008400043C080E090E8A7E2B4E48093050590936C
:100850000605A0930705B093080580E090E0A6E1A7
:10086000B4E432C080E090E0A1EEB3E480930505EB
:1008700090930605A0930705B093080580E090E0EB
:10088000A8ECB3E421C080E090E0A5EAB3E4809353
:10089000050590930605A0930705B093080580E031
:1008A00090E8A3E9B3E410C080E090E0A6E6B3E4EA
:1008B0008093050590930605A0930705B09308055E
:1008C00080E090E0ADE4B3E48093010590930205ED
:1008D000A0930305B0930405DF91CF911F910F9171
:1008E0000895CF93DF93EC0185EC9EE0A0D120E04A
:1008F00042E06EE1CE012EDF60E270E0CE0146DF25
:1009000081E0DF91CF9108956F927F928F929F92B5
:10091000AF92BF92CF92DF92EF92FF920F931F930D
:10092000CF93DF93EC016EE185EC9EE089D1E091FD
:10093000C50EF091C60E0190F081E02D63E085ECCC
:100940009EE0199585EC9EE0F9D146E06EE185ECDC
:100950009EE0F0D185EC9EE0D5D00697DCF385ECE7
:100960009EE0D8D0682E85EC9EE0D4D0782E85EC21
:100970009EE0D0D0C82E85EC9EE0CCD0D82E85EC61
:100980009EE0C8D0882E85EC9EE0C4D0982EB62C70
:10099000A12CA728B501882777FD8095982F0E9464
:1009A000CB9F6D837E838F839887F82CE12CE92879
:1009B000B701882777FD8095982F0E94CB9F698784
:1009C0007A878B879C871C2D00E00D29B80188272A
:1009D00077FD8095982F0E94CB9F6D877E878F87AC
:1009E000988B198A1A8A1B8A1C8ADF91CF911F91D2
:1009F0000F91FF90EF90DF90CF90BF90AF909F90BE
:100A00008F907F906F900895CF92DF92EF92FF9238
:100A10000F931F93CF93DF938C01EB0184E2FB01D3
:100A200011928A95E9F7C8016FDF84E290E0A0E0B7
:100A3000B0E088839983AA83BB83F801858996896E
:100A4000A789B08D8C839D83AE83BF8382E090E0C5
:100A5000A0E0B0E088879987AA87BB87188A198A9F
:100A60001A8A1B8AC0900505D0900605E0900705FC
:100A7000F0900805A70196016581768187819085B0
:100A80000E94FF9E20E030E048EC52E40E945FA10B
:100A90006C8B7D8B8E8B9F8BA7019601F8016185F6
:100AA0007285838594850E94FF9E20E030E048ECAB
:100AB00052E40E945FA1688F798F8A8F9B8F20916B
:100AC0000105309102054091030550910405F8019C
:100AD00065857685878590890E94FF9E20E030E0BD
:100AE00048EC52E40E945FA16C8F7D8F8E8F9F8FA8
:100AF00081E0DF91CF911F910F91FF90EF90DF90F8
:100B0000CF9008958091F50E90E02091F60E821B13
:100B1000910908952091F60E8091F50E281750F452
:100B2000E22FF0E0E950F14F808190E02F5F2093B9
:100B3000F60E08958FEF9FEF0895E091F60E8091E5
:100B4000F50EE81730F4F0E0E950F14F808190E0C5
:100B500008958FEF9FEF08950895CF92DF92EF925F
:100B6000FF920F931F93CF93DF937C01CB018A01F8
:100B70002091D10E222389F0EB016B01C40ED51E0A
:100B8000CC15DD0561F06991D701ED91FC910190E3
:100B9000F081E02DC7011995F3CF642F91D1C801E1
:100BA000DF91CF911F910F91FF90EF90DF90CF9049
:100BB0000895CF93DF931F92CDB7DEB7698320915D
:100BC000D10E2223D1F02091D20E203240F021E02C
:100BD00030E0FC013383228380E090E014C08091F8
:100BE000D30EE82FF0E0EC52F14F998190838F5FA4
:100BF0008093D30E8093D20E04C061E0CE010196A3
:100C00005FD181E090E00F90DF91CF910895FC01DA
:100C10001382128248EE53E060E070E04483558313
:100C20006683778385E19BE09183808308951092AA
:100C3000F60E1092F50E1092D30E1092D20E83C0C3
:100C400081E08093D10E6093F40E1092D30E109237
:100C5000D20E0895F5CF0F93062F21E04091D20ECA
:100C600064ED7EE08091F40ED4D01092D30E1092F9
:100C7000D20E1092D10E0F9108958F929F92AF9243
:100C8000BF92CF92DF92EF92FF920F931F93CF9379
:100C9000DF93EC01F62ED42E48015901EE2009F124
:100CA000CFDF1E2D143008F013E01150B8F0E881AA
:100CB000F98128E0129FB0011124A501940104C01C
:100CC00056954795379527956A95D2F7CA01B90188
:100CD0000190F081E02DCE011995E7CF60E0CE01C3
:100CE000BADF4D2D413208F040E22C2D67EF7EE057
:100CF0008F2D47D01092F60E8093F50EDF91CF9195
:100D00001F910F91FF90EF90DF90CF90BF90AF9029
:100D10009F908F900895CF92EF920F931F93C22EC2
:100D2000E12C00E010E09801A8DF1F910F91EF90F7
:100D3000CF90089521E0EFCF21E0EDCF61E08BCFA0
:100D400085EC9EE064CF1092840F81E08093820F47
:100D50001092810F61E084E10E941B9161E085E1C6
:100D60000E941B91E9EBF0E080818E7F808380817F
:100D70008D7F808388E48093B80085E48093BC00F5
:100D80000895413208F043C09091840F9111FCCF37
:100D900091E09093840F2093820F2FEF2093170FF1
:100DA00010925C0F240F20935B0F9093830F909110
:100DB000830F880F892B8093830F8091810F81305F
:100DC00061F41092810F8091830F8093BB0080911A
:100DD000BC0083FDF8CF85EC01C085EE8093BC009C
:100DE0008091840F8130E1F380915C0F841710F4BF
:100DF00040915C0F2DE53FE0FB01D9018A2F821B5A
:100E0000841718F48D918193F9CF842F089580E091
:100E100008950F93413208F04AC09091840F9111C8
:100E2000FCCF92E09093840F0093820F9FEF9093FA
:100E3000170F10925C0F40935B0FFB016DE57FE095
:100E4000DB019A2F961B941718F491919D93F9CF7B
:100E50001092830F9091830F880F892B8093830FBB
:100E60008091810F813061F41092810F8091830F06
:100E70008093BB008091BC0083FDF8CF85EC01C05E
:100E800085EE8093BC00222321F08091840F823074
:100E9000E1F38091170F8F3F61F08091170F80323F
:100EA00051F08091170F803341F483E007C081E057
:100EB00005C080E003C082E001C084E00F91089586
:100EC000613298F42091840F243089F46093390FB3
:100ED000FC018BE39FE0DC012A2F281B261718F466
:100EE00021912D93F9CF80E0089581E0089582E06B
:100EF000089585ED8093BC008091BC0084FDFCCFFB
:100F00001092840F089585EC8093BC001092840F9A
:100F100008951F920F920FB60F9211240BB60F92E5
:100F20002F933F934F935F936F937F938F939F93F1
:100F3000AF93BF93EF93FF938091B900887F803682
:100F400009F49DC070F5883209F45CC090F48031DA
:100F500009F455C038F4882309F4F3C0883009F443
:100F60004EC0F2C0883109F44DC0803209F45EC031
:100F7000EBC0803409F469C050F4803309F456C0E2
:100F8000883309F0E1C08093170FBDDFDDC08035E5
:100F900009F44FC0883509F45DC0883409F0D4C025
:100FA000D2C0883909F4C3C0A8F4883709F467C0EF
:100FB00038F4883609F463C0803709F460C0C4C0CF
:100FC000883809F4B4C0803909F45FC0803809F06A
:100FD000BBC05BC0803B09F482C038F4803A09F49E
:100FE00066C0883A09F47BC0AFC0803C09F4A3C056
:100FF000883C09F4A0C0883B09F486C0A5C0809154
:10100000830F10C090915C0F80915B0F981770F563
:10101000E0915C0F81E08E0F80935C0FF0E0E35A6B
:10102000F04F80818093BB0085EC82C08093170FC6
:101030008AC0E0915C0F81E08E0F80935C0F8091FD
:10104000BB00F0E0E35AF04F808390915C0F8091F9
:101050005B0F6AC0E0915C0F81E08E0F80935C0FA4
:101060008091BB00F0E0E35AF04F80838091820FC3
:10107000811169C081E08093810F84EA5DC083E0C3
:101080008093840F1092180FCFCF8091180F803269
:1010900008F04DC0E091180F81E08E0F8093180F7B
:1010A0008091BB00F0E0E75EF04F8083BDCF2BDF87
:1010B0008091180F803230F4E091180FF0E0E75E75
:1010C000F04F10826091180F70E0E0917D0FF09169
:1010D0007E0F89E19FE019951092180F35C084E0CA
:1010E0008093840F10923A0F1092390FE0917F0F86
:1010F000F091800F19958091390F811105C081E021
:101100008093390F10923B0FE0913A0F81E08E0FE0
:1011100080933A0FF0E0E55CF04F80818093BB0054
:1011200090913A0F8091390F981708F47DCF85E898
:101130008093BC0009C085EC8093BC001092840FA2
:1011400003C01092170FD5DEFF91EF91BF91AF91C1
:101150009F918F917F916F915F914F913F912F91CF
:101160000F900BBE0F900FBE0F901F901895FC01B3
:1011700081E08083118243EC5BEA66E77BE3428394
:1011800053836483758348ED5BE666E77BE34683C0
:1011900057836087718742EF54EE64E67BE34287B2
:1011A0005387648775870895FC01DB014D915D913C
:1011B0006D917C9113974283538364837583149656
:1011C0004D915D916D917C91179746835783608710
:1011D000718718964D915D916D917C911B97428717
:1011E0005387648775870895CF93DF93FC01EB01E4
:1011F0004281538164817581488359836A837B83EB
:1012000046815781608571854C835D836E837F83C2
:1012100082859385A485B58588879987AA87BB87AA
:10122000DF91CF9108950F931F93CF93DF93082FF2
:101230006BEF76E08EE89FE00E945E96C7E0D0E01C
:1012400010E0B8010C2E02C0759567950A94E2F77C
:101250006170772742E050E08EE89FE00E94489757
:10126000219778F7DF91CF911F910F9108951F93E8
:10127000CF93DF931F92CDB7DEB7162F63E570E0F3
:1012800085EC9EE04983E6DC612F85EC9EE091DCF5
:101290004981642F85EC9EE08CDC85EC9EE00F900C
:1012A000DF91CF911F914ACDCF93DF93EC0185EC75
:1012B0009EE0BDDC40E06DE2CE01D9DF40E16DE2B1
:1012C000CE01D5DF48E06DE2CE01DF91CF91CFCFE7
:1012D0006F3F710534F4AB0177FF05C040E050E08B
:1012E00002C04FEF50E06DE1C2CFEF92FF921F932B
:1012F000CF93DF931F92CDB7DEB77C01142F462F1B
:101300006EE12983B4DF412F6FE1C701B0DF29818E
:10131000422F60E2C7010F90DF91CF911F91FF90A4
:10132000EF90A5CF6F3F710534F4AB0177FF05C097
:1013300040E050E002C04FEF50E061E298CF462F0E
:1013400062E295CF6F3F710534F4AB0177FF05C0C2
:1013500040E050E002C04FEF50E063E288CF6F3FC3
:10136000710534F4AB0177FF05C040E050E002C0E6
:101370004FEF50E064E27BCF6F3F710534F4AB0177
:1013800077FF05C040E050E002C04FEF50E065E25B
:101390006ECF6F3F710534F4AB0177FF05C040E0BD
:1013A00050E002C04FEF50E066E261CF6F3F710541
:1013B00034F4AB0177FF05C040E050E002C04FEFCE
:1013C00050E068E254CF6F3F710534F4AB0177FF12
:1013D00005C040E050E002C04FEF50E069E247CF67
:1013E000AF92BF92CF92DF92EF92FF920F931F9333
:1013F000CF93DF938C01C62F7A01690163E570E01A
:1014000085EC9EE027DC6C2F85EC9EE0D2DB85EC42
:101410009EE094DC63E570E085EC9EE01BDCA701B8
:1014200063E570E085EC9EE087DCE6015E01AC18C8
:10143000BD0885EC9EE066DB892B29F085EC9EE0FB
:1014400069DB8993F3CFAE14BF0421F0F801108259
:1014500081E0818385EC9EE0DF91CF911F910F9118
:10146000FF90EF90DF90CF90BF90AF9067CCCF927E
:10147000DF92EF92FF920F931F93CF93DF93EC01D4
:101480006B017A0189019C01225F3F4F46E050E0E9
:1014900062E3A6DF8F8590E0982F88272E85822B28
:1014A000F60191838083898990E0982F8827288985
:1014B000822BF701918380838B8990E0982F882776
:1014C0002A89822BF80191838083DF91CF911F912C
:1014D0000F91FF90EF90DF90CF9008959B012C5FCC
:1014E0003F4FAB014E5F5F4FC2CFAF92BF92CF92E3
:1014F000DF92EF92FF920F931F93CF93DF9300D071
:1015000000D0CDB7DEB77C015B01BE016F5F7F4FBE
:10151000E5DFCE0101966C01870175015E0197E060
:10152000A90EB11CF601619171916F01882777FDB9
:101530008095982F0E94CB9FF801228133814481AE
:1015400055810E945FA1F7016193719381939193FB
:101550007F010C5F1F4FCA14DB0421F726960FB6DC
:10156000F894DEBF0FBECDBFDF91CF911F910F91D9
:10157000FF90EF90DF90CF90BF90AF900895CF9302
:10158000DF931F92CDB7DEB79E012F5F3F4F41E043
:1015900050E06DE125DF898190E00F90DF91CF91E0
:1015A0000895AF92BF92CF92DF92EF92FF920F9386
:1015B0001F93CF93DF931F92CDB7DEB78C015B01F2
:1015C0006A0179019E012F5F3F4F41E050E06EE1DB
:1015D00007DF898190E0F501918380839E012F5F71
:1015E0003F4F41E050E06FE1C801FADE898190E0B1
:1015F000F601918380839E012F5F3F4F41E050E0D1
:1016000060E2C801EDDE898190E0F701918380837B
:101610000F90DF91CF911F910F91FF90EF90DF908E
:10162000CF90BF90AF900895CF93DF931F92CDB727
:10163000DEB79E012F5F3F4F41E050E061E2D0DE18
:10164000898190E00F90DF91CF910895CF93DF9340
:101650001F92CDB7DEB79E012F5F3F4F41E050E0B4
:1016600062E2BEDE898190E00F90DF91CF91089514
:10167000CF93DF931F92CDB7DEB79E012F5F3F4F11
:1016800041E050E063E2ACDE898190E00F90DF91B1
:10169000CF910895CF93DF931F92CDB7DEB79E0110
:1016A0002F5F3F4F41E050E064E29ADE898190E095
:1016B0000F90DF91CF910895CF93DF931F92CDB715
:1016C000DEB79E012F5F3F4F41E050E065E288DECC
:1016D000898190E00F90DF91CF910895CF93DF93B0
:1016E0001F92CDB7DEB79E012F5F3F4F41E050E024
:1016F00066E276DE898190E00F90DF91CF910895C8
:10170000CF93DF931F92CDB7DEB79E012F5F3F4F80
:1017100041E050E068E264DE898190E00F90DF9163
:10172000CF910895CF93DF931F92CDB7DEB79E017F
:101730002F5F3F4F41E050E069E252DE898190E047
:101740000F90DF91CF910895CF93DF931F92CDB784
:10175000DEB79E012F5F3F4F41E050E06CE240DE7C
:1017600069816F7070E066507109882777FD8095F8
:10177000982F0E94CB9F9B01AC0160E070E080E05D
:1017800090E40E94C2A120E030E048EC50E40E94C6
:101790005FA10F90DF91CF910895EF92FF920F9389
:1017A0001F93CF93DF931F92CDB7DEB78C01CB0190
:1017B000BA0120E030E048EC50E40E94FF9E0E9415
:1017C000989FE12CF12C759567956115710521F0B5
:1017D0008FEFE81AF80AF7CF8AE0E816F10484F4EC
:1017E0009E012F5F3F4F41E050E06CE2C801F8DD01
:1017F00046E04E0D8981807F482B6CE2C80137DDC1
:101800000F90DF91CF911F910F91FF90EF9008956E
:10181000CF93DF931F92CDB7DEB79E012F5F3F4F6F
:1018200041E050E060E3DCDD89810F90DF91CF91F2
:101830000895DF92EF92FF920F931F93CF93DF9360
:101840001F92CDB7DEB78C01F62EE42ED22E9E016C
:101850002F5F3F4F41E050E0C3DD898121E030E060
:101860000E2C01C0220F0A94EAF7DD2011F0282B7C
:1018700002C020952823298349816F2DC801F7DCF8
:101880000F90DF91CF911F910F91FF90EF90DF901C
:101890000895262F47E050E061E3CBCF262F46E0A6
:1018A00050E067E2C6CF262F45E050E067E2C1CFA7
:1018B000262F44E050E067E2BCCF262F42E050E004
:1018C00067E2B7CF262F41E050E067E2B2CF262F84
:1018D00040E050E067E2ADCF262F47E050E067E2FE
:1018E000A8CF262F43E050E067E2A3CF262F43E0A6
:1018F00050E06AE29ECF262F42E050E06AE299CFA4
:10190000262F41E050E06AE294CF262F40E050E0DD
:101910006AE28FCF262F44E050E06CE28ACF242F7A
:10192000462F50E06FE285CF242F462F50E06EE225
:1019300080CF1F93CF93DF931F92CDB7DEB7142FC5
:101940009E012F5F3F4F41E050E04ADD898190E0EA
:1019500002C0959587951A95E2F781700F90DF91F7
:10196000CF911F91089547E050E061E3E2CF46E058
:1019700050E067E2DECF45E050E067E2DACF44E0D6
:1019800050E067E2D6CF42E050E067E2D2CF41E0DC
:1019900050E067E2CECF40E050E067E2CACF43E0DC
:1019A00050E067E2C6CF43E050E06AE2C2CF42E0D7
:1019B00050E06AE2BECF41E050E06AE2BACF40E0D8
:1019C00050E06AE2B6CF46E050E06BE2B2CF45E0CD
:1019D00050E06BE2AECF44E050E06BE2AACF42E0D1
:1019E00050E06BE2A6CF41E050E06BE2A2CF40E0D6
:1019F00050E06BE29ECF43E050E06BE29ACF44E0D0
:101A000050E06CE296CF462F50E060E392CF462F35
:101A100050E06FE28ECF462F50E06EE28ACFEF9219
:101A2000FF920F931F93CF93DF931F92CDB7DEB733
:101A30007C0161E27BE08EE89FE00E945E969E0161
:101A40002F5F3F4F41E050E060E0C701C9DC898172
:101A5000EADB6AE37BE08EE89FE00E9489960DE175
:101A600010E068E97AE08EE89FE00E945E9640E12F
:101A700050E0B8018EE89FE00E94489760EE79E060
:101A80008EE89FE00E945E969E012F5F3F4F41E0EF
:101A900050E0602FC701A4DC8981C5DB6AE37BE0ED
:101AA0008EE89FE00E9489960F5F1F4F0A33110551
:101AB000C1F60F90DF91CF911F910F91FF90EF90A2
:101AC0000895FF920F931F93CF93DF93FC01008142
:101AD000C181D281F8948981F02EF0948F2189837D
:101AE00078941DE7115009F182E090E082D288815C
:101AF0008023C1F3F8948A818F218A838981802B86
:101B00008983789480EE91E074D2F89489818F2152
:101B1000898386E490E06DD28881802311E009F00A
:101B200010E078948AE991E064D2812FDF91CF911F
:101B30001F910F91FF9008951F93CF93DF93FC01A6
:101B40001081C181D281912F909560FF11C0F894CE
:101B50008A8189238A838981812B89838AE090E025
:101B600048D28A81812B8A83789487E390E010C0E1
:101B7000F8948A8189238A838981812B898381E4EE
:101B800090E037D28A81812B8A83789485E090E037
:101B9000DF91CF911F912DC20F931F93CF93DF93AE
:101BA000FC011081C181D281F8948981812B8983C4
:101BB0008A81012F009580238A8383E090E019D2E7
:101BC0008981802389838AE090E013D2C881789448
:101BD00085E390E00ED21C2381E009F480E0DF91E0
:101BE000CF911F910F910895CF92DF92EF92FF92C4
:101BF0000F931F93CF93DF931F92CDB7DEB76C0186
:101C0000E62E08E010E0FF24F39461E09F2D9E2172
